:100000000C947F510C94B0510C94B0510C94B0519D
:100010000C94B0510C94B0510C94B0510C94B0515C
:100020000C94B0510C94B0510C94B0510C94B0514C
:100030000C9462850C94B0510D945A100D949E0D41
:100040000C94B0510D94C1180C94B0510C94B05153
:100050000C94B0510C94B0510C94B0510C943E7768
:100060000C94B0510C94BD630C94B0510C94B051ED
:100070000C94B0510C943DBA0C94B0510C94B05106
:100080000D94A4120C94B0510C94B0510C94B05136
:100090000C9479630C94B0510C94B0510C94B05101
:1000A0000C94B0510C94B0510D94C30A0C94B051FF
:1000B0000C94B0510D94B80A0C94B0510C94B051FA
:1000C0000C94B0510C94B0510C94B0510D94780A2A
:1000D0000C94B0510C94B0510C94B0510C94B0519C
:1000E0000C94B0510000000000000000000000006F
:1000F0000000000000000000000000000000000000
:10010000A55AB44BC82E8301D964767393ED64F07D
:10011000170349037703A203D1032D046004B90434
:10012000EE0450058C05BF05D205E205F205050673
:100130001506210631065E067C069106AF06CF063F
:10014000DE06ED06020742075F07730778078B0795
:1001500093079907A607B207BE07D307DE07EB0789
:10016000F9070808170828084608A80806092509F5
:10017000160390099909A209AB09E109000A0F0ABF
:10018000170A830A9F0AEF0A530BE40B0E0C5A0C52
:10019000A60CCF0CF60C190D750D920DCC0D410E61
:1001A0006B0EBC0EFB0E0F0F370F5F0F8C0FB40FD3
:1001B000FA0F5910B81051115611601166117411CF
:1001C0008111891191119B11A011AB11B211BC11B8
:1001D000FE11091214121C122412160328123012D6
:1001E0003B124912581266127912861291129C1211
:1001F000AF12BD12CD12DE12EF12FB120913131350
:10020000191329133413591363136A137D138213BB
:1002100016038F13A013AD13B713C313D613E5132F
:10022000F61309141914271438144B145A146314B0
:1002300072147A1483149214A2141603AC14B41416
:10024000B9141603BE14CD14D314D8141603E6142F
:10025000F114F91407150A150E1520153115581546
:1002600063156D1592159F15AE15B515C915CE15EB
:10027000D815E315F5151603FD1506160F161C16F1
:100280002A163C1649161603571667167516841655
:100290009716A416B616C616D416E416F416041746
:1002A000161725172E17391716033E1748174F171D
:1002B00055175B17A117D117E617F71709181C1860
:1002C00037187018E1180D194219B619251A711A44
:1002D000BD1AF51A121B311B371B531B941BCA1B6B
:1002E000321C751CCC1CFE1C811DC81D071E3E1E29
:1002F000541EB21ED91E391FAA1F3C20B4200F2144
:100300008A2105229222FE2207230D23132316039E
:100310001C23212380238B239023A423B623C923CA
:10032000D623E023F123032416030F2420242A24B8
:100330003A24492459246E247924862493241603CC
:100340009E24B024C324C924D624DD24F224052508
:1003500016252A253E2553256725702593259B259F
:100360001603E425F52505261226252635264926D9
:100370005B266D267E269326A226B326C326D2268A
:10038000E426F9260C27182729273C274E27632720
:10039000772788279C27B127C2271603D227DC2777
:1003A000E927FA270C281B282F28372848285A28FD
:1003B0006C287C2888289D28B2281603C728D628B0
:1003C000EB280029142925292529352949295B29C4
:1003D0006D297E299129A629B929CC29D929E22973
:1003E000F629022A0C2A4B2A8D2AC52A0F2B542BB8
:1003F000972BD42B012C372C5B2CD82C622D8B2DDA
:10040000B92DF32DFC2D0A2E192E292E542E632ED4
:10041000B92EC22EC52E004574742070726F626CA6
:10042000656D206861722075707073748F74742CA0
:10043000205A2D6E6976656C6C6572696E672075E1
:100440007466EF72732E2E2E0042E164646E69763C
:10045000656C6C6572696E67656E2066656C61645B
:10046000652E205574736B72696674656E206176B3
:100470006272EF74732E0055707076E1726D6E6962
:100480006E67206176616B74697665726164206164
:10049000762073E16B65726865747374696D65725B
:1004A0002E00472D636F64652067656E6572657207
:1004B00061642066EF7220656E20616E6E616E2051
:1004C0006E69768F2E20466F727473E17474613F8B
:1004D00000472D636F64652067656E6572657261A4
:1004E000642066EF7220656E20616E6E616E206E14
:1004F00069768F2E2056E16E6C6967656E20726595
:100500002D67656E6572657261206D6F64656C6CD8
:10051000656E206967656E2E205574736B7269660F
:1005200074656E2061766272EF74732E00472D63DE
:100530006F64652067656E6572657261642066EF41
:100540007220656E206E79617265206669726D77C2
:100550006172652E20466F727473E17474613F009E
:10056000472D636F64652067656E657265726164AF
:100570002066EF7220656E206E7961726520666973
:10058000726D776172652E2056E16E6C6967656EDB
:1005900020757070646174657261206669726D7730
:1005A0006172652E205574736B72696674656E2076
:1005B00061766272EF74732E00472D636F6465205D
:1005C00067656E6572657261642066EF7220656EA4
:1005D00020616E6E616E20736B72697661727479E0
:1005E000702E20466F727473E17474613F00472D62
:1005F000636F64652067656E65726572616420660D
:10060000EF7220656E20616E6E616E20736B726991
:100610007661727479702E2056E16E6C6967656E32
:100620002072652D67656E6572657261206D6F64FD
:10063000656C6C656E206967656E2E205574736BF2
:1006400072696674656E2061766272EF74732E0053
:10065000547279636B20708F206B6E617070656E61
:100660002066EF72206174742066EF7276E1726D1D
:1006700061206D756E737479636B6574206F636848
:1006800020666F727473E17474612E0056E16E6CB3
:100690006967656E20747279636B20708F206B6E52
:1006A000617070656E2066EF7220617474206D61F8
:1006B00074612075742066696C616D656E74006F7D
:1006C000636820747279636B20708F206B6E617029
:1006D000700053E1747420692066696C616D656E09
:1006E000740046E1726720656A206B6F7272656BF9
:1006F000740046696C616D656E7420656A206C617A
:1007000064646174008E6E6472696E67206B6F72D0
:1007100072656B74004C61646461722066E172679B
:10072000008E6E6472696E6720757466EF72642164
:1007300000B370706E612069646C6572206F6368CD
:1007400020746120626F72742066696C616D656EE1
:10075000746574206D616E75656C6C742E004C79D7
:10076000636B616465732066696C616D656E747539
:10077000746D61746E696E67656E3F0056E16E6CF4
:100780006967656E20757070677261646572612E4D
:10079000004E79206669726D7761726520766572A8
:1007A000732074696C6C67E16E676C69673A005618
:1007B000E16E74617220708F2050494E44412D7358
:1007C0006F6E64656E73206B796C6E696E67005630
:1007D000E16E6C6967656E2076E16E746100496E4A
:1007E00067656E2072EF72656C73652E0056E16E60
:1007F00074617220708F20616E76E16E6461726543
:100800002E0053746162696C206F6D6769766E6942
:100810006E677374656D70657261747572203231C4
:100820002D323643206B72E176732073616D742034
:100830006574742073747976742073746174697646
:100840002E00557466EF722058595A2D6B616C69F1
:1008500062726572696E672066EF7273742E00466D
:10086000EF7276E1726D206D756E737479636B65EE
:1008700074210046454C3A005920617673748F6E9E
:10088000642066728F6E206D696E0056E16E73741F
:1008900065720048EF676572004DE1747420736BF8
:1008A0006576686574004C8F6720736B6576686544
:1008B000740048EF6720736B6576686574005B3081
:1008C0003B305D2070756E6B7466EF72736B6A758A
:1008D000746E004A75737465726172205A004261C9
:1008E0006B73696461205BE46D5D0046726F6E74CA
:1008F000736964615BE46D5D0048EF676572207346
:100900006964615BE46D5D0056E16E7374736964E4
:1009100061205BE46D5D0053E174742074656D705B
:100920006572617475723A008E7220628F64612004
:100930005A2D7661676E61726E612068656C7420F5
:10094000757070653F004B616C69627265726172AF
:100950002058595A2E205672696420767265646553
:10096000742066EF722061747420666C797474610F
:10097000205A2D7661676E61726E612075707020ED
:1009800074696C6C20E16E6473746F7070656E2EA8
:10099000204B6C69636B61206EE17220647520E10D
:1009A00072206B6C61722E004B616C6962726572B1
:1009B0006172205A2E2056726964207672656465D1
:1009C000742066EF722061747420666C79747461AF
:1009D000205A2D736CE16461726E61207570702015
:1009E00074696C6C20E16E6473746F70702E204BB0
:1009F0006C69636B61206EE17220647520E1722086
:100A00006B6C61722E0050494E44412D6B616C69D4
:100A100062726572696E67206D6973736C79636B5E
:100A2000616465730050494E44412D6B616C69628D
:100A3000726572696E67656E20E172206B6C61721F
:100A4000206F636820616B7469762E2050494E4494
:100A500041206B616C6962726572696E67206B61BF
:100A60006E20696E616B74697665726173206920AE
:100A70006D656E796E20496E7374E16C6C6E696E93
:100A80006761722D3E50494E4441206B616C2E00CF
:100A9000466C79747461205A00466C7974746120D4
:100AA0005900466C79747461205800536B69766103
:100AB00020252E37730A5A206F66667365743A20B4
:100AC000252B312E33666D6D0A2563466F72747364
:100AD000E17474610A2563907465727374E16C6CDF
:100AE0000056E16E6C6967656E206C61646461201C
:100AF00066696C616D656E742066EF7273742E00AA
:100B000056E16C6A2066696C616D656E743A003EF0
:100B10004176627279740041747420757466EF7264
:100B2000612067756964656E206B6F6D6D657220FD
:100B30006174742072616465726120616B747565A3
:100B40006C6C61206B616C6962726572696E67734F
:100B5000696E7374E16C6C6E696E676172206F63AD
:100B6000682062EF726A61206F6D2066728F6E205E
:100B700062EF726A616E2E20466F727473E1747454
:100B8000613F0046EF7276E1726D6572206D756EA1
:100B9000737479636B652E2056E16E74612E005676
:100BA000E16E6C6967656E2073E17474206920667C
:100BB000696C616D656E7465742069206578747206
:100BC000756465726E2C20747279636B2073656432
:100BD000616E20708F206B6E617070656E2066EFA5
:100BE0007220696E6C6164646E696E672E2E0056A9
:100BF000E16E6C6967656E2073E17474206920662C
:100C0000696C616D656E74657420692064656E2021
:100C100066EF72737461206B616E616C656E20703B
:100C20008F204D4D553A6E206F6368207472796342
:100C30006B20736564616E20708F206B6E617070C5
:100C4000656E2066EF7220696E6C6164646E696E19
:100C5000672E00536B7269766172656E2062EF7267
:100C60006A617220736B7269766120757420656E9B
:100C7000207369636B7361636B6C696E6A652E20A8
:100C800056726964207672656465742074696C6C50
:100C900073206475206E6172206F7074696D616C71
:100CA0002068EF6A642E204B6F6E74726F6C6C65F7
:100CB0007261206D65642062696C6465726E61208A
:100CC000692068616E64626F6B656E20284B616C91
:100CD0006962726572696E67736B617069746C6565
:100CE00074292E0056E16C6A2074656D706572611E
:100CF00074757220736F6D207061737361722064FC
:100D0000697474206D6174657269616C2E0056E1BE
:100D10006C6A206574742066696C616D656E742000
:100D200066EF722066EF72737461206C61677265A2
:100D30007473206B616C6962726572696E67206F93
:100D400063682076E16C6A20646574206920736BA7
:100D5000E1726D6D656E796E2E004E7520736B615C
:100D6000206A6167206B616C6962726572612061E3
:100D70007673748F6E646574206D656C6C616E2023
:100D80006D756E737479636B6574732073706574BD
:100D900073206F63682076E1726D6562E16464734D
:100DA0007974616E2E005A2D6B616C696272657286
:100DB000696E672072656B6F6D6D656E64657261DB
:100DC000732E204BEF722064656E206E753F0054C9
:100DD0006120626F7274206D6574616C6C736B69F5
:100DE00076616E2066728F6E2076E1726D6562E1CB
:100DF0006464656E2E004C6967676572206D65746A
:100E0000616C6C736B69766120708F2076E1726D16
:100E10006562E16464656E3F00536520766172200F
:100E200068616E64626F6B206F6368208F7467E126
:100E30007264612070726F626C656D65742E2090B3
:100E4000746572757070746120736564616E20677B
:100E5000756964656E2067656E6F6D2061747420BE
:100E6000737461727461206F6D20736B7269766147
:100E700072656E2E00416C6C7420E172206B6C61A7
:100E800072742E20476F64207574736B7269667478
:100E900021004475206B616E20616C6C7469642064
:100EA0008F74657275707074612067756964656EA2
:100EB0002066728F6E204B616C6962726572696E1A
:100EC00067202D3E2047756964652E004F6D2064B4
:100ED00075206861722079747465726C69676172DB
:100EE00065206D6574616C6C736B69766F722C2014
:100EF0006B616C69627265726120646572617320F6
:100F000066EF72696E7374E16C6C6E696E67617224
:100F1000206920496E7374E16C6C6E696E67617252
:100F2000202D20485720696E7374E16C6C6E696ED9
:100F300067202D204D6574616C6C736B6976612E32
:100F40000052656E67EF722062E16464656E206F27
:100F5000636820747279636B20736564616E2070BE
:100F60008F206B6E617070656E2E0056696C6C2000
:100F70006475207570707265706120736973746137
:100F8000207374656765742066EF72206A757374E8
:100F900065726120617673748F6E646574206D650F
:100FA0006C6C616E206D756E737479636B65742003
:100FB0006F63682062E16464656E3F0056E16C6AAD
:100FC000206D756E737479636B7366EF7276E17280
:100FD0006D6E696E677374656D706572617475723C
:100FE00020736F6D20706173736172206469747413
:100FF000206D6174657269616C2E008E7220666965
:101000006C616D656E74206C61646461743F004E48
:101010007520736B61206A61672066EF7276E172FA
:101020006D61206D756E737479636B65742066EF06
:101030007220504C412E004A6167206B6F6D6D65C8
:10104000722061747420757466EF7261207A2D6B62
:10105000616C6962726572696E67206E752E0054EC
:1010600061206E7520626F7274207465737475747C
:10107000736B72696674656E2066728F6E206D6523
:1010800074616C6C736B6976616E2E0056E16E6CE8
:101090006967656E20746120626F72742066726188
:1010A0006B74696E7361747365726E612066EF7242
:1010B00073742E004A6167206B6F6D6D65722061DD
:1010C000747420757466EF726120656E2078797A89
:1010D0002D6B616C6962726572696E67206E752E28
:1010E0002044657420746172207570702074696C7E
:1010F0006C203234206D696E2E0046EF72737420BE
:101100006B6F6D6D6572206A616720617474207504
:101110007466EF726120736AE16C7674657374654E
:10112000742066EF7220617474206B6F6E74726F3E
:101130006C6C6572612064652076616E6C696761B4
:10114000737465206D6F6E746572696E677370720B
:101150006F626C656D656E2E0048656A2C206A6151
:101160006720E1722064696E205072757361206996
:10117000332D736B7269766172652E2056696C6CC3
:1011800020647520617474206A616720736B61202C
:101190006775696461206469672067656E6F6D209B
:1011A000696E7374616C6C6174696F6E7370726F69
:1011B00063657373656E3F0048656A2C206A6167DA
:1011C00020E1722064696E2050727573612069336A
:1011D0002D736B7269766172652E204A6167206794
:1011E0007569646172206469672067656E6F6D2040
:1011F000656E206B6F727420696E7374616C6C61C4
:1012000074696F6E7370726F636573732C2064E121
:1012100072205A2D6178656C6E206B6F6D6D6572F2
:1012200020617474206B616C696272657261732EE7
:1012300020536564616E20E17220647520726564DC
:101240006F2061747420736B726976612075742EDF
:10125000005061757300465320616B74696F6E00B6
:10126000467274732E00462E73746F707020736B09
:1012700065747400462E206175746F6C6164646ED1
:1012800000462E20736C757400536BE172617265B9
:1012900000466CE16B74666172740042E164640044
:1012A000466CE16B74636865636B004D6F64656CDD
:1012B0006C004D756E737479636B650056E16E6CEE
:1012C0006967656E206D6174612075742066696C54
:1012D000616D656E7465742066EF727374206F6360
:1012E00068207570707265706120736564616E202E
:1012F00064656E6E61208F7467E172642E004B6FBF
:101300006E74726F6C6C6572004D756E73742064D0
:1013100069612E00416C666162657400536F72747E
:10132000657261005469640053442D6B6F727400E0
:1013300056E16C6A207370728F6B004D756E73741A
:1013400079636B736279746500485720696E7374B2
:10135000E16C6C6E696E67004C6164646E696E6707
:10136000737465737400496E616B7469766572613C
:10137000207374657070657200466C7974746120B6
:1013800061786C61720054656D706572617475721C
:101390000050494E4441206B616C2E009074657280
:1013A0007374E16C6C2058595A2D6B616C2E005689
:1013B00069736120E16E646CE167656E00504944B9
:1013C000206B616C6962726572696E670042E164EC
:1013D000646E69768F206B6F7272656B740042E188
:1013E00064647974736A7573746572696E67004BAF
:1013F000616C696272657261205A004B616C69624E
:10140000726572612058595A00536AE16C767465AE
:101410007374004775696465005465737461722064
:1014200066696C616D656E74004C61646461206115
:101430006C6C610056E16E6C6967656E20746120AA
:1014400075742066696C616D656E746574206F6D6E
:101450006564656C6261727400907465727374E1A6
:101460006C6C0044EF70206F6D0046EF7273746116
:101470006C61676572206B616C69622E0056E16C6D
:101480006A004D6574616C6C736B69766F720046AF
:10149000656C73746174697374696B204D4D55008C
:1014A00046656C73746174697374696B005374611D
:1014B00074697374696B004B616C696272657269FF
:1014C0006E67004175746F6C616464612066696C5D
:1014D000616D656E74004C616464612066696C6165
:1014E0006D656E7400546120626F72742066696C61
:1014F000616D656E74004C6164642074696C6C206D
:101500006D756E737479636B0046EF726C61646421
:101510006E696E67204D4D5500496E6765742053A6
:10152000442D6B6F727400536B7269762075742052
:1015300066728F6E2053440090746572757070747B
:1015400061207574736B72696674005061757361A4
:10155000207574736B726966740047EF72206B6C50
:1015600061720053657420696E7465206B6C6172E2
:10157000740046EF7276E1726D005374E16C6C207A
:10158000696E004C697665206A75737465726120B6
:101590005A005570707265706120747279636B6562
:1015A0007400496E666F736BE1726D00456E206763
:1015B0008F6E67004C6A75640048EF6774008E6E2A
:1015C0006472612066696C616D656E7400466CEFD3
:1015D00064650046617274004D61676E65747320C6
:1015E0006B6F6D702E005A2D736F6E64206E722EAD
:1015F000004EE1747665726B00496E7374E16C6C39
:101600006E696E676172004A61004E656A005374CC
:101610006F707061207574736B72696674656E00AB
:101620004B6F6E74726F6C6C657261722066696C60
:101630000046696C656E20E172206F66756C6C7394
:1016400074E16E6469672E20466F727473E174747E
:101650006120E16E648F3F00845570706461746531
:1016600072610048757675646D656E790056E16E3D
:1016700074617220708F206D756E737479636B73F3
:101680002D206F63682062E164646B796C6E696E13
:101690006700536AE16C7674657374204F4B005396
:1016A0006AE16C7674657374737461727400557456
:1016B000627974740046726F6E742F76E16E737483
:1016C000657220666CE16B74004178656C0041784E
:1016D000656C6CE16E6764004CEF732070756C6C28
:1016E0006579008E6E646C61676520696E74652033
:1016F0006E8F7474008E6E646CE16765008E6E642C
:101700006CE167656E004B6162656C66656C0042FA
:10171000E164642F56E1726D61726500496E746513
:1017200020616E736C7574656E0056E1726D617246
:10173000652F5465726D6973746F72004B6F6E74B0
:10174000726F6C6C6572613A00536AE16C76746515
:10175000737466656C21005574736B72696674737B
:10176000666CE16B743A00486F74656E642D666C4C
:10177000E16B743A004B616C696272657261722050
:1017800068656D00536AE16C7674657374657420E6
:1017900066656C61646500416C6C74206B6F72727D
:1017A000656B74004B6F6E74726F6C6C2073656E3A
:1017B000736F726572004B6F6E74726F6C6C206821
:1017C0006F74656E64004B6F6E74726F6C6C206228
:1017D000E16464004B6F6E74726F6C6C205A2D6103
:1017E00078656C004B6F6E74726F6C6C20592D6154
:1017F00078656C004B6F6E74726F6C6C20582D6145
:1018000078656C004B6F6E74726F6C6C20E16E6467
:101810006CE167656E004B6F727420626F72747456
:10182000616765740054696C6C62616B610041753D
:10183000746F206B7261667400547973740048EFA2
:1018400067206B7261667400537472696B74005622
:1018500061726E6100496E67656E00486F74656EF7
:10186000642074656D7065726174757220E1722018
:101870003238304321208E72206D756E7374796317
:101880006B65742062797474206F6368207370E1F3
:101890006E7420656E6C6967742073706563733F46
:1018A0000046EF722062797465206176206D756E56
:1018B000737479636B652C2073650A20707275737D
:1018C000612E696F2F6E6F7A7A6C652D6D6B337335
:1018D00000504944206B616C6962726572696E6781
:1018E000206B6C617200504944206B616C696272BC
:1018F0006572696E672E005574736B7269667465E4
:101900006E20706175736164005574736B726966E3
:1019100074656E2061766272EF7473004B6F70694C
:10192000657261206465742076616C6461207370F7
:10193000728F6B65743F004D756E737479636B7352
:101940006469616D657465726E20736B696C6A653C
:1019500072207369672066728F6E20472D636F64F3
:1019600065656E2E20466F727473E17474613F007A
:10197000536B72697661726D756E737479636B65A2
:101980007473206469616D6574657220736B696C32
:101990006A6572207369672066728F6E20472D63B7
:1019A0006F6465656E2E204B6F6E74726F6C6C6524
:1019B00072612076E172646574206920696E7374C7
:1019C000E16C6C6E696E6761726E612E2055747386
:1019D0006B72696674656E2061766272EF74732E45
:1019E000004465742066696E6E7320696E67656E6B
:1019F0002066696C616D656E74206C6164646164FD
:101A00002E20466F727473E17474613F00446574F4
:101A10002066696E6E7320696E67656E2066696CFC
:101A2000616D656E74206C61646461642E20557410
:101A3000736B72696674656E2061766272EF74739F
:101A40002E004465742066696E6E7320666F727432
:101A5000666172616E646520657474206265686F8A
:101A600076206176206174742067EF7261205A2DB0
:101A70006B616C6962726572696E672E2046EF6CED
:101A80006A206D616E75616C656E2C206B617020D3
:101A900046EF727374612073746567656E2C206104
:101AA0007673204B616C6962726572696E677366EA
:101AB0006CEF64652E00536B7269766172656E20FF
:101AC00068617220696E7465206B616C6962726511
:101AD0007261747320E16E6E752E2056E16E6C6932
:101AE00067656E2066EF6C6A206D616E75616C656E
:101AF0006E2C206B61706974656C2046EF72737494
:101B0000612073746567656E2C206176736E6974ED
:101B100074204B616C6962726572696E6773666C82
:101B2000EF64652E00536AE16C7674657374206B04
:101B30006F6D6D65722061747420757466EF7261EB
:101B4000732066EF7220617474206B616C6962723D
:101B5000657261206578616B742073656E736F7256
:101B60006CEF732068656D706F736974696F6E2EAA
:101B70000047616D6C6120696E7374E16C6C6E6915
:101B80006E6761722066756E6E612E205374616E91
:101B900064617264205049442C20457374657073ED
:101BA000206574632E206B6F6D6D65722061747497
:101BB000207374E16C6C617320696E2E0056617243
:101BC0006E696E673A20628F646520736B72697606
:101BD0006172747970206F6368206D6F6465726BD9
:101BE0006F7274737479702068617220E16E647230
:101BF0006174732E005661726E696E673A20736B62
:101C0000726976617274797020E16E6472617473C6
:101C10002E005661726E696E673A206D6F64657250
:101C20006B6F72747374797020E16E647261642EEC
:101C300000536B69766100457474206F76E16E74B1
:101C400061742066656C20696E7472E16666616419
:101C5000652E004D3630302066696C616D656E749E
:101C6000627974652E204C6164646120656E206E1B
:101C7000792066696C616D656E7420656C6C657247
:101C8000206D6174612075742064656E2067616DDC
:101C90006C612E00546120626F72742064656E2046
:101CA0007574736B6A75746E612066696C616D65BD
:101CB0006E742066728F6E206672616D73696461E6
:101CC0006E206176204D4D552E0046696C616D6524
:101CD0006E742075707074E1636B746573206F7639
:101CE000E16E7461742E2053652074696C6C206100
:101CF000747420696E67656E2066696C616D656ECF
:101D00007420E172206C61646461642E204B6F6EFC
:101D100074726F6C6C6572612073656E736F72653F
:101D2000726E61206F6368206B61626C61726E61BC
:101D30002E00496E7465726E74206BEF7274696464
:101D40007366656C2E2050726F7661208F74657299
:101D50007374E16C6C61204D4D5520656C6C65723F
:101D600020757070646174657261206669726D7748
:101D70006172652E004D4D55206669726D776172F6
:101D80006576657273696F6E20E17220696E6B6FA4
:101D90006D7061746962656C206D656420736B722F
:101DA00069766172656E732046572E205570706497
:101DB00061746572696E672074696C6C20766572F7
:101DC00073696F6E20332E302E332E004D4D55200B
:101DD0004669726D7761726520696E7465726E74A2
:101DE0002066656C2C2076E16E6C6967656E208FCD
:101DF0007465727374E16C6C204D4D552E00426514
:101E000067E172742066696C616D656E74766572E7
:101E10006B74796720E17220696E74652074696C57
:101E20006C67E16E676C69677420708F2064656E03
:101E30006E6120688F7264766172612E204B6F6EC6
:101E400074726F6C6C65726120472D636F64656599
:101E50006E2066EF72207665726B74796773696EB7
:101E6000646578207574616E66EF7220696E7465C2
:101E70007276616C6C6574202854302D5434292E90
:101E8000004B616E20696E746520757466EF726137
:101E9000208F7467E17264656E2C2066696C616DD9
:101EA000656E7420E17220726564616E206C6164FD
:101EB0006461742E20546120626F727420646574B2
:101EC0002066EF7273742E004D4D5520737661724B
:101ED000617220696E7465206B6F7272656B742E0F
:101EE000204B6F6E74726F6C6C657261206B6162F7
:101EF0006C61726E61206F6368206B6F6E74616BD2
:101F00007465726E612E004D4D552073766172615D
:101F10007220696E74652E204B6F6E74726F6C6CDC
:101F2000657261206B61626C61726E61206F6368C3
:101F3000206B6F6E74616B7465726E612E004D65FF
:101F4000726120646574616C6A6572206F6E6C6981
:101F50006E652E0049646C65726E206B616E20693F
:101F60006E74652066696E6E612068656D706F7352
:101F70006974696F6E2E204B6F6E74726F6C6C6536
:101F80007261206F6D206465742066696E6E7320C7
:101F90006E8F676F7420736F6D20626C6F636B65FB
:101FA00072617220646573732072EF72656C736581
:101FB0002E004B616E20696E746520666C797474B6
:101FC000612076E16C6A6172656E20656C6C657289
:101FD0002049646C65726E2E0056E16C6A61726510
:101FE0006E206B616E20696E74652066696E6E612D
:101FF0002068656D706F736974696F6E2E204B6F0A
:102000006E74726F6C6C657261206F6D20646574A4
:102010002066696E6E73206E8F676F7420736F6DAC
:1020200020626C6F636B65726172206465737320EC
:1020300072EF72656C73652E004465742067696386
:102040006B20696E746520617474206C61646461D6
:102050002074696C6C2065787472756465726E2E7C
:1020600020496E7370656B746572612066696C617E
:102070006D656E747370657473656E7320666F72D0
:102080006D2E2046EF7266696E612073656E736F08
:10209000726B616C6962726572696E67656E2076DB
:1020A0006964206265686F762E0056E16C6A617221
:1020B000656E206B616E20696E74652072EF7261CF
:1020C0002073696720708F206772756E6420617657
:1020D000206174742046494E444120646574656BE8
:1020E000746572617220656E2066696C616D656EE3
:1020F000742E2053652074696C6C2061747420699F
:102100006E67657420676CEF6474728F6420E1728F
:1021100020692076E16C6A6172656E206F636820C9
:102120006174742046494E44412066756E6765723D
:102130006172206B6F7272656B742E0046696C6100
:102140006D656E7473656E736F726E2074726967FD
:1021500067616465732066EF7220746964696774EF
:1021600020756E646572206C6164646E696E6720B0
:1021700074696C6C2065787472756465722E4B6F2F
:102180006E74726F6C6C65726120504646452D739B
:102190006C616E67206F6368206174742073656E74
:1021A000736F726E206CE1736572206B6F72726573
:1021B0006B742E0052656D736B6976616E73206D62
:1021C0006F746F72207374616E6E6164652E20533C
:1021D000652074696C6C206174742072656D736B1A
:1021E0006976616E206B616E2072EF726120736997
:1021F00067206F6368206B6F6E74726F6C6C6572B2
:1022000061206C65646E696E6761726E612E004656
:10221000696C616D656E7473656E736F726E207438
:10222000726967676164657320696E7465206176A1
:10223000206EE1722066696C616D656E7465742054
:102240006C616464616465732075722E53652074DB
:10225000696C6C206174742066696C616D656E7464
:102260006574206B616E2072EF7261207369672064
:102270006F6368206174742073656E736F726E2073
:1022800066756E67657261722E0046696C616D6578
:102290006E7473656E736F726E20747269676761B6
:1022A00064657320696E7465206176206EE172202A
:1022B00066696C616D656E746574206C61646461DF
:1022C00064657320696E2E53652074696C6C20619F
:1022D00074742066696C616D656E746574206B61E1
:1022E0006E2072EF726120736967206F63682061EE
:1022F00074742073656E736F726E2066756E676599
:102300007261722E0046494E4441207374E16E673B
:1023100064657320696E7465206176206EE17220B9
:1023200066696C616D656E746574206C616464616E
:102330006465732075722E2046EF7273EF6B206117
:102340007474206C61646461207572206D616E75B7
:10235000656C6C742E2053652074696C6C206174FC
:10236000742066696C616D656E746574206B616E56
:102370002072EF726120736967206F636820617457
:10238000742046494E44412066756E6765726172DD
:102390002E0046494E444120747269676761646546
:1023A0007320696E74652076696420696E6C61645F
:1023B000646E696E672061762066696C616D6D651B
:1023C0006E742E2053652074696C6C2061747420C7
:1023D00066696C616D656E74206B616E2072EF7260
:1023E0006120736967206F636820617474204649B7
:1023F0004E44412066756E67657261722E00496EAB
:10240000616B7469762E0053746F7070004C616458
:102410006461004C61646461207572004967656E97
:102420000042E164646E6976656C6C6572696E6722
:10243000656E2066656C6164652E2053656E736FF2
:10244000726E2075746CEF7374657320696E7465B9
:102450002E20536B72E17020708F206D756E737437
:1024600079636B65743F2056E16E74617220708FE2
:10247000208F7465727374E16C6C6E696E672E00E8
:102480004BE16E736C6967686574004B6C61720038
:1024900090746572757070746172207574736B726C
:1024A0006966740050494E44412075707076E1723F
:1024B0006D6E696E67004B616C6962726172696E04
:1024C0006720757466EF7264004B616C69627265B7
:1024D000726172205A0042E16464206B6C61720088
:1024E00042E16464656E2076E1726D7320757070F0
:1024F0000055707076E1726D6E696E67206B6C616D
:10250000722E0055707076E1726D6E696E670053C1
:10251000656E61737465207574736B72696674009F
:102520004D4D552066656C6172004D4D552D6C61A9
:1025300064646E2066656C6172004D4D5520737445
:1025400072EF6D617662722E004D61746572696121
:102550006C7574627974656E0053656E6173746531
:10256000207574736B726966747366656C00546F62
:1025700074616C612066656C0046696C2E20617622
:1025800062726F74740054656D70657261747572F7
:1025900065720053656E736F72696E666F0058598D
:1025A0005A206B616C2E20646574616C6A657200E0
:1025B000536B7269766172656E7320495020616455
:1025C000723A006F6BE16E64004D4D5520616E7381
:1025D0006C7574656E00446174756D3A0061747455
:1025E00020746120626F72742066696C616D656E23
:1025F0007400617474206C616464612066696C614C
:102600006D656E7400547279636B20708F206B6EF1
:10261000617070656E0046EF7276E1726D657220D2
:1026200066EF7220736BE172610046EF7276E16DC6
:1026300065722066EF722075746D61746E0046EFEE
:102640007276E1726D657220666F722075746D61CD
:10265000746E0046EF7276E1726D65722066EF72FD
:10266000206C6164646E004B796C61206E65720051
:10267000457874727564657261732066696C616D0A
:10268000656E74206D65642072E174742066E17279
:10269000673F004D617461207574004175746F6C03
:1026A0006164646E696E672061762066696C616D35
:1026B000656E7420E17220616B7469762C207472EF
:1026C00079636B20708F206B6E617070656E206F08
:1026D00063682073E1747420692066696C616D65BC
:1026E0006E742E00546F74207574736B7269667407
:1026F0007374696400416E76E16E742066696C6182
:102700006D656E74005574736B7269667473746969
:1027100064004D617461722074696C6C204653656D
:102720006E736F7200466C79747461722076E16C1E
:102730006A61726500466C79747461722074696CA8
:102740006C2068656D706F730044726120696E2043
:1027500066728F6E2046494E4441004D617461722D
:102760002075742066696C616D656E7400506172CD
:102770006B657261722076E16C6A617265009074BB
:10278000657276E16E64616E64652076E16C6A6103
:10279000726500557466EF7220736BE1726E696E3C
:1027A0006700507265737361722066696C616D6554
:1027B0006E740046EF726265726564657220626CC9
:1027C00061640056E16C6A2066696C2E2073708F1C
:1027D000720054617220626F72742066696C616D60
:1027E000656E740046454C20544D43206D697373EB
:1027F0006C79636B616465730046454C20486AE1FF
:102800006C702066696C616D656E740046454C2085
:10281000496E7465726E740046454C20496E76E1CF
:102820006E74617220616E76004176736C757461AE
:102830007220666C7974746E696E6700556E64768A
:10284000696B657220736C69706E696E67004D61AB
:102850007461722074696C6C206D756E7374796329
:102860006B65004D617461722074696C6C206578D1
:10287000747275646572004D617461722074696C64
:102880006C2046494E4441004C61646420757220BE
:10289000742E2072656D736B697661004C6164649F
:1028A00061722075722074696C6C2046494E4441F7
:1028B000004B6F70706C61722075722049646C659A
:1028C00072004B6F70706C6120696E2049646C659A
:1028D00072004F4B8E4E542046454C0046494C41A9
:1028E0004D454E54425954450046494C414D454E84
:1028F000542055544153544154004C4144444120C8
:102900005552204D414E55454C4C5400465720528F
:10291000554E54494D452046454C004D4D55204699
:102920005720555044415445204B528E5653004B2E
:10293000B32046554C4C004F47494C54494754200E
:102940005645524B54594700462E20524544414E5D
:1029500020494E4C4144444154004B4F4D4D554E3F
:10296000494B4154494F4E5346454C004D4D55201F
:1029700053564152415220494E5445004D4D552029
:102980004D43552046454C004D4D5520534A8E4CE5
:1029900056544553542046454C41444500544D43FC
:1029A00020445249564552204B4F5254534C555493
:1029B0004E00544D4320554E44455253508E4E4E7A
:1029C000494E4746454C00544D43204452495645D4
:1029D000522046454C00544D4320B356455248457D
:1029E00054544E494E475346454C005641524E4969
:1029F0004E4720544D432046B352205641524D007D
:102A000049444C4552204B414E20454A20464C59A2
:102A10005454410049444C45522048454D504F5371
:102A20002046454C00568E4C4A4152452046415363
:102A3000544E4154004D49534C554B54204C414445
:102A4000444120455854522E004B4F4E54524F4C47
:102A50004C4552412046494E4441004653454E5351
:102A60004F522046B3522054494449470052454DE5
:102A7000534B49564120464153544E41540046530E
:102A8000454E534F522046494C2E2053544F5050E0
:102A9000004653454E534F522054524947474144F4
:102AA0004520454A2E0046494E44412046494C4166
:102AB0004D2E2053544F50500046494E444120540F
:102AC000524947474144455320454A00526F746577
:102AD00072617220696E746500526F746174696FFF
:102AE0006E0056E16E737420686F74656E642066C4
:102AF0006CE16B743F0046726F6E74666CE16B74D0
:102B00003F00466CE16B74746573740058595A2D1C
:102B10006B616C6962726572696E67206F6B2E20E3
:102B2000536B6576686574206B6F6D6D657220619F
:102B30007474206B6F72726967657261732061755E
:102B4000746F6D617469736B742E0058595A2D6BD4
:102B5000616C6962726572696E67206F6B2E2058B6
:102B60002F592D61786C61726E6120E172206D7950
:102B7000636B6574206C69746520736B6576612E78
:102B800020427261206A6F62626174210058595A52
:102B90002D6B616C6962726572696E67206F6B2E56
:102BA00020582F592D61786C61726E6120617220FE
:102BB00076696E6B656C72E174612E204772617488
:102BC000746973210058595A2D6B616C6962726582
:102BD00072696E67206B6F6D70726F6D657474656E
:102BE0007261642E204672E16D72652068EF206B81
:102BF000616C6962726572696E677370756E6B7411
:102C00006572206B616E20656A206E8F732E00588E
:102C1000595A2D6B616C6962726572696E67206BBF
:102C20006F6D70726F6D657474657261642E20468D
:102C300072E16D7265206B616C6962726572696EBA
:102C4000677370756E6B74206B616E20656A206EA1
:102C50008F732E0058595A2D6B616C6962726572C0
:102C6000696E672066656C6164652E2048EF676554
:102C700072206672E16D7265206B616C69627265CB
:102C800072696E677370756E6B74206B616E206510
:102C90006A206E8F732E0058595A2D6B616C6962D1
:102CA000726572696E672066656C6164652E204688
:102CB00072E16D7265206B616C6962726572696E3A
:102CC000677370756E6B74206B616E20656A206E21
:102CD0008F732E0058595A2D6B616C696272657240
:102CE000696E672066656C6164652E20536520629D
:102CF00072756B73616E7669736E696E67656E2E41
:102D00000058595A2D6B616C6962726572696E6701
:102D10002066656C6164652E204B616C696272652A
:102D200072696E677370756E6B74657220656A2068
:102D300066756E6E612E00506C6163657261206D08
:102D40006574616C6C736B69766120708F2076E1BD
:102D5000726D6562E16464656E2E00417673748FF6
:102D60006E646574206D656C6C616E206D756E733C
:102D70007479636B657473207370657473206F630B
:102D8000682062E164647974616E20686172206910
:102D90006E7465207374E16C6C747320696E20E14D
:102DA0006E6E752E2056E16E6C6967656E2066EF5B
:102DB0006C6A206D616E75616C656E2046EF727392
:102DC0007461206C616772657473206B616C6962F9
:102DD000726572696E672E00506C61636572612066
:102DE000657474207061707065727361726B2075A8
:102DF0006E646572206D756E737479636B65742093
:102E0000756E646572206B616C6962726572696E61
:102E100067656E2061762064652066EF7273746169
:102E200020342070756E6B7465726E612E204F6D4C
:102E3000206D756E737479636B657420668F6E6731
:102E400061722070617070657265742C207374E11A
:102E50006E67206176206F6D6564656C6261727467
:102E60002E0053EF6B6572206566746572206B618E
:102E70006C6962726572696E677370756E6B7420CF
:102E800066EF722062E16464656E004DE1746E6904
:102E90006E67206176207265666572656E7368EF95
:102EA0006A642066EF72206B616C69627265726998
:102EB0006E677370756E6B740052656E67EF72208B
:102EC0006D756E737479636B65742066EF72206B39
:102ED000616C6962726572696E672E204B6C696302
:102EE0006B61206EE17220647520E172206B6C6171
:102EF000722E004175746F2068656D00536BE1722E
:102F00002066696C616D656E740055746D61742026
:102F100066728F6E204D4D55004C61646461722065
:102F200066696C616D656E74004D4D552066EF727B
:102F300073EF6B206967656E3A20907465727374E5
:102F4000E16C6C65722074656D7065726174757288
:102F50002E2E2E00536F7274657261722066696C3A
:102F600065720056697373612066696C6572206BC7
:102F70006F6D6D657220696E746520617474207365
:102F80006F7274657261732E204D61782E20616EB0
:102F900074616C2066696C657220692031206D61F6
:102FA00070702066EF7220736F72746572696E675D
:102FB00020E172203130302E0053544F50504144A4
:102FC0002E00417600508F0000000000000000003D
:102FD00000000000000000000000000000000000F1
:102FE00000000000000000000000000000000000E1
:102FF00000000000000000000000000000000000D1
:1030000000000000000000000000000000000000C0
:103600000000536F6D652070726F626C656D206590
:103610006E636F756E74657265642C205A2D6C65CF
:1036200076656C696E6720656E666F72636564208F
:103630002E2E2E0001004D65736820626564206C9B
:103640006576656C696E67206661696C65642E20BD
:103650005072696E742063616E63656C65642E00E0
:10366000020048656174696E672064697361626C09
:103670006564206279207361666574792074696D70
:1036800065722E000300472D636F646520736C69BB
:1036900063656420666F7220612064696666657286
:1036A000656E74206C6576656C2E20436F6E746950
:1036B0006E75653F000400472D636F646520736C71
:1036C0006963656420666F7220612064696666655F
:1036D00072656E74206C6576656C2E20506C656129
:1036E00073652072652D736C69636520746865204D
:1036F0006D6F64656C20616761696E2E2050726920
:103700006E742063616E63656C6C65642E000500E9
:10371000472D636F646520736C6963656420666F11
:10372000722061206E65776572206669726D7761BF
:1037300072652E20436F6E74696E75653F000600DA
:10374000472D636F646520736C6963656420666FE1
:10375000722061206E65776572206669726D77618F
:1037600072652E20506C656173652075706461749C
:103770006520746865206669726D776172652E20B8
:103780005072696E742063616E63656C6C65642E43
:10379000000700472D636F646520736C696365647F
:1037A00020666F72206120646966666572656E745A
:1037B000207072696E74657220747970652E204372
:1037C0006F6E74696E75653F000800472D636F6406
:1037D0006520736C6963656420666F722061206484
:1037E0006966666572656E74207072696E74657262
:1037F00020747970652E20506C6561736520726548
:103800002D736C69636520746865206D6F64656CE9
:1038100020616761696E2E205072696E7420636149
:103820006E63656C6C65642E00090050726573737D
:1038300020746865206B6E6F6220746F20707265F3
:1038400068656174206E6F7A7A6C6520616E6420A1
:10385000636F6E74696E75652E000A00506C656149
:10386000736520707265737320746865206B6E6F6A
:103870006220746F20756E6C6F61642066696C6184
:103880006D656E74000B00616E64207072657373F9
:1038900020746865206B6E6F62000C00496E736562
:1038A00072742066696C616D656E74000D00436F03
:1038B0006C6F72206E6F7420636F72726563740038
:1038C0000E0046696C616D656E74206E6F74206CBD
:1038D0006F61646564000F004368616E6765642012
:1038E000636F72726563746C790010004C6F616471
:1038F000696E6720636F6C6F720011004368616EC0
:103900006765207375636365737321001200506CE3
:1039100065617365206F70656E2069646C657220E7
:10392000616E642072656D6F76652066696C616D8D
:10393000656E74206D616E75616C6C792E0013007C
:103940005761732066696C616D656E7420756E6C6D
:103950006F6164207375636365737366756C3F0094
:103960001400506C656173652075706772616465E1
:103970002E0015004E6577206669726D776172655D
:103980002076657273696F6E20617661696C616221
:103990006C653A00160057616974696E6720666F3E
:1039A000722050494E44412070726F626520636FEF
:1039B0006F6C696E67001700506C656173652077E6
:1039C0006169740018004E6F206D6F76652E0019C6
:1039D000005761697420666F7220757365722E2EB0
:1039E0002E001A00537461626C6520616D62696516
:1039F0006E742074656D70657261747572652032C5
:103A0000312D323643206973206E6565646564200C
:103A100061207269676964207374616E64206973E0
:103A20002072657175697265642E001B00506C65AB
:103A30006173652072756E2058595A2063616C69F4
:103A400062726174696F6E2066697273742E001CF5
:103A5000005072656865617420746865206E6F7AC5
:103A60007A6C6521001D004552524F523A001E00EB
:103A7000592064697374616E63652066726F6D208E
:103A80006D696E001F004C65667400200052696706
:103A900068740021004D6561737572656420736BF5
:103AA0006577002200536C6967687420736B6577D3
:103AB00000230053657665726520736B657700247B
:103AC000005B303B305D20706F696E74206F6666FE
:103AD00073657400250041646A757374696E6720AC
:103AE0005A002600526561722073696465205BE4A8
:103AF0006D5D00270046726F6E7420736964655BAC
:103B0000E46D5D002800526967687420736964651C
:103B10005BE46D5D0029004C656674207369646523
:103B2000205BE46D5D002A005365742074656D7040
:103B3000657261747572653A002B00417265206C84
:103B400065667420616E64207269676874205A2DFE
:103B500063617272696167657320616C6C20757056
:103B60003F002C0043616C6962726174696E67206A
:103B700058595A2E20526F746174652074686520FC
:103B80006B6E6F6220746F206D6F76652074686550
:103B9000205A2063617272696167652075702074B4
:103BA0006F2074686520656E642073746F70706533
:103BB00072732E20436C69636B207768656E206496
:103BC0006F6E652E002D0043616C696272617469CD
:103BD0006E67205A2E20526F746174652074686578
:103BE000206B6E6F6220746F206D6F766520746835
:103BF00065205A2063617272696167652075702063
:103C0000746F2074686520656E642073746F7070C3
:103C10006572732E20436C69636B207768656E2034
:103C2000646F6E652E002E0050494E444120636142
:103C30006C6962726174696F6E206661696C65643B
:103C4000002F0050494E44412063616C69627261EB
:103C500074696F6E2069732066696E697368656444
:103C600020616E64206163746976652E204974203A
:103C700063616E2062652064697361626C656420B3
:103C8000696E206D656E752053657474696E677317
:103C90002D3E50494E44412063616C2E003000455A
:103CA000787472756465720031004D6F7665205AC4
:103CB0000032004D6F766520590033004D6F7665F8
:103CC0002058003400536865657420252E37730A28
:103CD0005A206F66667365743A20252B312E336641
:103CE0006D6D0A2563436F6E74696E75650A256391
:103CF0005265736574003500506C65617365206CA6
:103D00006F61642066696C616D656E7420666972AE
:103D100073742E00360053656C6563742066696C9D
:103D2000616D656E743A0037003E43616E63656C89
:103D300000380052756E6E696E672057697A61723D
:103D4000642077696C6C2064656C657465206375AC
:103D50007272656E742063616C6962726174696FFE
:103D60006E20726573756C747320616E6420737459
:103D70006172742066726F6D207468652062656779
:103D8000696E6E696E672E20436F6E74696E75651D
:103D90003F00390050726568656174696E67206E16
:103DA0006F7A7A6C652E20506C656173652077613F
:103DB00069742E003A00506C6561736520696E73FA
:103DC0006572742066696C616D656E7420696E74CD
:103DD0006F207468652065787472756465722C2034
:103DE0007468656E20707265737320746865206BEB
:103DF0006E6F6220746F206C6F61642069742E0096
:103E00003B00506C6561736520696E736572742048
:103E100066696C616D656E7420696E746F2074687C
:103E2000652066697273742074756265206F662000
:103E3000746865204D4D552C207468656E20707235
:103E400065737320746865206B6E6F6220746F20D9
:103E50006C6F61642069742E003C005468652070AA
:103E600072696E7465722077696C6C20737461720C
:103E700074207072696E74696E672061207A696758
:103E80002D7A6167206C696E652E20526F746174A3
:103E90006520746865206B6E6F6220756E74696C46
:103EA00020796F7520726561636820746865206F82
:103EB0007074696D616C206865696768742E204351
:103EC0006865636B207468652070696374757265DA
:103ED0007320696E207468652068616E64626F6F1C
:103EE0006B202843616C6962726174696F6E206334
:103EF000686170746572292E003D0053656C6563BE
:103F0000742074656D706572617475726520776870
:103F1000696368206D61746368657320796F757279
:103F2000206D6174657269616C2E003E0053656C92
:103F300065637420612066696C616D656E742066CE
:103F40006F7220746865204669727374204C6179C1
:103F500065722043616C6962726174696F6E206181
:103F60006E642073656C65637420697420696E20CB
:103F7000746865206F6E2D73637265656E206D6564
:103F80006E752E003F004E6F7720492077696C6C6C
:103F90002063616C69627261746520646973746125
:103FA0006E6365206265747765656E207469702044
:103FB0006F6620746865206E6F7A7A6C6520616E1A
:103FC00064206865617462656420737572666163FC
:103FD000652E0040005A2063616C696272617469E9
:103FE0006F6E207265636F6D6D656E6465642E2003
:103FF00052756E206974206E6F773F004100506CDF
:10400000656173652072656D6F7665207374656593
:104010006C2073686565742066726F6D20686561D9
:10402000746265642E004200497320737465656C88
:10403000207368656574206F6E20686561746265C1
:10404000643F004300506C6561736520636865637D
:104050006B206F75722068616E64626F6F6B206198
:104060006E6420666978207468652070726F626C77
:10407000656D2E205468656E20726573756D6520C0
:104080007468652057697A6172642062792072656C
:10409000626F6F74696E6720746865207072696EF4
:1040A0007465722E004400416C6C20697320646F4B
:1040B0006E652E204861707079207072696E746927
:1040C0006E6721004500596F752063616E20616C39
:1040D0007761797320726573756D652074686520EA
:1040E00057697A6172642066726F6D2043616C69F2
:1040F00062726174696F6E202D3E2057697A617219
:10410000642E004600496620796F752068617665E7
:10411000206164646974696F6E616C207374656595
:104120006C207368656574732C2063616C696272BE
:104130006174652074686569722070726573657456
:104140007320696E2053657474696E6773202D2027
:104150004857205365747570202D20537465656C25
:10416000207368656574732E004700506C65617339
:104170006520636C65616E206865617462656420AA
:10418000616E64207468656E20707265737320744C
:104190006865206B6E6F622E004800446F20796F57
:1041A000752077616E7420746F207265706561741C
:1041B000206C617374207374657020746F20726555
:1041C00061646A7573742064697374616E636520D9
:1041D0006265747765656E206E6F7A7A6C652061B2
:1041E0006E6420686561746265643F0049005365D0
:1041F0006C656374206E6F7A7A6C65207072656886
:104200006561742074656D70657261747572652086
:104210007768696368206D61746368657320796F7E
:104220007572206D6174657269616C2E004A004977
:10423000732066696C616D656E74206C6F61646576
:10424000643F004B004E6F7720492077696C6C20EB
:1042500070726568656174206E6F7A7A6C6520662D
:104260006F7220504C412E004C00492077696C6CD5
:104270002072756E207A2063616C69627261746964
:104280006F6E206E6F772E004D004E6F7720726537
:104290006D6F766520746865207465737420707224
:1042A000696E742066726F6D20737465656C20731F
:1042B000686565742E004E00506C656173652072F0
:1042C000656D6F7665207368697070696E672068C8
:1042D000656C706572732066697273742E004F008E
:1042E000492077696C6C2072756E2078797A20632A
:1042F000616C6962726174696F6E206E6F772E20D7
:1043000049742077696C6C2074616B65207570202E
:10431000746F203234206D696E732E005000466930
:104320007273742C20492077696C6C2072756E2032
:104330007468652073656C667465737420746F208F
:10434000636865636B206D6F737420636F6D6D6F51
:104350006E20617373656D626C792070726F626C30
:10436000656D732E00510048692C204920616D2035
:10437000796F7572204F726967696E616C20507237
:10438000757361206933207072696E7465722E20B6
:10439000576F756C6420796F75206C696B65206D43
:1043A0006520746F20677569646520796F75207466
:1043B00068726F75676820746865207365747570BE
:1043C0002070726F636573733F00520048692C2040
:1043D0004920616D20796F7572204F726967696E2F
:1043E000616C205072757361206933207072696E40
:1043F0007465722E20492077696C6C20677569643A
:104400006520796F75207468726F75676820612008
:1044100073686F72742073657475702070726F6347
:104420006573732C20696E207768696368207468EF
:1044300065205A2D617869732077696C6C206265FC
:104440002063616C696272617465642E20546865D2
:104450006E2C20796F752077696C6C2062652072F4
:104460006561647920746F207072696E742E0053D8
:1044700000506175736500540046532041637469B0
:104480006F6E005500436F6E742E005600462E204E
:104490006A616D20646574656374005700462E2060
:1044A0006175746F6C6F6164005800462E207275E0
:1044B0006E6F7574005900437574746572005A000C
:1044C00046616E207370656564005B004265640040
:1044D0005C0046616E7320636865636B005D004D30
:1044E0006F64656C005E004E6F7A7A6C65005F00E9
:1044F000506C6561736520756E6C6F6164207468C3
:10450000652066696C616D656E742066697273748E
:104510002C207468656E2072657065617420746803
:10452000697320616374696F6E2E00600043686573
:10453000636B730061004E6F7A7A6C6520642E00A5
:104540006200416C706861626574006300536F7251
:104550007400640054696D650065004E6F726D6192
:104560006C00660053442063617264006700536509
:104570006C656374206C616E6775616765006800C7
:104580004E6F7A7A6C65206368616E6765006900BA
:104590004857205365747570006A004C6F616469F8
:1045A0006E672054657374006B0044697361626CBC
:1045B00065207374657070657273006C004D6F7662
:1045C000652061786973006D0054656D7065726176
:1045D00074757265006E0050494E44412063616CF1
:1045E0002E006F0052657365742058595A2063611C
:1045F0006C6962722E00700053686F7720656E647C
:104600002073746F70730071005049442063616CB3
:104610006962726174696F6E007200426564206C39
:104620006576656C20636F72726563740073004D0C
:1046300065736820426564204C6576656C696E67B9
:1046400000740043616C696272617465205A007580
:104650000043616C6962726174652058595A007632
:104660000053656C667465737400770057697A61EE
:10467000726400780054657374696E672066696CB3
:10468000616D656E740079004C6F616420416C6CE3
:10469000007A00506C656173652070756C6C206FDA
:1046A00075742066696C616D656E7420696D6D65E9
:1046B00064696174656C79007B0052657365740090
:1046C0007C0052656E616D65007D00466972737491
:1046D000206C617965722063616C2E007E005365E9
:1046E0006C656374007F00537465656C2073686546
:1046F000657473008000537570706F727400810070
:104700004661696C207374617473204D4D5500824D
:10471000004661696C207374617473008300537484
:10472000617469737469637300840043616C6962C6
:10473000726174696F6E0085004175746F4C6F61B2
:10474000642066696C616D656E740086004C6F61F3
:10475000642066696C616D656E74008700556E6CCF
:104760006F61642066696C616D656E740088004CD1
:104770006F616420746F206E6F7A7A6C65008900B7
:104780005072656C6F616420746F204D4D55008AC6
:10479000004E6F2053442063617264008B0050729E
:1047A000696E742066726F6D205344008C005265F0
:1047B00073756D65207072696E74008D005061753F
:1047C0007365207072696E74008E00536574205298
:1047D00065616479008F00536574206E6F74205298
:1047E000656164790090005072656865617400913C
:1047F0000054756E650092004C6976652061646AAC
:10480000757374205A00930052657072696E74005B
:104810009400496E666F2073637265656E00950043
:104820004173736973740096004F6E63650097005F
:10483000536F756E640098004C6F75640099004664
:10484000696C2E2073656E736F72009A0043686105
:104850006E67652066696C616D656E74009B0046CD
:104860006C6F77009C005370656564009D004D611E
:10487000676E65747320636F6D702E009E004E2FFF
:1048800041009F005A2D70726F6265206E722E007B
:10489000A0004D65736800A10053657474696E676C
:1048A0007300A20059657300A3004E6F00A400536B
:1048B000746F70207072696E7400A5004368656340
:1048C0006B696E672066696C6500A60046696C6559
:1048D00020696E636F6D706C6574652E20436F6E1A
:1048E00074696E756520616E797761793F00A70004
:1048F000845265667265736800A8004D61696E0038
:10490000A90057616974696E6720666F72206E6FC7
:104910007A7A6C6520616E642062656420636F6FD3
:104920006C696E6700AA0053656C667465737420C9
:104930004F4B00AB0053656C6674657374207374E1
:1049400061727400AC005377617070656400AD00F3
:1049500046726F6E742F6C6566742066616E7300AC
:10496000AE004178697300AF0041786973206C65CF
:104970006E67746800B0004C6F6F73652070756C63
:104980006C657900B100456E6473746F70206E6F52
:10499000742068697400B200456E6473746F7000AF
:1049A000B3004D6F746F7200B400456E6473746F22
:1049B000707300B500576972696E67206572726F17
:1049C0007200B6004265642F48656174657200B775
:1049D000004E6F7420636F6E6E656374656400B81B
:1049E000004865617465722F546865726D697374EF
:1049F0006F7200B900506C65617365206368656310
:104A00006B3A00BA0053656C667465737420657206
:104A1000726F722100BB0046696C616D656E742017
:104A200073656E736F7200BC005072696E7420669D
:104A3000616E3A00BD00486F74656E642066616EF9
:104A40003A00BE0043616C6962726174696E6720EE
:104A5000686F6D6500BF0053656C66746573742084
:104A60006661696C656400C000416C6C20636F72A4
:104A70007265637400C100436865636B696E67208B
:104A800073656E736F727300C200436865636B6910
:104A90006E6720686F74656E6400C3004368656369
:104AA0006B696E672062656400C400436865636B70
:104AB000696E67205A206178697300C50043686594
:104AC000636B696E672059206178697300C6004383
:104AD0006865636B696E672058206178697300C7E9
:104AE00000436865636B696E6720656E6473746FFD
:104AF000707300C800436172642072656D6F7665E3
:104B00006400C9004261636B00CA004175746F2084
:104B1000706F77657200CB0053696C656E7400CC62
:104B2000004D6F646500CD004869676820706F773D
:104B3000657200CE0053747269637400CF005761D0
:104B4000726E00D0004E6F6E6500D100486F7465C4
:104B50006E64206174203238304321204E6F7A7A9F
:104B60006C65206368616E67656420616E642074A3
:104B700069676874656E656420746F20737065631F
:104B8000733F00D200466F722061204E6F7A7A6CBC
:104B900065206368616E676520706C656173652070
:104BA000726561640A70727573612E696F2F6E6F22
:104BB0007A7A6C652D6D6B337300D30050494420B5
:104BC00063616C2E2066696E697368656400D40049
:104BD0005049442063616C2E00D5005072696E7498
:104BE0002070617573656400D6005072696E742020
:104BF00061626F7274656400D700436F70792073CF
:104C0000656C6563746564206C616E67756167656A
:104C10003F00D8004E6F7A7A6C65206469616D65DB
:104C200074657220646966666572732066726F6D62
:104C30002074686520472D636F64652E20436F6E76
:104C400074696E75653F00D9004E6F7A7A6C652085
:104C50006469616D65746572206469666665727306
:104C60002066726F6D2074686520472D636F6465E0
:104C70002E20506C6561736520636865636B2074DA
:104C800068652076616C756520696E207365747443
:104C9000696E67732E205072696E742063616E6353
:104CA000656C6C65642E00DA005468657265206975
:104CB00073206E6F2066696C616D656E74206C6F19
:104CC000616465642E20436F6E74696E75653F0084
:104CD000DB005468657265206973206E6F20666919
:104CE0006C616D656E74206C6F616465642E20501C
:104CF00072696E742063616E63656C6C65642E000E
:104D0000DC005468657265206973207374696C6C8B
:104D10002061206E65656420746F206D616B652075
:104D20005A2063616C6962726174696F6E2E2050E3
:104D30006C6561736520666F6C6C6F772074686555
:104D4000206D616E75616C2C206368617074657292
:104D50002046697273742073746570732C207365B8
:104D60006374696F6E2043616C6962726174696F0C
:104D70006E20666C6F772E00DD005072696E746570
:104D80007220686173206E6F74206265656E2063A7
:104D9000616C69627261746564207965742E20505B
:104DA0006C6561736520666F6C6C6F7720746865E5
:104DB000206D616E75616C2C206368617074657222
:104DC0002046697273742073746570732C20736548
:104DD0006374696F6E2043616C6962726174696F9C
:104DE0006E20666C6F772E00DE0053656C6674650E
:104DF00073742077696C6C2062652072756E207404
:104E00006F2063616C6962726174652061636375B0
:104E1000726174652073656E736F726C6573732055
:104E20007265686F6D696E672E00DF004F6C6420DD
:104E300073657474696E677320666F756E642E2077
:104E400044656661756C74205049442C2045737428
:104E5000657073206574632E2077696C6C206265C1
:104E6000207365742E00E0005761726E696E673AB8
:104E700020626F7468207072696E74657220747934
:104E8000706520616E64206D6F74686572626F6119
:104E900072642074797065206368616E6765642E42
:104EA00000E1005761726E696E673A207072696E38
:104EB0007465722074797065206368616E676564DB
:104EC0002E00E2005761726E696E673A206D6F7452
:104ED000686572626F6172642074797065206368BE
:104EE000616E6765642E00E300536865657400E4D5
:104EF00000556E6578706563746564206572726FC5
:104F000072206F636375727265642E00E5004D3622
:104F100030302046696C616D656E74204368616E47
:104F200067652E204C6F61642061206E6577206676
:104F3000696C616D656E74206F7220656A6563745B
:104F400020746865206F6C64206F6E652E00E6002B
:104F500052656D6F76652074686520656A65637457
:104F600065642066696C616D656E742066726F6D34
:104F7000207468652066726F6E74206F6620746896
:104F800065204D4D552E00E70046696C616D656EDC
:104F90007420646574656374656420756E657870EB
:104FA00065637465646C792E20456E737572652037
:104FB0006E6F2066696C616D656E74206973206C1C
:104FC0006F616465642E20436865636B2074686557
:104FD0002073656E736F727320616E6420776972DF
:104FE000696E672E00E800496E7465726E616C2010
:104FF00072756E74696D65206572726F722E2054C1
:10500000727920726573657474696E67207468655F
:10501000204D4D55206F72207570646174696E6704
:1050200020746865206669726D776172652E00E98B
:10503000004D4D552046572076657273696F6E207E
:10504000697320696E636F6D70617469626C65204D
:1050500077697468207072696E7465722046572E85
:1050600055706461746520746F2076657273696F22
:105070006E20332E302E332E00EA004D4D55204643
:1050800069726D7761726520696E7465726E616CAC
:10509000206572726F722C20706C6561736520726E
:1050A0006573657420746865204D4D552E00EB00C6
:1050B0005265717565737465642066696C616D65B0
:1050C0006E7420746F6F6C206973206E6F74206132
:1050D0007661696C61626C65206F6E2074686973BB
:1050E0002068617264776172652E20436865636B26
:1050F0002074686520472D636F646520666F722099
:10510000746F6F6C20696E646578206F7574206FA2
:10511000662072616E6765202854302D5434292E24
:1051200000EC0043616E6E6F7420706572666F7282
:105130006D2074686520616374696F6E2C206669E8
:105140006C616D656E7420697320616C7265616459
:1051500079206C6F616465642E20556E6C6F61649C
:105160002069742066697273742E00ED004D4D55F0
:10517000206E6F7420726573706F6E64696E672045
:10518000636F72726563746C792E20436865636B1C
:105190002074686520776972696E6720616E64208B
:1051A000636F6E6E6563746F72732E00EE004D4D0B
:1051B00055206E6F7420726573706F6E64696E67D0
:1051C0002E20436865636B20746865207769726977
:1051D0006E6720616E6420636F6E6E6563746F72BC
:1051E000732E00EF004D6F72652064657461696C09
:1051F00073206F6E6C696E652E00F0005468652038
:1052000049646C65722063616E6E6F7420686F6DA7
:10521000652070726F7065726C792E2043686563CB
:105220006B20666F7220616E797468696E672062A8
:105230006C6F636B696E6720697473206D6F766540
:105240006D656E742E00F10043616E2774206D6FE2
:1052500076652053656C6563746F72206F722049A8
:10526000646C65722E00F2005468652053656C65AD
:1052700063746F722063616E6E6F7420686F6D650A
:105280002070726F7065726C792E20436865636B55
:1052900020666F7220616E797468696E6720626C37
:1052A0006F636B696E6720697473206D6F76656DCF
:1052B000656E742E00F3004C6F6164696E67207434
:1052C0006F206578747275646572206661696C65BB
:1052D000642E20496E73706563742074686520665F
:1052E000696C616D656E742074697020736861709B
:1052F000652E20526566696E652074686520736549
:105300006E736F722063616C6962726174696F6E33
:105310002C206966206E65656465642E00F4005378
:10532000656C6563746F722063616E2774206D6FA6
:1053300076652064756520746F2046494E4441208F
:10534000646574656374696E6720612066696C6169
:105350006D656E742E204D616B65207375726520CE
:105360006E6F2066696C616D656E7420697320696B
:105370006E2053656C6563746F7220616E642046A5
:10538000494E444120776F726B732070726F706565
:10539000726C792E00F50046696C616D656E742043
:1053A00073656E736F722074726967676572656486
:1053B00020746F6F206561726C79207768696C6505
:1053C000206C6F6164696E6720746F2065787472F9
:1053D000756465722E20436865636B20746865721E
:1053E000652069736E277420616E797468696E67D1
:1053F00020737475636B20696E2050544645207489
:105400007562652E20436865636B20746861742043
:1054100073656E736F722072656164732070726F52
:105420007065726C792E00F60050756C6C65792091
:105430006D6F746F72207374616C6C65642E20459F
:105440006E73757265207468652070756C6C657913
:105450002063616E206D6F766520616E64206368E5
:1054600065636B2074686520776972696E672E00CA
:10547000F70046696C616D656E742073656E736FBD
:1054800072206469646E277420737769746368207E
:105490006F6666207768696C6520756E6C6F6164F5
:1054A000696E672066696C616D656E742E20456E4D
:1054B000737572652066696C616D656E74206361D9
:1054C0006E206D6F766520616E6420746865207350
:1054D000656E736F7220776F726B732E00F80046E3
:1054E000696C616D656E742073656E736F72206494
:1054F00069646E27742074726967676572207768C3
:10550000696C65206C6F6164696E672074686520E2
:1055100066696C616D656E742E20456E737572657B
:10552000207468652073656E736F722069732063E1
:10553000616C6962726174656420616E6420746874
:10554000652066696C616D656E7420726561636863
:1055500065642069742E00F90046494E4441206478
:1055600069646E277420737769746368206F666658
:10557000207768696C6520756E6C6F6164696E6711
:105580002066696C616D656E742E20547279207589
:105590006E6C6F6164696E67206D616E75616C6CB5
:1055A000792E20456E737572652066696C616D6534
:1055B0006E742063616E206D6F766520616E64206D
:1055C00046494E444120776F726B732E00FA0046B5
:1055D000494E4441206469646E277420747269677F
:1055E000676572207768696C65206C6F6164696EAD
:1055F00067207468652066696C616D656E742E2025
:10560000456E73757265207468652066696C616D9E
:10561000656E742063616E206D6F766520616E64C7
:105620002046494E444120776F726B732E00FB0079
:1056300044697361626C6500FC0053746F7000FD17
:10564000004C6F616400FE00556E6C6F616400FF7A
:105650000052657365744D4D5500000152657472BA
:1056600079000101426564206C6576656C696E673E
:10567000206661696C65642E2053656E736F7220BD
:105680006469646E277420747269676765722E207E
:10569000446562726973206F6E206E6F7A7A6C65F2
:1056A0003F2057616974696E6720666F722072656A
:1056B0007365742E00020153656E736974697669AF
:1056C0007479000301446F6E6500040152657375BF
:1056D0006D696E67207072696E7400050150494EE5
:1056E00044412048656174696E6700060143616C3E
:1056F0006962726174696F6E20646F6E6500070184
:1057000043616C6962726174696E67205A000801B6
:1057100042656420646F6E6500090142656420483B
:10572000656174696E67000A0148656174696E6736
:1057300020646F6E652E000B0148656174696E67A9
:10574000000C01546F74616C000D014C6173742086
:105750007072696E74000E014D4D55206661696C62
:1057600073000F014D4D55206C6F616420666169B7
:105770006C730010014D4D5520706F776572206677
:1057800061696C730011014D6174657269616C200F
:105790006368616E6765730012014C6173742070F9
:1057A00072696E74206661696C75726573001301AD
:1057B000546F74616C206661696C75726573001456
:1057C0000146696C2E2072756E6F75747300150139
:1057D00054656D706572617475726573001601535E
:1057E000656E736F7220696E666F0017014578747D
:1057F000727564657220696E666F00180158595A97
:105800002063616C2E2064657461696C73001901FA
:105810005072696E74657220495020416464723A16
:10582000001A01756E6B6E6F776E001B014D4D5542
:1058300020636F6E6E6563746564001C014461745F
:10584000653A001D01746F20756E6C6F616420668F
:10585000696C616D656E74001E01746F206C6F6100
:10586000642066696C616D656E74001F015072651D
:10587000737320746865206B6E6F62002001507234
:105880006568656174696E6720746F206375740064
:10589000210150726568656174696E6720746F20BC
:1058A000656A656374002201507265686561746998
:1058B0006E6720746F20756E6C6F616400230150F9
:1058C000726568656174696E6720746F206C6F61C2
:1058D00064002401436F6F6C646F776E002501468E
:1058E000696C616D656E7420657874727564696E3B
:1058F000672026207769746820636F72726563740D
:1059000020636F6C6F723F002601456A6563740007
:1059100027014175746F6C6F6164696E67206669F9
:105920006C616D656E74206973206163746976655E
:105930002C206A75737420707265737320746865A7
:10594000206B6E6F6220616E6420696E7365727485
:105950002066696C616D656E742E2E2E00280154D0
:105960006F74616C2066696C616D656E74002901ED
:10597000546F74616C207072696E742074696D6507
:10598000002A0146696C616D656E742075736564EB
:10599000002B015072696E742074696D65002C01D2
:1059A00046656564696E6720746F204653656E7343
:1059B0006F72002D014D6F76696E672073656C659F
:1059C00063746F72002E01486F6D696E67002F015E
:1059D000526574726163742066726F6D2046494E21
:1059E0004441003001456A656374696E67206669E9
:1059F0006C616D656E740031015061726B696E6728
:105A00002073656C6563746F720032015265747542
:105A1000726E696E672073656C6563746F720033B4
:105A200001506572666F726D696E672063757400F0
:105A3000340150757368696E672066696C616D65C5
:105A40006E74003501507265706172696E67206214
:105A50006C61646500360153656C656374696E67DB
:105A60002066696C2E20736C6F74003701556E6C64
:105A70006F6164696E672066696C616D656E740044
:105A8000380145525220544D43206661696C65646B
:105A90000039014552522048656C702066696C617E
:105AA0006D656E74003A0145525220496E746572FC
:105AB0006E616C003B01455252205761697420664B
:105AC0006F722055736572003C0146696E69736898
:105AD000696E67206D6F76656D656E7473003D014C
:105AE00041766F6964696E67206772696E64003E13
:105AF0000146656564696E6720746F206E6F7A7AFF
:105B00006C65003F0146656564696E6720746F20AF
:105B100065787472756465720040014665656469F4
:105B20006E6720746F2046494E4441004101556E16
:105B30006C6F6164696E6720746F2070756C6C6542
:105B400079004201556E6C6F6164696E6720746FF5
:105B50002046494E4441004301446973656E6761C4
:105B600067696E672069646C6572004401456E6701
:105B70006167696E672069646C65720045014F4B0F
:105B8000004601554E4B4E4F574E204552524F52F4
:105B900000470146494C414D454E54204348414E33
:105BA000474500480146494C414D454E5420454A21
:105BB0004543544544004901554E4C4F4144204D06
:105BC000414E55414C4C59004A0146572052554EC2
:105BD00054494D45204552524F52004B014D4D55B1
:105BE00020465720555044415445204E4545444594
:105BF00044004C0151554555452046554C4C004DEF
:105C000001494E56414C494420544F4F4C004E01DF
:105C100046494C2E20414C5245414459204C4F415D
:105C2000444544004F01434F4D4D554E4943415467
:105C3000494F4E204552524F520050014D4D552074
:105C40004E4F5420524553504F4E44494E470051F9
:105C5000014D4D55204D4355204552524F52005253
:105C6000014D4D552053454C465445535420464113
:105C7000494C4544005301544D4320445249564534
:105C8000522053484F52544544005401544D432030
:105C9000554E444552564F4C54414745204552526B
:105CA000005501544D432044524956455220524517
:105CB000534554005601544D4320445249564552D1
:105CC000204552524F52005701544D43204F5645E4
:105CD0005248454154204552524F520058015741B5
:105CE000524E494E4720544D4320544F4F20484F69
:105CF0005400590149444C45522043414E4E4F54A3
:105D0000204D4F5645005A0149444C4552204341CD
:105D10004E4E4F5420484F4D45005B0153454C4576
:105D200043544F522043414E4E4F54204D4F564501
:105D3000005C0153454C4543544F522043414E4E65
:105D40004F5420484F4D45005D014C4F4144205475
:105D50004F20455854522E204641494C4544005E40
:105D600001494E53504543542046494E4441005F3B
:105D7000014653454E534F5220544F4F20454152F8
:105D80004C5900600150554C4C45592043414E4EF2
:105D90004F54204D4F56450061014653454E534FD9
:105DA000522046494C2E20535455434B0062014625
:105DB00053454E534F52204449444E542054524967
:105DC00047472E00630146494E44412046494C4115
:105DD0004D2E20535455434B00640146494E4441D7
:105DE000204449444E542054524947474552006587
:105DF000014E6F74207370696E6E696E6700660184
:105E00005370696E6E696E670067014C6566742039
:105E1000686F74656E642066616E3F00680146724B
:105E20006F6E74207072696E742066616E3F0069D7
:105E30000146616E2074657374006A0158595A20D6
:105E400063616C6962726174696F6E20616C6C2051
:105E500072696768742E20536B65772077696C6C64
:105E600020626520636F727265637465642061757A
:105E7000746F6D61746963616C6C792E006B01588D
:105E8000595A2063616C6962726174696F6E206136
:105E90006C6C2072696768742E20582F59206178C5
:105EA00065732061726520736C696768746C792012
:105EB000736B657765642E20476F6F64206A6F622D
:105EC00021006C0158595A2063616C6962726174D7
:105ED000696F6E206F6B2E20582F59206178657383
:105EE000206172652070657270656E646963756C9F
:105EF00061722E20436F6E67726174756C61746994
:105F00006F6E7321006D0158595A2063616C69628C
:105F1000726174696F6E20636F6D70726F6D6973FB
:105F200065642E2052696768742066726F6E7420F3
:105F300063616C6962726174696F6E20706F696E03
:105F400074206E6F7420726561636861626C652E87
:105F5000006E0158595A2063616C696272617469FC
:105F60006F6E20636F6D70726F6D697365642E2044
:105F700046726F6E742063616C6962726174696FDE
:105F80006E20706F696E7473206E6F74207265611D
:105F9000636861626C652E006F0158595A20636115
:105FA0006C6962726174696F6E206661696C6564A8
:105FB0002E2052696768742066726F6E7420636168
:105FC0006C6962726174696F6E20706F696E7420A3
:105FD0006E6F7420726561636861626C652E00701B
:105FE0000158595A2063616C6962726174696F6EFD
:105FF000206661696C65642E2046726F6E74206342
:10600000616C6962726174696F6E20706F696E7421
:1060100073206E6F7420726561636861626C652EB7
:1060200000710158595A2063616C69627261746928
:106030006F6E206661696C65642E20506C656173BB
:106040006520636F6E73756C7420746865206D6174
:106050006E75616C2E00720158595A2063616C692B
:1060600062726174696F6E206661696C65642E206E
:106070004265642063616C6962726174696F6E204D
:10608000706F696E7420776173206E6F7420666F15
:10609000756E642E007301506C6561736520706CC1
:1060A00061636520737465656C2073686565742031
:1060B0006F6E20686561746265642E0074014469C6
:1060C0007374616E6365206265747765656E2074B4
:1060D0006970206F6620746865206E6F7A7A6C65CF
:1060E00020616E6420746865206265642073757237
:1060F0006661636520686173206E6F7420626565F8
:106100006E20736574207965742E20506C65617300
:106110006520666F6C6C6F7720746865206D616EAA
:1061200075616C2C206368617074657220466972B9
:1061300073742073746570732C2073656374696F56
:106140006E204669727374206C6179657220636198
:106150006C6962726174696F6E2E007501506C61BA
:1061600063652061207368656574206F66207061C7
:1061700070657220756E64657220746865206E6F3C
:106180007A7A6C6520647572696E67207468652020
:1061900063616C6962726174696F6E206F662066FC
:1061A00069727374203420706F696E74732E204985
:1061B0006620746865206E6F7A7A6C6520636174FE
:1061C00063686573207468652070617065722C2047
:1061D000706F776572206F666620746865207072D4
:1061E000696E74657220696D6D6564696174656C52
:1061F000792E007601536561726368696E6720626B
:1062000065642063616C6962726174696F6E20708D
:106210006F696E740077014D6561737572696E67A1
:10622000207265666572656E63652068656967687A
:1062300074206F662063616C6962726174696F6E4D
:1062400020706F696E74007801506C656173652011
:10625000636C65616E20746865206E6F7A7A6C6518
:1062600020666F722063616C6962726174696F6E1F
:106270002E20436C69636B207768656E20646F6EB7
:10628000652E0079014175746F20686F6D65007A25
:10629000014375742066696C616D656E74007B01E5
:1062A000456A6563742066726F6D204D4D55007CA4
:1062B000014C6F6164696E672066696C616D656E23
:1062C00074007D014D4D552052657472793A20520B
:1062D0006573746F72696E672074656D7065726145
:1062E000747572652E2E2E007E01536F7274696E66
:1062F000672066696C6573007F01536F6D6520666A
:10630000696C65732077696C6C206E6F74206265B0
:1063100020736F727465642E204D61782E204E6F4D
:106320002E206F662066696C657320696E203120AF
:10633000666F6C64657220666F7220736F72746929
:106340006E67206973203130302E00800153544F26
:10635000505045442E0081014F66660082014F6E09
:1063600000656E717565696E67202200446F6E6509
:10637000207072696E74696E672066696C65004E84
:106380006F204C696E65204E756D6265722077696D
:10639000746820636865636B73756D2C204C617342
:1063A00074204C696E653A20004E6F204368656327
:1063B0006B73756D2077697468206C696E65206EEB
:1063C000756D6265722C204C617374204C696E652A
:1063D0003A2000636865636B73756D206D69736D3A
:1063E000617463682C204C617374204C696E653A4B
:1063F00020004C696E65204E756D62657220697370
:10640000206E6F74204C617374204C696E65204E51
:10641000756D6265722B312C204C617374204C6950
:106420006E653A2000257520627974657320777255
:10643000697474656E20746F202553206174206127
:10644000646472657373203078253038780A0044AC
:106450002564202D20526561642F57726974652070
:1064600025530A003F3F00526F6D616E6100487214
:10647000766174736B69004D616779617200536C6A
:106480006F76656E63696E61004E6F72736B005359
:1064900076656E736B61004E656465726C616E64E7
:1064A0007300506F6C736B69004974616C69616E45
:1064B0006F004672616E6361697300457370616E4F
:1064C0006F6C004465757473636800436573746929
:1064D0006E6100456E676C6973680020436F756E6E
:1064E0007420583A200045303A25642052504D20FF
:1064F00050524E313A25642052504D204530403A9A
:1065000025752050524E31403A25750A0052657368
:10651000656E640025533A20256C640A25530A00F1
:106520002F2F616374696F6E3A6E6F746966696369
:106530006174696F6E2025530A0046696C616D6550
:106540006E742072756E6F75742064657465637403
:106550006564210064697361626C656400656E61E5
:10656000626C656400454550524F4D005352414D99
:1065700000442D31202D20456E646C657373206CB2
:106580006F6F700A00416374697665204578747294
:10659000756465723A203000496E76616C696420DA
:1065A0006578747275646572004D323230205325FF
:1065B00064005344207072696E74696E672062795A
:1065C00074652000257500556E6B6E6F776E2063C5
:1065D0006F6D6D616E643A2022004D32303020497B
:1065E0006E76616C6964206578747275646572207A
:1065F000007A5F6D61783A20007A5F6D696E3A20AB
:1066000000795F6D696E3A20005452494747455200
:106610004544006F70656E00785F6D696E3A2000CA
:106620005265706F7274696E6720656E6473746F03
:106630007020737461747573004D31313220636161
:106640006C6C65642E20456D657267656E6379209C
:1066500053746F702E002F2F616374696F6E3A75DB
:10666000766C6F5F7265636F766572795F72656174
:1066700064790053494C454E54004E4F524D414CA5
:10668000002553204D4F44453A2050657263656E96
:106690007420646F6E653A20256868643B207072D0
:1066A000696E742074696D652072656D61696E69CB
:1066B0006E6720696E206D696E733A2025643B20F9
:1066C0004368616E676520696E206D696E733A205C
:1066D00025640A005072696E746572537461746542
:1066E0003A2025640A00456E642066696C65206C5A
:1066F00069737400426567696E2066696C65206C19
:1067000069737400556E6B6E6F776E20256320631E
:106710006F64653A2025730A000A50494E444120AF
:1067200074656D70657261747572653A20252E31DD
:1067300066205A20736869667420286D6D293A2096
:10674000252E3366000A537465703A2025642F366F
:106750000A000A537465703A2025642F3620287386
:106760006B6970706564290A50494E444120746514
:106770006D70657261747572653A202564205A20C7
:10678000736869667420286D6D293A300A000A5AC8
:1067900045524F3A20252E33660A00737461727495
:1067A0002074656D70657261747572653A20252E6E
:1067B00031660A0025642020252E326600255320EC
:1067C000583A20252E356620593A20252E35662048
:1067D0005A3A20252E35660A00536C6565702E2EB8
:1067E0002E0045303A25642052504D0A50524E300A
:1067F0003A25642052504D0A004D3130370025367D
:106800002E32666D6D0025530A25530A25533A0A28
:1068100025533A0025332E32668100252D31342E42
:106820003134533A0A25530A252D31342E3134534D
:106830003A25332E3266810A252D31342E313453D8
:106840003A25332E3266810020203000202031008E
:10685000423A20253364202020202058643A2536EF
:10686000640A533A20253364202020202059643ABA
:106870002536640046494E44410050494E4441008B
:1068800057697A61726420656E64207374617465FF
:106890003A2025640A0053706F6F6C4A6F696E006E
:1068A0004669726D77617265005375706572504903
:1068B0004E44410048426564206F6E206C6F6164F5
:1068C00000466C617368416972004572723A484FC4
:1068D00054454E442046414E204552524F52002FBF
:1068E0002F616374696F6E3A726573756D656400CC
:1068F0002F2F616374696F6E3A726573756D6500F1
:106900002F2F616374696F6E3A7265616479002F2D
:106910002F616374696F6E3A6E6F745F7265616444
:1069200079002F2F616374696F6E3A63616E6365DE
:106930006C004F4B004C434420737461747573209A
:106940006368616E6765640053442063617264200C
:1069500072656C6561736564002F2F616374696F84
:106960006E3A7374617274004D3834004D373032B2
:10697000004732382057004D3530300042616420E6
:10698000696E7465727275707400576174636864BF
:106990006F672074696D656F7574005374617469F5
:1069A00063206D656D6F7279206861730A62656539
:1069B0006E206F7665727772697474656E004649F1
:1069C000524D57415245204352415348210A437288
:1069D00061736820726561736F6E3A0A00202050FF
:1069E0006C616E6E65724275666665724279746539
:1069F000733A20002046726565204D656D6F72798F
:106A00003A2000207C20417574686F723A20002083
:106A10004C61737420557064617465643A20002081
:106A2000536F6674776172652052657365740020D8
:106A30005761746368646F672052657365740020E2
:106A400042726F776E206F757420526573657400A3
:106A50002045787465726E616C20526573657400B0
:106A6000506F7765725570006572726F7220777221
:106A70006974696E6720746F2066696C6500446F85
:106A80006E6520736176696E672066696C652E009D
:106A90006F6B0046696C616D656E7400312F390053
:106AA000880020746F6F206C6F6E67206578747239
:106AB0007573696F6E2070726576656E74656400BB
:106AC00020636F6C6420657874727573696F6E20D3
:106AD00070726576656E746564004D6F76652061D1
:106AE000626F72746564004572723A5052494E5436
:106AF0002046414E204552524F52002563253364B3
:106B00002F256481005A25362E32662563005A20CF
:106B100020202D2D2D2000862533642525002D2DA8
:106B20002D252500253364252500205344002020F1
:106B3000200020484F002046524D2000872D2D3A3E
:106B40002D2D2020008725337568202563256300BF
:106B500087253032753A2530327525632563002F3D
:106B60002F616374696F6E3A706175736564002F8D
:106B70002F616374696F6E3A706175736500447557
:106B80006D7020746F2073657269616C0068656C4C
:106B9000702E707275736133642E636F6D00666F53
:106BA00072756D2E707275736133642E636F6D0034
:106BB000707275736133642E636F6D004D373031C1
:106BC0000025533A0A2531382E32666D200A2553A6
:106BD0003A0A2531306C64642025303264682025FF
:106BE0003032646D0025533A0A2531382E32666DF5
:106BF000200A25533A0A2531306C6468202530324A
:106C0000646D202530326473004D65617375726563
:106C10006420736B6577733A2025662025660A0029
:106C200046697474696E67206661696C6564203DAD
:106C30003E2063616C6962726174696F6E20666187
:106C4000696C65642E0A0043616C696272617469E3
:106C50006F6E20737563636573732E0A00416C6CED
:106C600020342063616C6962726174696F6E207098
:106C70006F696E747320666F756E642E0A00312F13
:106C80003400312F3400312F390050727573612078
:106C90006933204D4B322E35204F4B2E005344206C
:106CA00063617264206F6B006F70656E526F6F74FA
:106CB000206661696C656400766F6C756D652E6920
:106CC0006E6974206661696C656400534420696E66
:106CD0006974206661696C006F70656E2066616919
:106CE0006C65642C2046696C653A200043616E6EC9
:106CF0006F7420656E746572207375626469723A90
:106D000020004D363030004D3234004D32332025D6
:106D100073005072696E7465722073746F70706561
:106D2000642064756520746F206572726F72732EB3
:106D3000205375706572766973696F6E2072657124
:106D400075697265642E0047312045252D2E336606
:106D5000204632373030004D383300084AD73B3BAD
:106D6000CE016E84BCBFFDC12F3D6C74319ABD56FF
:106D7000833DDA3D00C77F11BED9E4BB4C3E916B29
:106D8000AAAABE000000803F05A84CCDB2D44EB9DF
:106D90003836A9020C50B9918688083CA6AAAA2ABE
:106DA000BE000000803F07634236B79BD8A71A3960
:106DB000685618AEBAAB558C1D3CB7CC5763BD6D49
:106DC000EDFD753EF6177231BF000000803F0800F0
:106DD0000000BE922449123EABAAAA2ABECDCCCC5A
:106DE0004C3E00000080BEABAAAAAA3E00000000F4
:106DF000BF000000803F0000000000084178D3BBC6
:106E00004387D1133D190E3CC3BD4282AD2B3E6872
:106E1000EC8276BED98FE1A93E4C80EFFFBE01C463
:106E2000FF7F3F00000000000C94B9EA0C9457C6A5
:106E30000D943A040C941BBB0C94D4CE0C9419D929
:106E40000D94639D0C94B2FC0C94C7E70C9485C11F
:106E50000D9488970C9485CE0C9490770C949AD8C6
:106E60000C945D770D94E3240C9414EA0C9437BBD6
:106E70000C949ED10C9403D20C9442CE0C94A6D8C0
:106E80000C942CCC0D94FF140C9418BD0C94D9CEFA
:106E90000D9410090C94E4770D940D0B0D940B0DCB
:106EA0000C94C6730D94949D0D94AB240D94B8016D
:106EB0000C9459C90C9423BB0D9456240C9497BD83
:106EC0000C9448CD0D9414050D94DB240C94D0EA59
:106ED0000C9452CD0C94C6E30C94CCCD0C94C7C149
:106EE0000C94ABF70C9442E70C94B4CD0C9443BBD8
:106EF0000D942A240C9466C20D9418050C949AFCE7
:106F00000C94C0CD0C944AFC0C9410D90C949BF6B4
:106F10000D947F9D0D94AD230D94829D0C9450BED5
:106F20000C94A3F70C94E8F40C94E0D10C94A4DC3A
:106F30000C940CBD0C9471CE0C94C3CD0D949E306A
:106F40000C94CCD10C9473BE0C943CC60D94229737
:106F50000C9461BD0C9421D20C9480BD0C9434F639
:106F60000D9481970D9469020C9477770C9417D245
:106F70000C944EC00D9464970D94CF010D94C70CE2
:106F80000C9431D90D94F4230C9436BB0D94EB245E
:106F90000C945ACE0C94C4D10C947EC40C942DDD68
:106FA0000C9452CE0D94F5040D948E040C9440EA8A
:106FB0000C944BBD0C9489C10D9478010C9439C983
:106FC0000C944AEA0C9431BB0D946B0C0C9480C168
:106FD0000D94C5230C9447BF0C9400BB0C9467C15F
:106FE0000C94F2D40C94F9D10C949FF60C9404D91F
:106FF0000C9441BD0C94EEF40C943ABE0D946F08C1
:107000000C9476DC0C9410E90C940BBB0C9413D903
:107010000D94CB240C943FBB0C94E4EA0D948A2489
:107020000C9404BB0C944ACE0D941D9D0C946CC121
:107030000D94869D0C94C7EA0C9490DC0C94EAD1D4
:107040000C9458E70C94B7CD0C949EEA0C94D2772C
:107050000C9411BB0C9462C10C9482770D94932410
:107060000C94AFEA0C9499F70C94E6C60C9457BDB7
:107070000C94B5EA0C94BACD0D9459240C942DBB04
:107080000C94F3BF0D94A3240C94A6770C9448BBE6
:107090000D9432010C94AFBC0C9480CE0D948D24D1
:1070A0000C94C0C50C945FC20C941EBE0D9409973D
:1070B0000C949FF70D94CD090D949B240C942A6495
:1070C0000C9429BB0C942DBD0C9475BD0C94AF771A
:1070D0000C942BD20D94F7230C94AABD0D945C2430
:1070E0000C9424F70D9484970C9423C60C9458DDCB
:1070F0000C944EC60C9476C10C9453D50C9445C692
:107100000D9486020C94F6BA0C9474C20C94BABC1A
:107110000C9416D90C94C1F70C947DCD0C9430E4EA
:107120000C9482CE0C9425D90C94F8C30C94CBFB10
:107130000C94DD730D94ED230C94FCBA0C946DC289
:107140000D94D3240D94250A0C9408BB0C9411C003
:107150000C9457BE0D94FD0D0C9405790C94D0CA77
:107160000D947A020D941E020C94BED80C947BC22E
:107170000D94270D0C94A9BC0C946BBD0C9499D163
:107180000C940DD20C947BC10C9484D60D945D02AA
:107190000C9434EA0D94EA230C94B2D10C94BCD133
:1071A0000C9466CE0C9423BD0C94A7F70C9467E165
:1071B0000C9441D70C9471C10D94C3240D94902468
:1071C0000C94FDBC0C94D6D10C941FBB0C94B3CC86
:1071D0000C9435C20C9415BB0C94A8D10C94BDCD65
:1071E0000D949F630C941FF80C941ECF0D94B32440
:1071F0000C9412CA0C941A7B0C9435FC0D94FA0C66
:107200000D9489020D94BB240D947E0C0C9484EA99
:107210000C9491D10C9420F90C94F1BC0C9437BDD2
:107220000C943BBB0D948F9D6E616E00696E660081
:1072300000407A10F35A00A0724E18090010A5D42D
:10724000E80000E87648170000E40B54020000CA8A
:107250009A3B000000E1F5050000809698000000D0
:1072600040420F000000A08601000000102700002F
:107270000000E803000000006400000000000A00B5
:10728000000000000100000000002C76D888DC67B8
:107290004F0823DFC1DFAE59E1B1B796E5E3E45310
:1072A000C63AE651997696E8E6C28426EB898C9B2D
:1072B00062ED407C6FFCEFBC9C9F40F2BAA56FA5CD
:1072C000F490055A2AF75C936B6CF9676DC11BFC4F
:1072D000E0E40D47FEF520E6B500D0ED902E03006A
:1072E000943577050080841E080000204E0A0000B7
:1072F00000C80C333333330F986E12831141EF8D76
:107300002114893BE65516CFFEE6DB18D1844B38B5
:107310001BF77C1D901DA4BBE424203284725E22E6
:107320008100C9F124ECA1E53D272200002045534E
:107330005000204E535000204F464600204F4E0034
:107340005056303100205B4D505D2000256920688B
:107350006F757273202569206D696E757465730091
:1073600052582074696D656F7574004D333130006B
:107370004D313132004D3131300046756C6C205248
:1073800058204275666665720053657474696E674D
:10739000732053746F7265640053746F7265642058
:1073A00073657474696E677320726574726965764B
:1073B00065640048617264636F6465642044656657
:1073C00061756C742053657474696E6773204C6FBB
:1073D0006164656400563200000000C8420000C8C5
:1073E000420000C843000005430000484300004835
:1073F00043000040410000F042E8030000E80300C1
:1074000000C80000008813000000409C4400409C1D
:10741000440000000000000000204E00000000209A
:107420004100002041CDCCCC3E0000904000000047
:10743000000000000000000000CDCCCC3E3D0A81E1
:1074400041FF08433EB099AB438F42FC42E65A34B9
:107450003F4C62B045000000000040400000344254
:10746000000000000000000000000041000000E0FB
:107470003F00002C4300002C43000040410000F07E
:1074800042C0030000C0030000C8000000881300D1
:10749000001010101000409C440000803F000000CD
:1074A0003F19140000002030780020307800657209
:1074B000726F723A2000443233202D20656D657260
:1074C00067656E63792073657269616C2064756DA0
:1074D0007000437573746F6D004E796C6F6E504120
:1074E00000536174696E20200054657874757200D1
:1074F000536D6F6F746800312E3000312E3500559A
:107500004E4B4E4F574E004C413130433A204C6960
:107510006E65617220416476616E6365206D6F6493
:10752000653A20004C413130433A2041646A75731A
:1075300074656420452D4A65726B3A200093ED64B2
:10754000F03E0FA8AF00480069960000DF602555A7
:107550005887680427F2E0005E3403CC1960F33CDE
:107560000EF88F00DB08029492003E1C079A8700F9
:10757000E524008528527E06001BE4007E78127008
:10758000787061F812788F884178427078706178ED
:107590002570787061F850788F88D1F0252707879B
:1075A00061F025278F88412C0D27AA50D1BC0707F1
:1075B000871161BE788F881141785270787061F8B8
:1075C00052788F88412012788870632052788870B2
:1075D00063485278888743031117997064181278AA
:1075E000F870654412F8F8F045184278F87065189C
:1075F0002578F87065185278F87065185078F8702A
:10760000650C078F872365A20F8F8F114500120627
:10761000227069001207222749002506227069009E
:10762000250722274900120622276C026236A27023
:107630006C40456C44704C03622222706C43888815
:1076400088F04C7812BC88806E7852BC88806E3886
:10765000127888706F78127888874F3842788870EF
:107660006F38257888706F3A0079AC786F3D079A4B
:10767000AC786F7850788887EF39497888706F08D0
:1076800052BC8880729852F88F985220127870F00D
:107690007348127863875320527870F07348527899
:1076A0006387531007870F2473127863872453600E
:1076B000699A988BE22304E4443074104E444324C6
:1076C000747C12888960753C5088887055782528AC
:1076D0008960757949088960753C12887070790CE9
:1076E00012885222594412F124F07A4452F124F0C3
:1076F0007A8C52F0368F5A4420F124F07A004014EC
:1077000054CDCCCC3D0AD7233C17B7D13877CC2BFE
:10771000329595E6241FB14F0A000020410000C8B1
:107720004200401C4620BCBE4CCA1B0E5AAEC59D32
:10773000744E414E494E4600007A430000524300C9
:1077400000524300000000000080C09A99193E00DA
:10775000000000000080C09A99193E20503A002095
:1077600042403A0020403A00202F002054303A0096
:10777000202F0020423A00202F00543A0025534584
:10778000786365737369766520626564206C6576DD
:10779000656C696E6720636F7272656374696F6E82
:1077A0003A202569206D6963726F6E730A00426525
:1077B00064206C6576656C696E67206661696C65CE
:1077C000642E20546F6F206D756368207661726936
:1077D0006174696F6E2066726F6D20656570726F7F
:1077E0006D206D65736800426564206C6576656C1C
:1077F000696E67206661696C65642E2053656E73DF
:107800006F722074726967676572656420746F6F48
:1078100020736F6F6E002020004D65617375726577
:107820006420706F696E74733A005A2073656172D8
:107830006368206865696768743A20352E30660091
:107840004E756D20582C593A20372C37004D6573F2
:107850006820626564206C6576656C696E67206E71
:107860006F74206163746976652E0020453A0020AC
:107870005A3A0020593A0020453A00205A3A00204E
:10788000593A00583A00202D3E200053706F6F6C1B
:107890004A6F696E3A20002C2000496E616374695A
:1078A000766974792053687574646F776E004B49FC
:1078B0004C4C45442E005072696E746572206861AC
:1078C0006C7465642E206B696C6C28292063616C74
:1078D0006C656421005A206C6976652061646A7564
:1078E0007374206F7574206F662072616E67652EE9
:1078F0002053657474696E6720746F20302E2043A6
:107900006C69636B20746F20636F6E74696E75654C
:107910002E005A206C6976652061646A7573742044
:107920006F7574206F662072616E67652E205365D7
:107930007474696E6720746F20300020453A3020DF
:10794000423A00543A00627573793A207061757357
:10795000656420666F7220696E707574006275735D
:10796000793A2070617573656420666F7220757353
:10797000657200627573793A2070726F6365737314
:10798000696E670073657269616C2064756D702043
:1079900000496E76616C6964205420636F64652EC3
:1079A000004475706C696361746520542D636F6465
:1079B000652069676E6F7265642E00416476616E42
:1079C0006365204B3D004B206F7574206F6620610E
:1079D0006C6C6F7765642072616E676521004D4B3A
:1079E000322E35004D4B322E354D4D5532001A4F4B
:1079F000FA002533642F2533640025336400200A00
:107A0000200A200A200025534172632053657474B4
:107A1000696E67733A20503A4D6178206C656E67E5
:107A20007468286D6D2920533A4D696E206C656E1F
:107A300067746820286D6D29204E3A436F72726515
:107A40006374696F6E7320523A4D696E2073656777
:107A50006D656E747320463A5365676D656E747319
:107A60002F7365632E0A255320204D323134205068
:107A7000252E32662053252E3266204E2564205254
:107A80002564204625640A00255346696C616D65AE
:107A90006E742073657474696E67733A20446973F9
:107AA00061626C65640A00255346696C616D656EA0
:107AB000742073657474696E67733A0A25532020C5
:107AC000204D3230302044252E32660A0025535294
:107AD0006574726163743A20533D4C656E677468D7
:107AE00020286D6D2920463A537065656420286D05
:107AF0006D2F6D29205A3A205A4C69667420286DE2
:107B00006D290A25532020204D3230372053252E51
:107B100032662046252E3266205A252E32660A25E8
:107B2000535265636F7665723A20533D457874729F
:107B300061206C656E67746820286D6D2920463A57
:107B4000537065656420286D6D2F6D290A255320BB
:107B500020204D3230382053252E32662046252EE7
:107B600032660A25534175746F2D526574726163D4
:107B7000743A20533D3020746F2064697361626CE5
:107B8000652C203120746F20696E74657270726587
:107B90007420657874727564652D6F6E6C79206DD4
:107BA0006F7665732061732072657472616374739C
:107BB000206F72207265636F7665726965730A253E
:107BC000532020204D323039205325640A0025539C
:107BD00050494420686561746265642073657474FB
:107BE000696E67733A0A25532020204D33303420C4
:107BF00050252E32662049252E32662044252E320D
:107C0000660A0025535049442073657474696E6791
:107C1000733A0A25532020204D3330312050252E31
:107C200032662049252E32662044252E32660A000F
:107C3000255353746570732070657220756E697476
:107C40003A0A255320204D39322058252E326620FD
:107C500059252E3266205A252E32662045252E3291
:107C6000660A25534D6178696D756D20666565649A
:107C7000726174657320286D6D2F73293A0A25533C
:107C800020204D3230332058252E32662059252EA3
:107C90003266205A252E32662045252E32660A2568
:107CA000534D6178696D756D20616363656C6572B4
:107CB0006174696F6E20286D6D2F7332293A0A2521
:107CC0005320204D3230312058256C752059256CB9
:107CD00075205A256C752045256C750A255341631E
:107CE00063656C65726174696F6E3A20503D7072A5
:107CF000696E742C20523D726574726163742C201D
:107D0000543D74726176656C0A255320204D3230E3
:107D1000342050252E32662052252E3266205425DE
:107D20002E32660A2553416476616E63656420765F
:107D300061726961626C65733A20533D4D696E20D2
:107D4000666565647261746520286D6D2F73292CDA
:107D500020543D4D696E2074726176656C206665B5
:107D600065647261746520286D6D2F73292C204223
:107D70003D6D696E696D756D207365676D656E74B7
:107D80002074696D6520287573292C20583D6D611C
:107D900078696D756D205859206A65726B20286D61
:107DA0006D2F73292C20205A3D6D6178696D756D9A
:107DB000205A206A65726B20286D6D2F73292C2044
:107DC00020453D6D6178696D756D2045206A65724D
:107DD0006B20286D6D2F73290A255320204D3230DA
:107DE000352053252E32662054252E32662042251A
:107DF0006C752058252E32662059252E3266205A61
:107E0000252E32662045252E32660A2553486F6D91
:107E100065206F666673657420286D6D293A0A25A2
:107E20005320204D3230362058252E3266205925D9
:107E30002E3266205A252E32660A004361703A259A
:107E4000533A25630A0050525553415F4D4D553208
:107E500000455854454E4445445F4D32300041552D
:107E6000544F5245504F52545F504F534954494F0D
:107E70004E004155544F5245504F52545F46414E6B
:107E800053004155544F5245504F52545F54454D45
:107E900050000044656C6574696F6E206661696CA2
:107EA00065642C2046696C653A200046696C652043
:107EB00064656C657465643A004E6F7420534420A9
:107EC0007072696E74696E67005072696E742073A7
:107ED00061766564005344207072696E742070612D
:107EE00075736564002533642F253364006676005E
:107EF0007468780050524E0022283229006E6F209C
:107F000076616C696420636F6D6D616E64007A6583
:107F1000726F72697A656400666163746F7279204A
:107F2000726573746F72656400696E6465782C2085
:107F300074656D702C2075737465702C20756D00E0
:107F400050494E44412063616C20737461747573B1
:107F50003A2000503A005761697420666F722050D1
:107F6000494E4441207461726765742074656D7078
:107F7000657261747572653A0020410020500020DE
:107F80004200204C00205200205A00204E4F542026
:107F9000494E495449414C495A4544005368656526
:107FA000742000205A2056414C5545204F555420EE
:107FB0004F462052414E474500496E76616C6964D8
:107FC0002073686565742049442E20416C6C6F777E
:107FD00065643A20302E2E004155544F004C414EDE
:107FE000472053454C20464F524345440020643AB5
:107FF0000020693A0020703A0020643A0020693A73
:108000000020703A00256925250A00256925250AE2
:108010000022283129002F2F0000204558545255A6
:108020004445525F434F554E543A3100204D414331
:1080300048494E455F545950453A00312E30002092
:108040006261736564206F6E204D61726C696E2091
:108050004649524D574152455F55524C3A687474E7
:1080600070733A2F2F6769746875622E636F6D2F76
:10807000707275736133642F50727573612D466928
:10808000726D776172652050524F544F434F4C5F71
:1080900056455253494F4E3A003030303030303030
:1080A0003030005F0038323337002B004649524DE4
:1080B000574152455F4E414D453A50727573612D9F
:1080C0004669726D7761726520004D3131332053FE
:1080D000006F6B200020636D2E00206D696E200004
:1080E000535441545320006E2F61003F546F736806
:1080F00069626120466C61736841697220476574EA
:108100004950206661696C65640A00000125301DD4
:108110000CFF24311C0BFF232F1B0A17FF04062220
:108120002B1A03363535382569206D696E2C2025CC
:10813000692073656300496E76616C6964204D2027
:10814000636F64653A2025730A0050494E4441200C
:1081500070726F62652063616C6962726174696FCD
:108160006E207374617274004E6F2050494E44410A
:1081700020746865726D6973746F72007365740042
:108180006E6F7A7A6C65004D424C004652004C7A14
:10819000004C616E6700315F37356D6D5F4D4B325E
:1081A000352D52414D426F3130612D453344763685
:1081B00066756C6C0052657600332E31342E312D8D
:1081C000383233370046697200534E20696E76614B
:1081D0006C696400534E005245534554004D4D5553
:1081E0005245530075766C6F0046414E0046414E35
:1081F00050494E54535400505255534100252E318E
:108200003053200025346400473120583130205944
:10821000313830204634303030004731205A313048
:10822000204631333030004D313430205330004D52
:1082300031303420533000473120452D302E303737
:10824000352046323130300047312046343030302E
:10825000004D323034205331303030004731205A15
:108260003520463732303000473120452D312E350C
:108270002046323130300047393000473120583500
:10828000204534204631303030004731205A302EDE
:1082900032204631303030004731205835352045C6
:1082A000323520463134303000473120592D3220CC
:1082B000463130303000473120583234302045329A
:1082C0003520204632323030004731205A302E33AC
:1082D0002046313030300047312058353520453880
:1082E0002046323030300047312058352045323971
:1082F000204631383030004731205835352045325E
:108300003920463130373300473932204530004775
:108310003238004D313039004D31393000252D31A2
:10832000322E313253252B382E3166004578747247
:10833000756465723A0025632531372E32666D6D9E
:1083400000583A00593A005A3A002563252D313336
:108350002E313353252B352E3366002533750050CF
:10836000494E44412063616C6962726174696F6E49
:10837000206661696C65642E20436F6E74696E754A
:10838000652077697468207072657373696E672001
:10839000746865206B6E6F622E0050494E44412018
:1083A00063616C6962726174696F6E20646F6E657F
:1083B0002E20436F6E74696E75652077697468202E
:1083C0007072657373696E6720746865206B6E6F79
:1083D000622E005A30005A3100593000593100588D
:1083E0003000583100456E642073746F70732064E0
:1083F00069616700473830004D3435004D34352011
:108400005A00473736004D37303120503000576919
:108410007A6172642073746174653A2025640A007D
:108420004578706572696D656E74616C00302E38C8
:108430003000302E363000302E343000302E3235C1
:108440000044697361626C65206661726D206D6FB6
:108450006465005265736574204D4D55004D4D5552
:10846000004D3434004739390044697361626C65EA
:10847000206661726D206D6F64653F004732382061
:108480005859004D20383400852E2E002533642F96
:1084900030002533642F30006C63645F73656C6655
:1084A000636865636B5F617869732025642C2025A0
:1084B000640A00486F74656E6400426564005A0087
:1084C000590058002D2D2D2D2D2D2D2D2D2D2D2DDF
:1084D0002D2D2D2D2D2D2D2D00537570657250498C
:1084E0004E44413A00F96737822F8227821A820868
:1084F00082473120582564205925642045252D2E9A
:108500003566004731204631303830004731205A37
:10851000252D2E3366204637323030004731205823
:10852000353020593135350008837782576D6882A0
:108530005C82518248824731205825642045252D90
:108540002E336620463130303000F782E782D78202
:10855000C9820883B682A98298828A827B82542546
:1085600064004731205A302E3420463130303000FC
:10857000473120592D3320463130303000F967180B
:108580008313830F8308834D3834205859004D31AD
:1085900030392053323830004731205831323520BD
:1085A0005A32303020463130303000496E76616CBE
:1085B0006964205049442063616C2E207265737594
:1085C0006C74732E204E6F742073746F7265642008
:1085D000746F20454550524F4D2E004D33303120A1
:1085E00050252E32662049252E32662044252E3213
:1085F00066004D333033204530205325337500520B
:108600004300444556004245544100414C504841C6
:108610000000002100240027002A002D0030003334
:108620000001010000040107010A010000220025E9
:108630000028002B002E003100340002010000054C
:108640000108010B01000020002300260029002C56
:10865000002F00320000010000030106010901059E
:10866000050505070508080808020202020A0A08AB
:1086700008040404040101010101010101030303D1
:108680000303030303040707070C0C0C0C0C0C0C6E
:108690000C0202020206060606060606060B0B0B75
:1086A0000B0B0B0B0B07070A0A0A0A0A0A0505053A
:1086B00004040408080102102020080810204010BB
:1086C0002040800201020108040201010204081096
:1086D00020408080402010080402018004020180B4
:1086E00040201008040201080402010102040810DD
:1086F00020408001020408102040801008040880F7
:10870000102040044080102040048000000A0B022A
:10871000090C0D0E08070304010000000000000012
:108720000000000000000000000000000000000049
:108730000000000000000012111000000000000006
:108740000000000000000000000000000000000029
:108750000000000000000000000000000000000019
:1087600000332E31342E31000A204F726967696E52
:10877000616C2050727573612069330A202020508B
:10878000727573612052657365617263680A253280
:10879000302E3230530053706F6F6C4A6F696E2009
:1087A000697320006164635F696E697400200A2048
:1087B0000A200A2000416C6C2044617461005365FA
:1087C00072766963652070726570005368697070B5
:1087D000696E672070726570005374617469737498
:1087E000696373004C616E6775616765004552414E
:1087F00053494E4720616C6C20646174610046618E
:1088000063746F727920524553455400505255534A
:1088100041334446570003000E00010040000300AE
:10882000020000000400556E6B6E6F776E003139E8
:1088300037302D30312D30312030313A30303A3030
:10884000300020332E31342E312D383233375F3023
:108850003030303030303030007374617274004D1D
:10886000323900252D392E39535B00200A200A2089
:108870000000004842000058419A998D413333531B
:10888000404D4D55323A004D494E54454D502042D1
:108890004544206669786564004D494E54454D5005
:1088A00020484F54454E44206669786564004578F9
:1088B00072656D65207370616E206F6620746865E7
:1088C000205A2076616C756573210025642F39006C
:1088D0004D4D55323A002533640018010419020A3F
:1088E000CD555755DD547054275495531D53B552EB
:1088F00066524652FA514652E351E351E351E35175
:10890000E351E351E351E351E351E351E351E351C7
:10891000E351E351E351E351E351E351E351E351B7
:10892000E351E351AC516B512151AE5079502F506E
:10893000E54F874F4E4F0C4FEF4E010101010101F2
:108940000102710171013232320303030303030395
:108950000303030303030303030303039393243871
:10896000039303010256036500660067006800690F
:10897000006A006B006C00730074007D007E00C90B
:1089800000D300DD00CA00D400DE002D0137014114
:10899000012E01380142012F013901430130013A12
:1089A00001440131013B014501320191019201F580
:1089B00001F601F701F801F901FA01FB01FC01845C
:1089C000035A56C3564F5646563F560859EF473836
:1089D000562E56252E3230530A70727573612E69E9
:1089E0006F2F3034256875007B5B4552523A003357
:1089F0002E31342E31005D5B4657523A005D5B5498
:108A0000494D3A005D5B464E4D3A005D5B46454D33
:108A10003A005D5B5043443A005B5446553A005B74
:108A200050524E3A005B50464E3A305D005B44492E
:108A3000413A005D5B4154423A005D5B4154303A3B
:108A4000005D5B5354423A005B5354303A007B5B09
:108A500050524E3A355D007B5B50524E3A305D00CD
:108A60007B5B50524E3A395D007B5B50524E3A3838
:108A70005D007B5B5245533A305D5B46494C3A00A2
:108A80007B5B5245533A315D5B46494C3A000000EE
:108A90002110422063308440A550C660E7700881F1
:108AA00029914AA16BB18CC1ADD1CEE1EFF1311268
:108AB000100273325222B5529442F772D662399341
:108AC00018837BB35AA3BDD39CC3FFF3DEE36224B8
:108AD000433420040114E664C774A44485546AA591
:108AE0004BB528850995EEE5CFF5ACC58DD5533648
:108AF000722611163006D776F6669556B4465BB7E1
:108B00007AA719973887DFF7FEE79DD7BCC7C44817
:108B1000E5588668A7784008611802282338CCC930
:108B2000EDD98EE9AFF9488969990AA92BB9F55AA7
:108B3000D44AB77A966A711A500A333A122AFDDB80
:108B4000DCCBBFFB9EEB799B588B3BBB1AABA66C77
:108B5000877CE44CC55C222C033C600C411CAEEDD0
:108B60008FFDECCDCDDD2AAD0BBD688D499D977E87
:108B7000B66ED55EF44E133E322E511E700E9FFF20
:108B8000BEEFDDDFFCCF1BBF3AAF599F788F8891D6
:108B9000A981CAB1EBA10CD12DC14EF16FE18010BA
:108BA000A100C230E3200450254046706760B983BD
:108BB0009893FBA3DAB33DC31CD37FE35EF3B1020A
:108BC0009012F322D2323542145277625672EAB5CD
:108BD000CBA5A89589856EF54FE52CD50DC5E2345A
:108BE000C324A01481046674476424540544DBA79D
:108BF000FAB79987B8975FE77EF71DC73CD7D326AA
:108C0000F2369106B01657667676154634564CD92C
:108C10006DC90EF92FE9C899E9898AB9ABA94458F9
:108C2000654806782768C018E1088238A3287DCBFC
:108C30005CDB3FEB1EFBF98BD89BBBAB9ABB754A49
:108C4000545A376A167AF10AD01AB32A923A2EFD8C
:108C50000FED6CDD4DCDAABD8BADE89DC98D267C99
:108C6000076C645C454CA23C832CE01CC10C1FEFDC
:108C70003EFF5DCF7CDF9BAFBABFD98FF89F176EE9
:108C8000367E554E745E932EB23ED10EF01E7C3C65
:108C90003E3F2F2A225C0024F4D43050C38E20C2E1
:108CA000A24017828B7011127A910D816CD90AA89B
:108CB00061E108C7586607615143061E4B5D05C157
:108CC00045A7041A411104093D9803713931034045
:108CD00036DB0265339102D4305402802E1D0263CC
:108CE0002CEE01752AC501B028A001102781018F43
:108CF0002564012B244B01E0223401AC211F018D9E
:108D0000200D01801FFC00841EED00971DDF00B8C0
:108D10001CD200E61BC600201BBC00641AB200B2C5
:108D200019A8000A19A0006A189900D117910040EB
:108D3000178B00B516840031167E00B31579003A02
:108D4000157300C7146F0058146A00EE136600888C
:108D500013630025135E00C7125B006C12570015E9
:108D6000125400C111510070114F0021114B00D657
:108D70001049008D1047004610440002104200C008
:108D80000F4000800F3E00420F3C00060F3B00CB1F
:108D90000E3800930E37005C0E3500270E3400F3BA
:108DA0000D3200C10D3100900D3000600D2E0032EB
:108DB0000D2D00050D2C00D90C2B00AE0C290085C3
:108DC0000C29005C0C2700350C27000E0C2600E84F
:108DD0000B2400C40B2400A00B23007D0B23005A9E
:108DE0000B2100390B2100180B2000F80A1F00D9B5
:108DF0000A1E00BB0A1E009D0A1D00800A1D00639A
:108E00000A1C00470A1B002C0A1B00110A1A00F753
:108E1000091A00DD091900C4091900AB09190092EB
:108E20000917007B091800630917004C0916003662
:108E3000091600200916000A091500F5081500E0BA
:108E4000081400CC081400B8081400A408140090FA
:108E50000813007D0812006B081300580812004622
:108E60000812003408110023081100120811000133
:108E7000081100F0071000E0071000D0071000C034
:108E8000071000B0070F00A107100091070E008324
:108E9000070F0074070F0065070E0057070E004903
:108EA000070E003B070D002E070E0020070D0013D4
:108EB000070D0006070D00F9060C00ED060D00E099
:108EC000060C00D4060C00C8060C00BC060C00B052
:108ED000060C00A4060B0099060C008D060B008200
:108EE000060B0077060B006C060B0061060A0057A4
:108EF000060B004C060A0042060A0038060A002E3D
:108F0000060A0024060A001A060A001006090007CD
:108F1000060A00FD050900F4050900EB050900E259
:108F2000050900D9050900D0050900C7050900BEDB
:108F3000050900B5050800AD050800A50509009C58
:108F4000050800940508008C050800840508007CCD
:108F5000050800740508006C050700650508005D3C
:108F6000050700560508004E0507004705070040A5
:108F700005080038050700310507002A050700230A
:108F80000507001C050600160507000F0507000869
:108F900005060002050700FB040600F5040700EEC5
:108FA000040600E8040600E2040700DB040600D51E
:108FB000040600CF040600C9040600C3040600BD71
:108FC000040600B7040600B1040500AC040600A6C0
:108FD000040600A00405009B04060095040500900B
:108FE0000406008A04050085040500800406007A52
:108FF00004050075040500700405006B0405006697
:10900000040500610405005C0405005704050052D6
:109010000405004D04050048040500430405003E16
:109020000404003A04050035040500300404002C53
:1090300004050027040400230405001E0404001A8C
:1090400004040016040500110404000D04040009C2
:109050000405000404040000040400FC030400F8F8
:10906000030400F4030400F0030400EC030400E82C
:10907000030400E4030400E0030400DC030400D85C
:10908000030400D4030400D0030400CC030400C88C
:10909000030300C503030024F404D9201BC40C5CA3
:1090A0000E9804C4095F0265077101F405F900FB1D
:1090B00004B30048048700C1036900580355000346
:1090C000034500BE023A008402310053022A0029FF
:1090D00002250004022000E4011C00C8011900AFB1
:1090E0000117009801140084011300710110006140
:1090F00001100051010E0043010D0036010B002B41
:10910000010B0020010B00150109000C01090003EF
:10911000010800FB000800F3000800EB000700E472
:10912000000600DE000600D8000600D2000600CCD3
:10913000000500C7000500C2000500BD000400B91D
:10914000000400B5000400B1000400AD000400A953
:10915000000400A5000300A20003009F0004009B80
:1091600000030098000300950002009300030090A4
:109170000003008D0002008B0003008800020086BF
:1091800000020084000300810002007F0002007DD5
:109190000002007B000200790002007700010076E7
:1091A0000002007400020072000100710002006FF2
:1091B0000002006D0001006C0002006A00010069FD
:1091C0000002006700010066000100650001006404
:1091D0000002006200010061000100600001005F08
:1091E0000002005D0001005C0001005B0001005A0C
:1091F000000100590001005800010057000100560D
:10920000000100550001005400010053000000530C
:109210000001005200010051000100500001004F08
:109220000001004E0000004E0001004D0001004C06
:109230000001004B0000004B0001004A0001004902
:1092400000010048000000480001004700010046FE
:1092500000000046000100450000004500010044F8
:1092600000010043000000430001004200000042F2
:109270000001004100000041000100400001003FEA
:109280000000003F0001003E0000003E0001003DE4
:109290000000003D0001003C0000003C0000003CDC
:1092A0000001003B0000003B0001003A0000003AD2
:1092B00000010039000000390001003800000038CA
:1092C00000000038000100370000003700010036C0
:1092D00000000036000000360001003500000035B7
:1092E00000000035000100340000003400000034AC
:1092F00000010033000000330000003300010032A1
:109300000000003200000032000100310000003196
:10931000000000310001003000000030000000308B
:109320000001002F0000002F0000002F0000002F80
:109330000001002E0000002E0000002E0001002D74
:109340000000002D0000002D0000002D0001002C69
:109350000000002C0000002C0000002C0001002B5D
:109360000000002B0000002B0000002B0001002A51
:109370000000002A0000002A0000002A0001002945
:109380000000002900000029000000290000002939
:10939000000100280000002800000028000000282C
:1093A000000000280001002700000027000000271F
:1093B0000000002700000027000100260000002612
:1093C0000000002600000026000000260001002505
:1093D00000000025000000250000002500000025F9
:1093E00000000025000100240000002400000024EB
:1093F00000000024000000240001002300000023DE
:1094000000000023000000230000002300000023D0
:1094100000000023000100220000002200000022C2
:1094200000000022000000220000002200010021B4
:1094300000000021000000210000002100000021A8
:109440000000002100000021000100200000002099
:10945000000000200000002000000020000000208C
:1094600000000020000000200001001F0000001F7D
:109470000000001F0000001F0000001F0000001F70
:109480000000001F0001001E0000001E0000001E62
:109490000000001E00000045303A20005A3A20002B
:1094A000593A2000583A20004D53312C4D53322068
:1094B00050696E7300504944204175746F74756E25
:1094C000652066696E697368656421205075742033
:1094D000746865206C617374204B702C204B69207C
:1094E000616E64204B6420636F6E7374616E74737D
:1094F0002066726F6D2061626F766520696E746F91
:1095000020436F6E66696775726174696F6E2E684D
:1095100000504944204175746F74756E6520666112
:10952000696C6564212074696D656F7574002040F5
:109530003A00543A00423A00504944204175746F51
:1095400074756E65206661696C6564212054656D73
:10955000706572617475726520746F6F20686967D9
:109560006800204B643A2000204B693A2000204BD1
:10957000703A200020436C61737369632050494442
:1095800020002054753A2000204B753A2000206DB1
:1095900061783A2000206D696E3A200020643A20FC
:1095A0000020626961733A2000504944204175747B
:1095B0006F74756E65207374617274005049442035
:1095C0004175746F74756E65206661696C65642E93
:1095D00020426164206578747275646572206E75CE
:1095E0006D6265722E00486F74656E642066616EF0
:1095F000207370656564206973206C6F77657220D5
:109600007468616E2065787065637465640050727B
:10961000696E742066616E2073706565642069737D
:10962000206C6F776572207468616E206578706554
:1096300063746564004D494E54454D502042454485
:10964000004D494E54454D50004D415854454D50E4
:10965000004D415854454D50204245440070012C66
:109660000190012701B0012201C0011D01F0011884
:10967000011002130130020E016002090190020480
:1096800001C002FF000003FA004003F5008003F070
:1096900000D003EB002004E6007004E100E004DCED
:1096A000004005D700C005D2004006CD00D006C856
:1096B000008007C3003008BE00F008B900C009B43C
:1096C00000B00AAF00B00BAA00D00CA500000EA09D
:1096D00000500F9B00C01096005012910000148C97
:1096E00000C0158700B0178200B0197D00D01B782C
:1096F00000001E730040206E0090226900F0246478
:109700000040275F0090295A00E02B5500102E5092
:109710000020304B0010324600E033410090353CD1
:10972000001037370070383200A0392D00B03A28C9
:1097300000A03B2300603C1E00103D1900903D142A
:1097400000103E0F00703E0A00C03E0500003F00C2
:109750000020484F54454E4420544845524D414CFA
:109760002052554E415741590020484541544245E9
:109770004420544845524D414C2052554E4157418A
:109780005900544845524D414C2052554E41574185
:10979000590042454420544845524D414C205255B1
:1097A0004E415741590020544845524D414C20529A
:1097B000554E415741592028505245484541542063
:1097C000484F54454E44290020544845524D414C81
:1097D0002052554E41574159202850524548454145
:1097E000542048454154424544290050524548457B
:1097F0004154204552524F52004245442050524558
:1098000048454154204552524F52002074726967B6
:1098100067657265642100486561746572732073C1
:1098200077697463686564206F66662E20003A204D
:10983000004572723A200000FF0102010002FFFFA2
:10984000FE0001FE01FF00506C65617365207265CA
:1098500073746172740055534152543220727820EF
:1098600046756C6C212121003A2000252D31322EC5
:10987000313253252D642F36002533642F252D33A7
:109880006400203A200025335300252D377300252E
:109890002D31352E313553252D35640A252D3135A1
:1098A0002E313553252D35640A0025530A20252DE8
:1098B00031362E313653252D33640A20252D31368D
:1098C0002E313653252D33640025530A20252D31A2
:1098D000362E313653252D33640A20252D31362E70
:1098E000313653252D33640A20252D31362E31365D
:1098F00053252D33640025530A20252D31362E3172
:109900003653252D33640A25530A20252D31362E52
:10991000313653252D33640A0020257325336481A5
:10992000200A0025752E25752E25752E25750020FB
:10993000002000466C6173684169722049502041E3
:109940006464723A004D4D552020202020202020B4
:109950004E2F410025642E25642E25640020465795
:109960003A00313937302D30312D30310045334414
:10997000763666756C6C0052414D426F3130610035
:10998000315F37356D6D5F4D4B3235002048617367
:10999000683A30303030303030303000205265702E
:1099A0006F3A556E6B6E6F776E0020332E31342E0A
:1099B000312D38323337004669726D776172653AFE
:1099C00000464C4558202D20203234302F353000B1
:1099D000464C4558202D2020323430005050202055
:1099E000202D20203235342F3130300050502020AF
:1099F000202D20203235340048495053202D20207E
:109A00003232302F3130300048495053202D202041
:109A10003232300041425320202D20203235352F64
:109A20003130300041425320202D20203235350086
:109A300050412020202D20203237352F3930005042
:109A4000412020202D202032373500505642202042
:109A50002D20203231352F37350050564220202D11
:109A600020203231350050432020202D2020323755
:109A7000352F3130350050432020202D2020323723
:109A8000350041534120202D20203236302F3130F7
:109A9000350041534120202D2020323630005045E2
:109AA0005420202D20203233302F3835005045549B
:109AB00020202D202032333000504C4120202D20FA
:109AC000203231352F363000504C4120202D2020BF
:109AD000323135006E6F7A7A6C65202D2020323558
:109AE000302F30006661726D2020202D202032350D
:109AF000302F3830001000C90210012C0140012223
:109B00000170011801B0010E01F00104015002FAC8
:109B100000B002F0003003E600D003DC009004D275
:109B2000007005C800A006BE000008B400B009AA75
:109B300000D00BA000600E960060118C0000158212
:109B40000020197800C01D6E00A0226400B0275AC2
:109B500000902C500000314600E0343C00103832B8
:109B600000903A2800603C1E00A03D1400803E0A90
:109B700000203F00004D6561737572652063656E5E
:109B800074657220200078797A63616C5F6D65611D
:109B9000737572655F656E7465720A0078797A63B1
:109BA000616C5F73706972616C382063783D256405
:109BB0002063793D2564207A303D256420647A3D18
:109BC0002564207261646975733D25642061643D7C
:109BD00025640A0078797A63616C5F7365617263EA
:109BE000685A206E6F207369676E616C0A20783D39
:109BF000256C6420793D256C64207A3D256C640ACF
:109C000000204F4E2D5349474E414C20617420781F
:109C10003D256420793D2564207A3D2564206164DA
:109C20003D25640A0078797A63616C5F73656172BF
:109C300063685A20783D256C6420793D256C64204A
:109C40007A3D256C640A002530327800205B256659
:109C50002025665D206D6D207061747465726E20C4
:109C600063656E7465720A00205B25662025665D5B
:109C70005B25665D206D6D20646976657267656E33
:109C800063650A000000F000F801FC03FE07FE0710
:109C9000FE07FE07FC03F801F000000000000000D2
:109CA000F000F801FC03FC03FC03FC03F801F000E6
:109CB0000000000078797A63616C5F6D656173758F
:109CC00072655F6C656176650A00203C2000574133
:109CD000524E494E473A2046726F6E7420706F693B
:109CE0006E74206E6F7420726561636861626C656A
:109CF0002E205920636F6F7264696E6174653A003B
:109D000000000040410000804000005C43000080F3
:109D10004000005C43000044430000404100004418
:109D20004325642F3400497465726174696F6E3A1B
:109D3000200043616C6962726174696F6E206661B4
:109D4000696C65642120436865636B2074686520D5
:109D50006178657320616E642072756E2061676141
:109D6000696E2E0078797A63616C5F7370697261D5
:109D70006C322063783D25642063793D2564207A28
:109D8000303D256420647A3D2564207261646975E4
:109D9000733D25642061643D25640A000A00436F19
:109DA000756E74646F776E3A202564200025640A0E
:109DB000005363616E20636F756E74646F776E3AE3
:109DC00020005061747465726E2063656E746572F4
:109DD000205B25662025665D2C206D6174636820FC
:109DE000256625250A00205B25662C2025665D5BFF
:109DF00025665D2066696E616C20636972636C65BF
:109E00000A000000A0400000A04000000040000048
:109E10007A43000056439AD95143FFFFFFE02D904B
:109E20003E8988B24111369C3E7777C14129CBB03B
:109E30003EEFEEDA41BA49CC3EEFEEFC4161C3F3AE
:109E40003EEFEE16429CA2133FCDCC36428AB011B3
:109E50003FABAA56428863DD3DABAA5642B8AF433A
:109E60003F555572421826533F33B38242302A5928
:109E70003FEF6E8642000070C10000C8420000C47F
:109E8000C10000A0410000E0C000002041000060CF
:109E9000C00000C0400000A0412222F2400000A00B
:109EA000C19A99A14000000CC255550542436F6FFD
:109EB0006C696E672074696D65722073746F707061
:109EC00065640048656174657220636F6F6C646FD0
:109ED000776E00436F6F6C696E672054696D656FB4
:109EE0007574207374617274656400536176696E71
:109EF0006720616E64207061726B696E67004865EF
:109F00006174657220636F6F6C646F776E2070652B
:109F10006E64696E6700526573756D696E6720586F
:109F2000595A004731205825642059252D2E326674
:109F30002045252D2E33660057726974696E67209F
:109F4000746F2066696C653A200046696C65206113
:109F50006C7265616479206F70656E6564007C5B0E
:109F60006B5B575B425B2C5B195B035BEF5ADE5A02
:109F7000C85A575B6B5BB45AA55A915A805A6B5AB0
:109F8000AF62555A435A305A1F5A0A5AF759E35981
:109F9000CE59C559B3599E594D363030204155548C
:109FA0004F0046494E44412066696C616D656E7490
:109FB0002072756E6F75742100436F6D6D756E69DB
:109FC000636174696F6E2074696D656F757400509C
:109FD000726F746F636F6C204572726F7200030052
:109FE0000356657273696F6E206D69736D6174637A
:109FF0006800436F6D6D616E64204572726F720010
:10A00000436F6D6D616E642072656A65637465642B
:10A01000004D4D5520427574746F6E2070757368D5
:10A020006564005265747279427574746F6E507213
:10A03000657373656400D95DC45DAD5D985D835DD6
:10A040006F5D5F5D485D315D1A5D065DF25CDC5CF5
:10A05000DC5CDC5CC75CC75CC75CB45CB45CB45CF7
:10A06000A15CA15CA15C8A5C8A5C8A5C755C755CA5
:10A07000755C5F5C5F5C5F5C4F5C3A5C245C0E5CB3
:10A08000FF5BF25BDB5BC85BB65BA35B915B815BF9
:10A09000427574746F6E00436865636B55736572C7
:10A0A000496E7075742D62746E4C4D52200052656D
:10A0B0007365745265747279417474656D707473EC
:10A0C0000046493A202046533A202020203E2020B6
:10A0D000822020208100486F74656E642074656D55
:10A0E000706572617475726520726561636865641C
:10A0F00000526573756D696E672054656D7000431D
:10A100006F6F6C646F776E20666C616720636C653F
:10A11000617265640020573A0020453A00543A00C5
:10A120004E6F2030784646207265636569766564B7
:10A130000053656E64696E67203078464600466954
:10A140006C652073656C6563746564002053697A7F
:10A15000653A200046696C65206F70656E65643AEB
:10A1600020004E6F772066726573682066696C65A3
:10A170003A20004E6F7720646F696E672066696CC5
:10A18000653A20002220706F730022207061726592
:10A190006E743A2200535542524F5554494E452051
:10A1A00043414C4C207461726765743A22007472AA
:10A1B00079696E6720746F2063616C6C20737562BF
:10A1C0002D67636F64652066696C657320776974B9
:10A1D0006820746F6F206D616E79206C6576656C98
:10A1E000732E00062833D036C23E013F154132425D
:10A1F0003B43F2443B45F24622473B48F2493B4A47
:10A20000F05898590C5A085B0C5C086110679B6EFB
:10A210002271077208FF095A0D000EF019145E082A
:10A2200020642B6D322FFF2022257322002025234E
:10A230006C78004449525F45584954004449525F84
:10A24000454E5445523A20257320222573220A0098
:10A250006175746F25692E6700041A446563726521
:10A260006D656E745265747279417474656D707445
:10A270007300081B1C0B14525354436F6D6D5469CB
:10A280006D656F7574002C206C6173742062797435
:10A2900065733A200022206661696C65643A204249
:10A2A00075666665722066756C6C21002200456ECD
:10A2B000717565696E6720746F20746865206672B9
:10A2C0006F6E743A2022004572726F723A004D4DE3
:10A2D0005532746F6F6C3D004D4D55323A004D4D07
:10A2E00055323A006563686F3A003E53302A633650
:10A2F0002E004D4D552069732000F0382A6411243A
:10A300001FBECFEFD1E2DEBFCDBF00E00CBF13E038
:10A31000A0E0B2E0E4E1F6E503E00BBF02C0079085
:10A320000D92A230B107D9F727E1A2E0B3E001C056
:10A330001D92A731B207E1F711E5CEE7D1E500E0C4
:10A3400006C021970109802FFE010F944EA5CD373D
:10A35000D10780E00807A9F70E9405EB0D94F8AA41
:10A360000C945A852F923F924F925F926F927F92F8
:10A370008F929F92AF92BF92CF92DF92EF92FF9215
:10A380000F931F93CF93DF93CDB7DEB72F970FB601
:10A39000F894DEBF0FBECDBF6C011B015A01FC015A
:10A3A0001782168283819E012F5F3F4F490181FDF5
:10A3B000D2C08FEF9FEFEEC2F12C512C00E00032A3
:10A3C00038F48B3209F190F48032F9F0833209F1DC
:10A3D00007FD34C020ED280F2A3020F506FF1BC0F2
:10A3E000FAE0FF9E200D1124F22E05C08D3279F087
:10A3F000803371F70160F10193FD859193FF8191A5
:10A400001F018111DCCF1AC002600460F4CF086024
:10A41000F2CF0061F0CF3AE0539E200D1124522E6E
:10A420000062E9CF8E3221F406FDB1C20064E3CFB1
:10A430008C3611F40068DFCF8836E9F29BEB980F79
:10A44000933008F05FC00061805E06FD02C046E008
:10A45000F42E102F1F73853609F05BC0106417FFB0
:10A4600061C08F2D9BE39F1508F48BE34424439434
:10A47000480E27E03501F4E06F0E711CF501608194
:10A48000718182819381042DA4010F94F7A05C0156
:10A49000F981FC87F0FF03C00DE2F3FF07C00BE278
:10A4A00011FD04C0012F047012FD00E22C852C70F8
:10A4B000E22E09F46BC00111D8C2F3E0E12CF515CE
:10A4C000A0F483E0E52CE81A13FD08C0B60180E291
:10A4D00090E00F94A6A2EA94E110F8CF002329F0AF
:10A4E000B601802F90E00F94A6A23C8528E2A22E10
:10A4F00022E7B22E33FD04C09CE2A92E92E7B92ECA
:10A50000107122C09BE9980F933008F047C10F7E6D
:10A510009CCF863611F41068A2CFFF2009F49FCF9C
:10A52000FA949DCFE7E02F2DEF1518F427E037E0E0
:10A53000F32E412C9FCF11118052B60190E00F9461
:10A54000A6A28FEFA81AB80AF50184918111F3CF62
:10A55000E11084C25301F6019381F10193FD8591CD
:10A5600093FF81911F01882309F411C2853241F4C0
:10A5700093FD859193FF81911F01853209F01CCFD6
:10A58000B60190E00F94A6A23501E4CF17FF6FC08B
:10A590004A0CFC85F4FF04C08A81813309F44A9493
:10A5A00014140CF086C028E0241510F488E0482E1E
:10A5B00085E090E017FF06C0C501B7FE02C090E03D
:10A5C00080E0019601110196FF2031F02F2D30E03F
:10A5D0002F5F3F4F820F931F5816190619F014F082
:10A5E000E52CE81A812F897011F4E11067C000236F
:10A5F00029F0B601802F90E00F94A6A213FD02C0AF
:10A60000E11063C017FF7CC08501B7FE02C010E0F7
:10A6100000E0C501841991092C016F2D70E0EE272F
:10A62000FF27E61BF70BFF87EE870F3F100729F484
:10A63000B6018EE290E00F94A6A2A016B1060CF42B
:10A640004BC0401651060CF047C0F501E01BF10B62
:10A65000E80DF91D8181015011092E853F850217F2
:10A660001307E4F1B60190E00F94A6A2DECF16FD29
:10A670009FCFEF2DF0E0EA15FB0534F03CEFA31679
:10A680003FEFB3060CF010683296E80DF91D01C0DB
:10A69000FA94FF2019F082918033D1F317FF88CF0D
:10A6A000442443944F0CFA141B0431F02CF0FA1894
:10A6B0007FCF442443947CCFF12C7ACFB60180E243
:10A6C00090E00F94A6A2EA9490CFB60180E390E0C8
:10A6D0000F94A6A2EA9494CF80E3BDCFA016B10652
:10A6E00041F49A81963350F4953319F43C8534FF44
:10A6F00005C0B60190E00F94A6A22ACF81E3F9CF5E
:10A700008A81813319F09C859F7E9C87B60190E0F9
:10A710000F94A6A2FF20A9F0B6018EE290E00F945C
:10A72000A6A2F394F394E2E001E00E0FE80DF92DF8
:10A73000F11D8081B60190E00F94A6A2E02F0F11C9
:10A74000F3CF85E690E014FF02C085E490E0B60107
:10A750000F94A6A2B7FC06C0A114B104C1F4EC8505
:10A76000E4FF15C0B194A194B1088DE2B60190E068
:10A770000F94A6A280E32AE0A216B10454F4B60115
:10A7800090E00F94A6A2B601C501C096B4CF8BE2AB
:10A79000EDCF8F5FFAE0AF1AB108EDCF8336C9F085
:10A7A000833771F1833509F05BC03501F2E06F0E3C
:10A7B000711CF501A080B1806F2D70E006FD02C014
:10A7C0006FEF7FEFC5010F943AA29D878C870068D9
:10A7D0000DC0350132E0630E711CF5018081898363
:10A7E00021E030E03D872C8754010F7703FD06C040
:10A7F0002C853D855216130609F0A8F4E52C2BC0D4
:10A80000350132E0630E711CF501A080B1806F2D1F
:10A8100070E006FD02C06FEF7FEFC5010F945FA2ED
:10A820009D878C87E2CFB60180E290E00F94A6A2CC
:10A830005A94DECFF50107FD859107FF81915F01F5
:10A84000B60190E00F94A6A2E110EA948C859D8554
:10A8500001979D878C87EC85FD85EF2B59F778CE86
:10A86000843619F0893609F074C0350107FF66C0D7
:10A87000F4E06F0E711CF50160817181828193811A
:10A88000102F1F7697FF08C0909580957095619561
:10A890007F4F8F4F9F4F10682AE030E0A4010F9444
:10A8A000CDA3A82EA818BA2C012F16FF0AC00E7F20
:10A8B000AF1438F414FF04C012FD02C0012F0E7E45
:10A8C000BF2C04FFA3C0FE01EA0DF11D808180337F
:10A8D00009F095C0097EF02FF870EF2E03FDA5C09A
:10A8E00000FF9FC0FA2CB51410F4F50CFB1804FF00
:10A8F000A2C0B60180E390E00F94A6A202FF09C0B7
:10A9000088E790E001FF02C088E590E0B6010F946F
:10A91000A6A2AF1408F49BC0AA940A2D10E00F5F02
:10A920001F4F080D191DF80182918F01B60190E0AB
:10A930000F94A6A280169106B1F70ACEF2E06F0E30
:10A94000711CF50160817181072E000C880B990B39
:10A9500097CF102F8537A9F41F7E2AE030E035010C
:10A9600017FF44C0F4E06F0E711CF5016081718126
:10A9700082819381A4010F94CDA3A82EA8181F77DC
:10A9800092CF197F8F3679F1F0F4883539F1F601DD
:10A99000868197812F960FB6F894DEBF0FBECDBF8C
:10A9A000DF91CF911F910F91FF90EF90DF90CF90AB
:10A9B000BF90AF909F908F907F906F905F904F90DF
:10A9C0003F902F900895803739F0883701F714FDB4
:10A9D000146020E130E0C3CF1061F9CF04FD1660B0
:10A9E00020E132E0BCCF28E030E0B9CFF2E06F0EDA
:10A9F000711CF5016081718190E080E0BBCF02FDA8
:10AA000002C0B39468CFB394B39465CF802F867897
:10AA100009F461CFF6CFB60180E290E00F94A6A2D0
:10AA2000B394B514C0F3E12C62CFE52CEB18B51448
:10AA300008F45DCFF8CF802F867809F46ACF8BE2D7
:10AA400001FF80E207FD8DE2B60190E060CFB60124
:10AA500080E390E00F94A6A2FA945BCFB60180E267
:10AA600090E00F94A6A2EA9473CD24E0E12C251582
:10AA700008F036CD84E026CD20E030E040E85FEB02
:10AA800060917E0270917F0280918002909181029C
:10AA90000F945BA6882321F1E0913812F0913912CE
:10AAA000E55BFF4E80818B7F8230D1F480E1EEE761
:10AAB000F2E0A1E6B2E101900D928A95E1F780E023
:10AAC00090E0A0E8BFEB80937E0290937F02A0937A
:10AAD0008002B093810280914D1290914E120895A0
:10AAE00081E090E0089580E1E9E2F6E0A1E6B2E1DC
:10AAF00001900D928A95E1F70895E0E0F7E7833041
:10AB000021F0E82FF0E0E350F94884910895809116
:10AB10004205909143052091440530914505821BE3
:10AB2000930B8F7799270895982F9F7083FF0DC0FF
:10AB300080917B00886080937B0080917C00887F7F
:10AB40009770892B80937C00089580917B00877F8C
:10AB5000F2CF4FEF5FEFBA0185EE9FE00F9474A440
:10AB60004FEF5FEFBA0189EE9FE00F9474A44FEFAF
:10AB70005FEFBA018DED9FE00F9474A44FEF5FEF8C
:10AB8000BA0181EE9FE00F9474A44FEF5FEFBA011A
:10AB900085ED9FE00F9474A44FEF5FEFBA0189ED4C
:10ABA0009FE00F9474A44FEF5FEFBA0185EC9FE034
:10ABB0000F9474A44FEF5FEFBA0189EC9FE00F94FC
:10ABC00074A44FEF5FEFBA018DEC9FE00F9474A473
:10ABD0004FEF5FEFBA0181ED9FE00D9474A48036D2
:10ABE0009105F8F440913812509139122091491092
:10ABF00030914A104217530739F460913C1270911A
:10AC00003D12161617066CF0B901680F791FFB018B
:10AC1000E359FF4F2417350730F481E04E175F07E3
:10AC200008F480E00895EE3EF140F8F06C5F7F4F4D
:10AC30006E3E714018F449365105B8F483599F4F60
:10AC40004817590770F34DEE51E0421B530B70E06B
:10AC500060E0C901855B9F4E0F9470AA8FB7F8948E
:10AC600010924A10109249108FBF81E00895809190
:10AC7000440590914505909343058093420580E9F2
:10AC80009AE69F938F9380913E1290913F12A091EC
:10AC90004012B09141120196A11DB11DBF93AF9317
:10ACA0009F938F938DE095E69F938F9384E195E634
:10ACB0009F938F930F9400A38DB79EB70A960FB6FC
:10ACC000F8949EBF0FBE8DBF08950F931F93CF932F
:10ACD000DF93EC01C60FD71F8C179D0779F08C010D
:10ACE0000F5F1F4F0F943EA48F3F31F081E0DF9143
:10ACF000CF911F910F910895C801EECF80E0F7CF5B
:10AD0000682F880F770B8091381290913912825BEF
:10AD10009F4E0F9495AA9C019093BC048093BB0412
:10AD200081E0232B09F480E008958091BB04909189
:10AD3000BC044AE050E070E060E001960F94C99FC7
:10AD4000862F08958091BB049091BC044AE050E0A6
:10AD500070E060E001960F94C99FCB0108950F93B6
:10AD60001F93CF93DF938C01862FEA010E948056B8
:10AD7000882319F10E94A2569C0197FF03C03195C8
:10AD800021953109253631059CF09F938F9387ECEF
:10AD900092EA9F938F938DE797E79F938F930F94FA
:10ADA00000A30F900F900F900F900F900F9080E0E6
:10ADB000DF91CF911F910F910895F8018081882331
:10ADC000B1F3CE01DF91CF911F910F910D943EA46D
:10ADD0008091BB049091BC044AE050E070E060E0D8
:10ADE00001960D94C99F60E086E69FE00F9462A4EF
:10ADF00060E088E69FE00F9462A460E085E69FE053
:10AE00000F9462A460E084E69FE00F9462A460E087
:10AE100082ED9EE00F9462A460E08FEC9EE00D94C2
:10AE200062A42F923F924F925F926F927F928F9285
:10AE30009F92AF92BF92CF92DF92EF92FF920F93C9
:10AE40001F93CF93DF93CDB7DEB7CC58D2400FB668
:10AE5000F894DEBF0FBECDBFCB58DD4F688379833A
:10AE60008A839B83C557D240FE01E754FE4F88E298
:10AE7000DF011D928A95E9F7E85BF1401F0180E947
:10AE800091E0DF01FC011D923197E9F7C75ADD4FD0
:10AE900019821882C955D2409E012F513E4FC15987
:10AEA000DD4F39832883CF56D2408E01075A1D4F7C
:10AEB000CE018F5C9D4FC359DD4F99838883CD565A
:10AEC000D2403C01490140EBA42E4FE0B42E53E2A6
:10AED000C52ED12CF12CE12CB6010D2C000C880BC9
:10AEE000990B0F94CC9ED4016D937D938D939D937C
:10AEF0004D01F801619171918F01072E000C880BB3
:10AF0000990B0F94CC9ED3016D937D938D939D935C
:10AF10003D01BFEFEB1AFB0AE6E0EE16F10409F083
:10AF200038C3CB58DD4F288139814A815B81C557B1
:10AF3000D240C159DD4FA881B981CF56D2406D9121
:10AF40007D918D919C910F94EFA7412C512C320152
:10AF500018160CF402C3C359DD4F08811981CD5670
:10AF6000D2400C5E1F4FC159DD4FE880F980CF56AB
:10AF7000D240B4E1EB0EF11C6E01EFEDCE1AEDEF15
:10AF8000DE0A9E012B553E4FCF58DD4F3983288373
:10AF9000C157D240D8014D905D906D907C90F701E3
:10AFA0006081718182819381D7015E914E913E9142
:10AFB0002E917D010F9465A54B015C01F801529122
:10AFC0004291329122918F01C301B2010F9465A584
:10AFD000A50194010F9465A6D6019E938E937E934E
:10AFE0006E936D01CF58DD4FE881F981C157D24092
:10AFF000B292A29292928292CF58DD4FF983E88367
:10B00000C157D240C359DD4F28813981CD56D24036
:10B010000217130709F0BECF4E013FE6831A3EEF39
:10B02000930A5E0183EFA81A8DEFB80A61018101CE
:10B03000EE24E394F12CD4014D905D906D907D90C1
:10B040004D012D913D914D915C91C301B2010F9441
:10B0500066A59B01AC010F9466A5F80164A775A7CE
:10B0600086A797A7F1E0EF16F10461F0D801989652
:10B070004D925D926D927C929B97F801448255822D
:10B0800066827782FFEFEF1AFF0AF5012081318196
:10B090004281538184E0A80EB11C64817581868150
:10B0A00097810F9465A520E030E040EC50E40F94C8
:10B0B0000B9FD601DC966D937D938D939C93DF97C8
:10B0C000045D1F4FB8E2CB0ED11CE5E0EE16F10493
:10B0D00009F0B1CF7E01FDE2EF0EF11C28E2A22EB5
:10B0E000B12C00EB1FEF24E0220E311CD7012D9173
:10B0F0003D914D915C91139798966D917D918D91B5
:10B100009C919B970F9465A62B013C016101C01A8D
:10B11000D10A88248394912CF601E00FF11FEA0DE7
:10B12000FB1D2081318142815381C301B2010F9403
:10B130000B9F9B01AC01F60160817181828193813B
:10B140000F9465A5D6016D937D938D939D936D01AD
:10B15000BFEF8B1A9B0AE6E08E169104E9F63CE2FB
:10B16000E30EF11C0852110988E2A80EB11C083345
:10B170009FEF190709F0BACF1E01F5EB2F0E311C16
:10B180006E0121EBC20ED11C7E0137E3E31A3EEFC4
:10B19000F30A04E010E04801B12CA12C412C512C01
:10B1A0003201F601EA0DFB1DD701AA0DBB1D2D9141
:10B1B0003D914D915C9160817181828193810F9469
:10B1C0000B9F9B01AC01C301B2010F9466A52B013B
:10B1D0003C018FEF881A980A94E0A90EB11CA5E0F3
:10B1E0008A169104F1F6A3019201F1016081718147
:10B1F000828193810F9465A5D6012D913D914D914A
:10B200005C910F9465A6F7016083718382839383B9
:10B2100001501109F8E22F1A31082CE2C21AD108A4
:10B2200034E0E31AF1080115110509F0B4CFCB5051
:10B23000DE4F88819981AA81BB81C55FD140CF57FC
:10B24000DD4F88839983AA83BB83C158D2401E01F6
:10B2500097E4291A9EEF390A10E000E0C159DD4F4A
:10B26000A881B981CF56D240CD90DD90ED90FD9070
:10B27000C159DD4FB983A883CF56D240CB58DD4F9B
:10B28000288139814A815B81C557D240C701B60107
:10B290000F945BA61816B4F0CB58DD4F2881398186
:10B2A0004A815B81C557D240C159DD4FE881F981A0
:10B2B000CF56D24060817181828193810F94EFA734
:10B2C00087FF18C00430110509F030C1CB58DD4F9D
:10B2D000288139814A815B81C557D240CF57DD4FE4
:10B2E000688179818A819B81C158D2400F945BA685
:10B2F00087FF1CC1D10114968D909D90AD90BC909C
:10B3000017978D919D910D90BC91A02DCF58DD4F39
:10B3100088839983AA83BB83C157D240F801EE0F7B
:10B32000FF1FEE0FFF1F21E931E02C0F3D1FE20F41
:10B33000F31F4080518062807380C359DD4FA88124
:10B34000B981CD56D2408D919D910D90BC91A02D8B
:10B35000C358DD4F88839983AA83BB83CD57D240DE
:10B36000A7019601CB58DD4F688179818A819B8145
:10B37000C557D2400F9465A56B017C0120E030E0F9
:10B3800040E450E40F94D6A8CB57DD4F688379830F
:10B390008A839B83C558D240C358DD4F28813981A9
:10B3A0004A815B81CD57D240C359DD4FE881F98195
:10B3B000CD56D24064817581868197810F9465A5B1
:10B3C000A30192010F9465A6C758DD4F6883798366
:10B3D0008A839B83C957D240A3019201C301B20162
:10B3E0000F9466A5CF58DD4F288139814A815B8152
:10B3F000C157D2400F940B9FC757DD4F68837983A5
:10B400008A839B83C958D240A3019201C501B4012C
:10B410000F940B9F9B01AC01C757DD4F6881798169
:10B420008A819B81C958D2400F9466A520E030E004
:10B4300040EC50E40F9465A69B01AC01C758DD4F6A
:10B44000688179818A819B81C957D2400F9465A513
:10B45000A70196010F940B9FC758DD4F688379832E
:10B460008A839B83C957D240CF58DD4F28813981C9
:10B470004A815B81C157D240C501B4010F9465A5D3
:10B480004B015C0120E030E040EC50E4C301B2012C
:10B490000F940B9F9B01AC01C501B4010F9465A6ED
:10B4A000CB57DD4F288139814A815B81C558D24015
:10B4B0000F940B9F4B015C0120E030E040E05FE324
:10B4C000CF58DD4F688179818A819B81C157D240F5
:10B4D0000F940B9F2B013C01A7019601C701B601F8
:10B4E0000F940B9F9B01AC01C301B2010F940B9F02
:10B4F0009B01AC01C501B4010F9466A59B01AC0191
:10B50000C758DD4F688179818A819B81C957D240B4
:10B510000F9466A5C358DD4F288139814A815B812C
:10B52000CD57D2400F9466A52B013C010F5F1F4FF2
:10B53000F4E02F0E311CC359DD4F28813981CD56DF
:10B54000D2402C5F3F4FC359DD4F39832883CD56FE
:10B55000D2400530110509F081CEC301B201C457B4
:10B56000DD4F0FB6F894DEBF0FBECDBFDF91CF9198
:10B570001F910F91FF90EF90DF90CF90BF90AF9011
:10B580009F908F907F906F905F904F903F902F9003
:10B590000895C5010F944CA4D8018D939C93B5E0F8
:10B5A000CB0ED11CE2E0AE0EB11C96CC0F931F93D4
:10B5B000CF9320910113213079F58C0180E50E9411
:10B5C0008056882349F10E949556C82F853020F572
:10B5D000013C82E0180749F0023C124069F08C2FD0
:10B5E000CF911F910F910D94E79D60E08C2FCF912B
:10B5F0001F910F910D942A9E8EEC9EE00F943EA415
:10B60000882351F00F94047A882331F08C2FCF9146
:10B610001F910F910D94A79ECF911F910F910895A7
:10B620008F929F92AF92BF92CF92DF92EF92FF9252
:10B630000F931F93CF93DF930091BB041091BC0431
:10B640000F5F1F4F68018FEFC81AD80AD801DC912D
:10B650008D2F90E00F94CFA17C01892B01F5DD3275
:10B6600001F56801B2E0CB0ED11CF801D181C1E037
:10B6700086010150110943E050E064E377E7C80117
:10B680000F9405A2892BC1F460E070E080E89FEF81
:10B69000C111DBC060E070E080E89FE7D6C08601A2
:10B6A000D1CFDB3239F46801F2E0CF0ED11CD801E2
:10B6B0001196DC91C0E0DCCF43E050E061E377E736
:10B6C000C8010F9405A2892B09F4CCC0F60110E043
:10B6D00000E020E030E0A9016F01D053DA3060F5DE
:10B6E000BC2E6894B1F88C2F8870C2FF09C08111FC
:10B6F00002C00F5F1F4F3196D601DC91CB2DECCFEE
:10B70000882311F001501109A5E0B0E00F94D3A4F3
:10B710009B01AC01220F331F441F551F2D0F311DFC
:10B72000411D511D2839B9E93B074B07B9E15B07BA
:10B7300010F3C660BC2EDFCFDE3F31F4C3FD33C053
:10B74000BC2E6894B3F8D7CFD53369F580818D329C
:10B7500031F4C061BF016E5F7F4F818105C0BF01C1
:10B760008B32C9F36F5F7F4F80538A30E0F4FB0167
:10B77000B0E8EB16BCE0FB065CF4B701660F771F80
:10B78000660F771FE60EF71EEE0CFF1CE80EF11C8D
:10B79000819180538A3060F3C4FF03C0F194E19437
:10B7A000F1080E0D1F1DCA01B9010F94CA9EC37086
:10B7B000C33009F490584B015C0120E030E0A9014E
:10B7C0000F945BA6882309F43EC0CDE2D7E717FFAC
:10B7D00005C0119501951109C5E1D7E76E01E8E1B2
:10B7E000CE1AD10880E2E82EF12C0DC0FE01259181
:10B7F0003591459154910E191F09C501B4010F945B
:10B800000B9F4B015C01D501C4010E151F0574F798
:10B810002497F594E794CC16DD06A9F78A2F880FB4
:10B820008B2F881F8F3F49F020E030E0A901C50130
:10B83000B4010F945BA6811106C082E290E0909360
:10B840000C1780930B17C501B401DF91CF911F91A5
:10B850000F91FF90EF90DF90CF90BF90AF909F90AF
:10B860008F90089560E070E080EC9FE7EECF2F921C
:10B870003F924F925F926F927F928F929F92AF9280
:10B88000BF92CF92DF92EF92FF920F931F93CF93CD
:10B89000DF93CDB7DEB7A1970FB6F894DEBF0FBE2A
:10B8A000CDBF84EC92E09D8F8C8F81E6282E82E1C3
:10B8B000382E09E216E091E09A8F198EEC8DFD8DFD
:10B8C0008191FD8FEC8F0E948056E82E882309F429
:10B8D00054C1F0905712FA8DFF220E94105B2B0189
:10B8E0003C01F8014082518262827382F98DF3300B
:10B8F00009F045C0DD24D394F11001C0D12C809013
:10B90000100290901102A0901202B090130220E059
:10B9100030E040E85FE3C501B4010F945BA68823E3
:10B9200059F1F11015C020916D1230916E124091B5
:10B930006F1250917012C301B2010F9465A560930C
:10B940003506709336068093370690933806DE2CC2
:10B95000A5019401609135067091360680913706F5
:10B96000909138060F940B9F6093350670933606BE
:10B970008093370690933806D11003C05FC0FF2034
:10B9800089F0F1012081318142815381F801608188
:10B990007181828193810F9466A5F8016083718320
:10B9A00082839383F98DF230D9F58091BB03823085
:10B9B00009F0EEC08CE0E0EAF2E0DE011D960190B5
:10B9C0000D928A95E1F78CE0ECEAF2E0DE01119647
:10B9D00001900D928A95E1F7C0903106D090320621
:10B9E000E0903306F090340620E030E0A901C70172
:10B9F000B6010F945BA687FF52C0CE0101967C0171
:10BA0000D12CF70161917191819191917F010F94F6
:10BA1000D7A68D2D0F94BE17D394F3E0DF12F1CF8C
:10BA2000F98DFF5FF98F8A8D880F8A8F94E0290E38
:10BA3000311C0C5F1F4FF43009F040CF86E40E94A8
:10BA40008056882399F00E94105B6B017C0120E0F6
:10BA500030E0A9010F94EFA7181644F4C0927A02BF
:10BA6000D0927B02E0927C02F0927D02A1960FB60A
:10BA7000F894DEBF0FBECDBFDF91CF911F910F9124
:10BA8000FF90EF90DF90CF90BF90AF909F908F90FE
:10BA90007F906F905F904F903F902F90089520E09F
:10BAA00030E048E453E4C701B6010F94EFA718163D
:10BAB000A4F4CE010D967C01D12CF7016191719116
:10BAC000819191917F010F94D7A68D2D0F94BE1770
:10BAD000D394F3E0DF12F1CFA3CFCE01019699A367
:10BAE00088A3FE013D96FF8FEE8F1B8EE8A1F9A182
:10BAF000C190D190E190F190F9A3E8A3EE8DFF8D74
:10BB00006191719181919191FF8FEE8FA7019601C3
:10BB10000F9465A520E030E048E453E40F9465A657
:10BB20004B015C0120913106309132064091330681
:10BB3000509134060F940B9F2B013C0120E030E024
:10BB4000A901C501B4010F940B9F9B01AC01C70172
:10BB5000B6010F9465A59B01AC01C301B2010F941E
:10BB600066A50F94D7A68B8D0F94BE17FB8DFF5F34
:10BB7000FB8FF33009F0BACF53CFF101808191816F
:10BB8000A281B381F80180839183A283B38348CFDC
:10BB9000EA8DEE0FEA8FF4E02F0E311C0C5F1F4F81
:10BBA00083E0898F8BCE609113177091141790E00A
:10BBB0008A3020F0895A9F4F0D94A6A2C096FCCFE0
:10BBC0002FB784FF1EC0F894909105019260909366
:10BBD00005012FBF2FB785FF19C0F894909105017B
:10BBE0009160909305012FBF86FF15C0459A87FF8E
:10BBF00014C0469A739A85E08A95F1F7000073980D
:10BC00000895F894909105019D7FE1CFF89490916B
:10BC100005019E7FE6CF4598EACF4698EBCF0F937C
:10BC20001F93CF93DF93C82FD62F8A0160FF15C0D3
:10BC30005F9A8AE18A95F1F700C08C2F0E94E05D3F
:10BC4000D1FD04C08C2F82950E94E05DC801DF9178
:10BC5000CF911F910F910C94C6D05F98EACFCF92ED
:10BC6000DF92EF92FF92CF93DF93EC016A017B01A9
:10BC70000F9446A46F3F7F4F8F4F9F4F59F4B701EA
:10BC8000A601CE01DF91CF91FF90EF90DF90CF9092
:10BC90000D9494A4DF91CF91FF90EF90DF90CF901F
:10BCA00008957F928F929F92AF92BF92CF92DF9230
:10BCB000EF92FF920F931F93CF93DF93CDB7DEB731
:10BCC00060970FB6F894DEBF0FBECDBF5C016B016D
:10BCD000742E81E0809378021F930F931F922F930D
:10BCE0008FE494E69F938F930F9400A381E40E94C6
:10BCF00080560F900F900F900F900F900F90882309
:10BD000089F08091BB049091BC04FC01218128370B
:10BD100009F056C040E150E070E060E002960F94F8
:10BD2000C99F5B0183E40E948056882309F44DC0BB
:10BD30000E94E8564B017501CA14DB0408F4760131
:10BD4000C4018E0D9F1DC816D90618F08E159F05CB
:10BD500018F446018E189F0888E50E9480568823B3
:10BD600009F471C02091BB043091BC042F5F3F4F98
:10BD7000CE0101965C01DC01D12CC12CF90180813E
:10BD80002F5F3F4F8823B9F190E1C916D10499F193
:10BD90008032A1F38A3079F190ED980F9A30C8F48F
:10BDA0008295807F9F012E5F3F4F918140ED490F2B
:10BDB0004A30B8F4842B8D93EFEFCE1ADE0ADECF33
:10BDC0000E94105B0F94D7A6ACCF88248A94982C3D
:10BDD000B2CF9FE9980F963058F48295807F8057B4
:10BDE000E1CF4FE9490F463018F49755892BE3CF3F
:10BDF000D194C194D108912C812CC814D90491F00C
:10BE0000F50161915F01C4018E0D9F1DF1E07F1668
:10BE100031F0FC016083FFEF8F1A9F0AEECF0F9481
:10BE200086A4F9CFFF92EF921F930F939F928F9268
:10BE300085E294E69F938F930F9400A30FB6F89436
:10BE4000DEBF0FBECDBF472DB401C70160960FB650
:10BE5000F894DEBF0FBECDBFDF91CF911F910F9140
:10BE6000FF90EF90DF90CF90BF90AF909F908F901A
:10BE70007F900D942D78682F70E090E080E00F9413
:10BE8000CA9E20E030E048E052E40F940B9F20E08F
:10BE900030E040E85FE30F9466A5089582E00F94D8
:10BEA00047186093691270936A1280936B12909393
:10BEB0006C1289E692E10D94333A4F925F926F9241
:10BEC0007F928F929F92AF92BF92CF92DF92EF922A
:10BED000FF920F931F93CF93DF9301E612E1CAE91C
:10BEE000D4E0288139814A815B81F80160817181C8
:10BEF000828193810F9465A54B015C012C813D816A
:10BF00004E815F81F80164817581868197810F94EC
:10BF100065A56B017C01CAE8D4E0288139814A819A
:10BF20005B81C501B4010F940B9F2B013C012C8157
:10BF30003D814E815F81C701B6010F940B9F9B012C
:10BF4000AC01C301B2010F9466A5F801608371834F
:10BF500082839383288539854A855B85C501B40131
:10BF60000F940B9F4B015C012C853D854E855F85B1
:10BF7000C701B6010F940B9F9B01AC01C501B40131
:10BF80000F9466A5F8016483758386839783DF9198
:10BF9000CF911F910F91FF90EF90DF90CF90BF90C6
:10BFA000AF909F908F907F906F905F904F9008958B
:10BFB0004F925F926F927F928F929F92AF92BF92B9
:10BFC000CF92DF92EF92FF920F931F93CF93DF9365
:10BFD00000D000D01F921F92CDB7DEB7DC01CD900C
:10BFE000DD90ED90FC901397C0926F03D092700398
:10BFF000E0927103F092720314960D911D912D91B0
:10C000003C91179709831A832B833C830093770312
:10C01000109378032093790330937A03DB010D9119
:10C020001D912D913C9113970D831E832F8338878B
:10C030000093730310937403209375033093760376
:10C0400014964D905D906D907C90179740927B0375
:10C0500050927C0360927D0370927E03FA016081AE
:10C0600071818281938160939A0470939B04809381
:10C070009C0490939D0484809580A680B7808092D4
:10C080009E0490929F04A092A004B092A10420E08C
:10C0900030E0A9010F945BA68111AAC020E030E036
:10C0A000A901C501B4010F945BA68111A1C0109232
:10C0B000A20420E030E040E85FE3C701B6010F943E
:10C0C0005BA6811121C020E030E0A9016D817E8155
:10C0D0008F8198850F945BA6811116C020E030E017
:10C0E000A90169817A818B819C810F945BA6811162
:10C0F0000BC020E030E040E85FE3C301B2010F94E1
:10C100005BA6882309F478C08091A20482608093A2
:10C11000A204A3019201C701B6010F940B9F4B012A
:10C120005C012D813E814F81588569817A818B81A7
:10C130009C810F940B9F9B01AC01C501B4010F942E
:10C1400065A54B015C01AC019B01C301B2010F94D9
:10C1500065A660938A0470938B0480938C049093FB
:10C160008D046D817E818F8198859058A501940101
:10C170000F9465A660938E0470938F04809390044F
:10C180009093910469817A818B819C819058A5015B
:10C1900094010F9465A66093920470939304809326
:10C1A000940490939504A5019401C701B6010F94DE
:10C1B00065A6609396047093970480939804909377
:10C1C000990428960FB6F894DEBF0FBECDBFDF915D
:10C1D000CF911F910F91FF90EF90DF90CF90BF9084
:10C1E000AF909F908F907F906F905F904F90089549
:10C1F00081E08093A2045DCF80E090E0A0E8BFE3FF
:10C2000080938A0490938B04A0938C04B0938D0444
:10C2100010928E0410928F04109290041092910448
:10C220001092920410929304109294041092950428
:10C230008093960490939704A0939804B0939904E4
:10C24000C0CF4F925F926F927F928F929F92AF92E8
:10C25000BF92CF92DF92EF92FF921F93CF93DF9323
:10C26000CDB7DEB7A8970FB6F894DEBF0FBECDBF2F
:10C2700048E050E06DED7FE0CE0101960F942EA4D2
:10C2800048E050E065ED7FE0CE0109960F942EA4C2
:10C2900048E050E065EE7FE0CE0141960F942EA479
:10C2A00089899A89AB89BC8989A39AA3ABA3BCA3CA
:10C2B0008F3F9F4FAF4FBF4F09F4B1C08D899E890B
:10C2C000AF89B88D8DA39EA3AFA3B8A78F3F9F4F13
:10C2D000AF4FBF4F09F4A3C089809A80AB80BC8068
:10C2E0008FEF88169806A806B80609F498C08D81C5
:10C2F0009E81AF81B885898F9A8FAB8FBC8F8F3F1E
:10C300009F4FAF4FBF4F09F48AC0C984DA84EB84D2
:10C31000FC848FEFC816D806E806F80609F47FC03B
:10C320008D859E85AF85B8898D8F9E8FAF8FB8A381
:10C330008F3F9F4FAF4FBF4F09F471C0298D3A8D8A
:10C340004B8D5C8DC501B4010F9402A82B013C01FB
:10C3500026E636E646E65FE30F945BA611E087FD2E
:10C360000BC02DEC3CEC4CE85FE3C301B2010F9431
:10C37000EFA718160CF010E02D8D3E8D4F8D58A1B3
:10C38000C701B6010F9402A82B013C0126E636E650
:10C3900046E65FE30F945BA687FD7FC02DEC3CEC87
:10C3A0004CE85FE3C301B2010F94EFA718160CF439
:10C3B00074C02DA13EA14FA158A569A17AA18BA15E
:10C3C0009CA10F9402A820E030E040E751E40F94D4
:10C3D000EFA718160CF411E0A5019401C701B601EE
:10C3E0000F940B9F6B017C012D8D3E8D4F8D58A1BD
:10C3F000698D7A8D8B8D9C8D0F940B9F9B01AC0169
:10C40000C701B6010F9466A59F772DEC3CEC4CEC70
:10C410005DE30F94EFA7181614F01123F1F00E94BA
:10C42000A95580E090E0A0E8BFE389839A83AB83BD
:10C43000BC831D821E821F82188619861A861B865F
:10C440001C868D879E87AF87B88B198A1A8A1B8AAC
:10C450001C8A1D8A1E8A1F8A188EAE014F5E5F4F8E
:10C46000BE01675F7F4FCE0101960E94D85FA896FC
:10C470000FB6F894DEBF0FBECDBFDF91CF911F91F5
:10C48000FF90EF90DF90CF90BF90AF909F908F90F4
:10C490007F906F905F904F90089511E08ACFCF9377
:10C4A000DF93CDB7DEB768970FB6F894DEBF0FBE47
:10C4B000CDBF80E090E0A0E8BFE389839A83AB839F
:10C4C000BC831D821E821F82188619861A861B86CF
:10C4D0001C868D879E87AF87B88B198A1A8A1B8A1C
:10C4E0001C8A1D8A1E8A1F8A188EAE014F5E5F4FFE
:10C4F000BE01675F7F4FCE0101960E94D85F6896AC
:10C500000FB6F894DEBF0FBECDBFDF91CF91089577
:10C510008091A2048823D1F00E944F620F945B188F
:10C5200080E00F94471860936112709362128093B9
:10C5300063129093641281E00F9447186093651220
:10C540007093661280936712909368120895809199
:10C5500063049091620489130BC090916104992344
:10C5600039F020911E0630911F068217130639F00C
:10C5700081E09091C403911103C080E0089581E0AF
:10C5800008952091630480911E0690911F0628173C
:10C59000190611F080E208958EE3089582E08093F9
:10C5A0005902809163048F5F8093630484E08093D9
:10C5B00060041092620410926104089580916004F6
:10C5C000843038F58091630490E020911E0630910C
:10C5D0001F062817390744F0019790931F06809390
:10C5E0001E0687E00F94062380911E062091920379
:10C5F00030E02D5F3F4F8217130659F054F09DEF46
:10C60000980F909392038450809362048FEF8093ED
:10C6100060040895E6E9F3E080E2DF011D928A9567
:10C62000E9F70895CF933FB7F894E0910204F091B1
:10C630000304E817F907C9F0C42F9093030480930B
:10C64000020470931F0660931E061092920382E00C
:10C65000809359023FBF222319F080E00F940623F4
:10C66000CC2321F0CF910C940A633FBFCF91089562
:10C67000DC01262F9091DF039730D8F4492F50E04A
:10C68000FA01EE0FFF1FE40FF51FE95AFC4F40912E
:10C690000204509103045183408380911E069F5FE2
:10C6A0009093DF03828341E070E060E0CD010C9461
:10C6B00012630895982F8091DF039817A8F4891BBF
:10C6C0008093DF0390E0FC01EE0FFF1FE80FF91FDE
:10C6D000E95AFC4F6281062E000C770B20E041E006
:10C6E000808191810C94126380E0EACF81E00C9408
:10C6F0005A631F920F920FB60F9211240BB60F922E
:10C700002F933F934F936F937F938F939F93EF93C9
:10C71000FF938091C80084FF12C08091CE00FF91EA
:10C72000EF919F918F917F916F914F913F912F91B9
:10C730000F900BBE0F900FBE0F901F901895409159
:10C74000CE0080911C06813051F720914205309136
:10C750004305C90101968F7799276091440570912F
:10C76000450586179707D9F22E533B4FF9014083B1
:10C770009093430580934205D2CF1F920F920FB63C
:10C780000F9211240BB60F922F933F934F936F93F9
:10C790007F938F939F93EF93FF938091C00084FFCB
:10C7A00012C08091C600FF91EF919F918F917F9170
:10C7B0006F914F913F912F910F900BBE0F900FBE35
:10C7C0000F901F9018954091C60080911C06811112
:10C7D000EACF2091420530914305C90101968F7738
:10C7E0009927609144057091450586179707D9F2FE
:10C7F0002E533B4FF90140839093430580934205AC
:10C80000D2CF80E1E1E6F2E1A0E9B2E001900D9241
:10C810008A95E1F780918E0290918F029093601239
:10C8200080935F1280915D1290915E1290935C12E2
:10C8300080935B1280915912809358128091571205
:10C8400083FB882780F9809356128091551280933C
:10C8500054120895CF93DF9387E696E10E94067AFB
:10C8600085EA94E1892B51F0C7E7D5E1A397CE0182
:10C870000E94067A84E1C53AD807C1F782E894E1BC
:10C880000E94067A8DE594E1DF91CF910C94067AAF
:10C89000CF93DF93C1E6D2E120E030E048EC51E4F1
:10C8A0006C857D858E859F850F9466A56C877D87B9
:10C8B0008E879F8763E373E383E590E4DF91CF91F5
:10C8C0000D94A84960E085EA9FE00F9462A460E0BF
:10C8D0008FE79CE00F9462A480E090E0A0E8BFEBBB
:10C8E00080937E0290937F02A0938002B093810296
:10C8F00082E08093790210927312089580915B1206
:10C9000090915C1220915D1230915E1228173907C8
:10C9100071F090935E1280935D1281E08093CB035F
:10C920000F94010B0F94E07382E08093CB03089582
:10C9300080917312882341F080918E0290918F0232
:10C940009093601280935F120895CF92DF92EF92DE
:10C95000FF92C090FF0DD090000EE090010EF0907D
:10C96000020E8091FE0D882309F44EC020E030E0D5
:10C97000A901C701B6010F94EFA718160CF044C027
:10C980002BED3FE049E450E4C701B6010F940B9F43
:10C99000A70196010F940B9F20E030E040E85EE392
:10C9A0000F940B9F9B01AC0160E070E080E89FE377
:10C9B0000F9465A66B017C016091750270917602FF
:10C9C00064367105A1F0072E000C880B990B0F94AB
:10C9D000CC9E2AE037ED43E25CE30F940B9F9B0172
:10C9E000AC01C701B6010F940B9F6B017C01C09293
:10C9F0001002D0921102E0921202F0921302FF9004
:10CA0000EF90DF90CF900895C12CD12C80E8E82ED4
:10CA10008FE3F82ED1CF8F929F92AF92BF92CF9299
:10CA2000DF92EF92FF9281EF9FE00F94476C6B01D2
:10CA30007C018DEE9FE00F94476C4B015C010F94DD
:10CA4000CD142CE330E040E050E00F94B1A4BA01E3
:10CA5000A901480D591D6A1D7B1D8DEE9FE00F94A5
:10CA600074A4609117067091180680911906909130
:10CA70001A0628EE33E040E050E00F94B1A4BA016A
:10CA8000A9014C0D5D1D6E1D7F1D81EF9FE00F9470
:10CA900074A40F946A16109217061092180610923A
:10CAA000190610921A0680910113813081F4609169
:10CAB00005137091061390E080E00F942F6C109294
:10CAC0000613109205131092081310920713FF908B
:10CAD000EF90DF90CF90BF90AF909F908F90089590
:10CAE000809155121F928F9380913E031F928F93D6
:10CAF000E7EBF3E0428153812CE3249FC001259FA3
:10CB0000900D11249F938F9340815181249FC001E8
:10CB1000259F900D11249F938F9386EE94E69F930B
:10CB20008F930F9400A38DB79EB70A960FB6F89413
:10CB30009EBF0FBE8DBF089588E493E00D942A0D2B
:10CB400020E030E040E752E40F9465A6089510928B
:10CB500077024091390350913A0360913B03709101
:10CB60003C0340937A0250937B0260937C02709363
:10CB70007D0290938F0280938E0288E493E00D945F
:10CB80002A0D1F93CF93DF93182F80917A029091F3
:10CB90007B02A0917C02B0917D0280933903909337
:10CBA0003A03A0933B03B0933C03C0918E02D09113
:10CBB0008F0284E690E090938F0280938E0288E447
:10CBC00093E00F942A0D10937702CE01DF91CF915D
:10CBD0001F910895CF92DF92EF92FF920F931F93D0
:10CBE000CF93DF9390E0EC01CC0FDD1FCC0FDD1F66
:10CBF000FE01E15BF8482591359145915491FE0184
:10CC0000E154F24FC080D180E280F3808E010F5951
:10CC10001D4EC701B6010F9466A5F80160837183AC
:10CC200082839383FE01ED5BF84825913591459110
:10CC300054918E010C5D1D4FC701B6010F9466A57E
:10CC4000F8016083718382839383FE01E95CF84875
:10CC50002591359145915491C85EDD4FC701B601CC
:10CC60000F9466A5688379838A839B83DF91CF9134
:10CC70001F910F91FF90EF90DF90CF90089540E0CB
:10CC800050E0BA018DEE9FE00F9474A440E050E0B4
:10CC9000BA0181EF9FE00F9474A40E94F35670E0F4
:10CCA00060E085E09FE00F9480A470E060E083E0A6
:10CCB0009FE00F9480A470E060E081E09FE00F941B
:10CCC00080A470E060E08FEF9EE00F9480A470E09D
:10CCD00060E083ED9EE00F9480A470E060E080ED62
:10CCE0009EE00F9480A440E050E0BA0188EA9CE006
:10CCF0000D9474A4F89488E19FE00FB6F894A89579
:10CD0000809360000FBE90936000FFCF85EA9FE0A4
:10CD10000F943EA491E0811101C090E0892F089505
:10CD20008091CD03811106C081E090918B039230F8
:10CD300009F080E008958091D71381110AC0809195
:10CD40004212811106C081E090918B03913009F06D
:10CD500080E00895CF93DF93C0917112C1111FC07D
:10CD60008091721281111CC00E949066811118C0BE
:10CD7000D0915E0DD43061F480915D1290915E127D
:10CD8000892B91F48091591290915A12892B61F458
:10CD90000E949B66C82F811103C0C1E0D111C0E081
:10CDA0008C2FDF91CF910895C1E0FACF0E94AA663F
:10CDB000882389F020E030E040E050E4609169127F
:10CDC00070916A1280916B1290916C120F945BA615
:10CDD000881F8827881F08950E949B66811118C0AC
:10CDE0000E949066811114C080917312811110C04D
:10CDF00080915E0D81110BC080910213811107C0DB
:10CE000080917112811104C080917212089581E0A5
:10CE1000089580E1E1E6F2E1A9E2B6E001900D9229
:10CE20008A95E1F708954F925F926F927F928F9269
:10CE30009F92AF92BF92CF92DF92EF92FF920F93A9
:10CE40001F93CF93DF9300D000D01F921F92CDB7D6
:10CE5000DEB720917312222309F473C12091CE030F
:10CE6000223009F46EC12091CE03213011F41092CA
:10CE7000CE032B013C011092551210915812609173
:10CE8000BC037091BD038091BE039091BF030F94CA
:10CE9000DEA6611731F0812F90E090935A128093B3
:10CEA00059120E947E648091541280935512909181
:10CEB000571280915612819589278870892780930F
:10CEC0005712A301920160919C0270919D02809182
:10CED0009E0290919F020F9465A56D837E838F8340
:10CEE0009887CE0105960F94003A1092400220E0F8
:10CEF00030E040E85FEB6091900270919102809188
:10CF00009202909193020F945BA6811120C08091B0
:10CF1000611290916212A0916312B0916412809399
:10CF2000900290939102A0939202B0939302809109
:10CF3000651290916612A0916712B0916812809369
:10CF4000940290939502A0939602B0939702A30146
:10CF5000920160919C0270919D0280919E0290913D
:10CF60009F020F9465A569837A838B839C83E090ED
:10CF70006912F0906A1200916B1210916C1220915C
:10CF800094023091950240919602509197026091DF
:10CF900090027091910280919202909193021F925F
:10CFA0001F921F921F92E2E68E2EE7E29E2EE6E788
:10CFB000AE2EE2E4BE2EFE0131966F010F945A3A76
:10CFC000A301920160919C0270919D0280919E024A
:10CFD00090919F020F9465A569837A838B839C83CC
:10CFE000E0909802F090990200919A0210919B02B1
:10CFF00020919402309195024091960250919702AF
:10D0000060919002709191028091920290919302AE
:10D010001F921F921F921F920F945A3AE09098020B
:10D02000F090990200919A0210919B022091940233
:10D030003091950240919602509197026091900232
:10D040007091910280919202909193021F921F928F
:10D050001F921F92812C912CF8EEAF2EF2E4BF2E7E
:10D06000ACE9CA2EA2E0DA2E0F945A3A0F945B185C
:10D0700011E01093400260914F127091501290E0B5
:10D0800080E00F94CA9E60937A0270937B02809333
:10D090007C0290937D0280915F1290916012909338
:10D0A0008F0280938E0280E1E0E9F2E0A1E6B2E136
:10D0B00001900D928A95E1F70E94096780917902AB
:10D0C0000FB6F894DEBF0FBECDBF811151C0609185
:10D0D00045127091461280914712909148126093C8
:10D0E000EB167093EC168093ED169093EE160F945A
:10D0F00086678091451290914612A0914712B09197
:10D1000048128093491290934A12A0934B12B09305
:10D110004C121093D71360E085EA9FE00F9462A44D
:10D1200060E08FE79CE00F9462A48AE89CE60E948E
:10D130007FDC82E0809379021092731281E0809309
:10D14000420D28960FB6F894DEBF0FBECDBFDF911B
:10D15000CF911F910F91FF90EF90DF90CF90BF90F4
:10D16000AF909F908F907F906F905F904F900895B9
:10D17000813089F68091451290914612A091471214
:10D18000B091481280933E1290933F12A0934012A8
:10D19000B093411210924810109247100E943756D7
:10D1A000BACF3F924F925F926F927F928F929F92EF
:10D1B000AF92BF92CF92DF92EF92FF920F931F93A5
:10D1C000CF93DF933090A204332009F480C08B0109
:10D1D000EC0131FE54C088809980AA80BB80FB019D
:10D1E000C080D180E280F380209177033091780372
:10D1F0004091790350917A03C501B4010F940B9FBC
:10D200002B013C0120917B0330917C0340917D03F5
:10D2100050917E03C701B6010F940B9F9B01AC0197
:10D22000C301B2010F9466A52B013C0120916F034D
:10D23000309170034091710350917203C501B401A4
:10D240000F940B9F4B015C01209173033091740389
:10D250004091750350917603C701B6010F940B9F5F
:10D260009B01AC01C501B4010F9466A56883798365
:10D270008A839B83F801408251826282738230FEEE
:10D2800026C020919A0430919B0440919C045091B7
:10D290009D04688179818A819B810F9466A568834A
:10D2A00079838A839B8320919E0430919F044091CF
:10D2B000A0045091A104F801608171818281938161
:10D2C0000F9466A5F8016083718382839383DF9155
:10D2D000CF911F910F91FF90EF90DF90CF90BF9073
:10D2E000AF909F908F907F906F905F904F903F9006
:10D2F00008952F923F924F925F926F927F928F92FA
:10D300009F92AF92BF92CF92DF92EF92FF920F93D4
:10D310001F93CF93DF9300D000D01F921F92CDB701
:10D32000DEB78C011B01FC0180819181A281B38158
:10D3300089839A83AB83BC83FB0180819181A28125
:10D34000B3818D839E83AF83B887BE016B5F7F4FB0
:10D35000CE0101960E94D168C980DA80EB80FC8002
:10D3600020E030E0A901C701B6010F945BA687FF5A
:10D3700035C019821A821B821C82FF24F3948D808F
:10D380009E80AF80B88420E030E040E850ECC501DA
:10D39000B4010F945BA687FF35C080E090E0A0E861
:10D3A000B0EC8D839E83AF83B887CD80DE80EF8025
:10D3B000F88489809A80AB80BC807090A204711040
:10D3C0004CC0F80180829182A282B382F101C082B6
:10D3D000D182E282F382FF24F39425C020E030E082
:10D3E0004AE753E4C701B6010F94EFA7F12C1816D2
:10D3F00034F680E090E0AAE7B3E489839A83AB83B4
:10D40000BC83BBCF20E030E042E553E4C501B4016A
:10D410000F94EFA718162CF480E090E0A2E5B3E497
:10D42000C0CFF110C2CF8F2D28960FB6F894DEBF73
:10D430000FBECDBFDF91CF911F910F91FF90EF9065
:10D44000DF90CF90BF90AF909F908F907F906F9024
:10D450005F904F903F902F90089570FE1CC02091D8
:10D460009A0430919B0440919C0450919D04C50105
:10D47000B4010F9465A54B015C0120919E0430918D
:10D480009F044091A0045091A104C701B6010F94DC
:10D4900065A56B017C0171FE9ECF20918A043091BD
:10D4A0008B0440918C0450918D04C501B4010F94FC
:10D4B0000B9F2B013C0120918E0430918F044091F1
:10D4C000900450919104C701B6010F940B9F9B01EA
:10D4D000AC01C301B2010F9466A5F80160837183AA
:10D4E0008283938320919204309193044091940419
:10D4F00050919504C501B4010F940B9F4B015C0141
:10D500002091960430919704409198045091990489
:10D51000C701B6010F940B9F9B01AC01C501B4017B
:10D520000F9466A5F101608371838283938353CF47
:10D53000CF93DF930E949C65C1E6D2E180E090E04A
:10D54000A0EAB0E488879987AA87BB8765E575E577
:10D5500085E591E40F945A4E8DEC9CECACE4BEE36F
:10D5600088839983AA83BB8383E393E3A3E7B0EC27
:10D570008C839D83AE83BF8365E672E1CE010E94FA
:10D58000796960E070E086E193E40F945A4E8AE98D
:10D5900099E9A9E1BEE388879987AA87BB8765E5F2
:10D5A00075E585E591E4DF91CF910D945A4ECF92C8
:10D5B000DF92EF92FF92CF93DF93EC01BC016C5F9F
:10D5C0007F4F0E947969C0902C02D0902D02E0908C
:10D5D0002E02F0902F02A7019601688579858A8531
:10D5E0009B850F945BA687FF04C0C886D986EA8610
:10D5F000FB86C0902002D0902102E0902202F090A1
:10D600002302A7019601688579858A859B850F94F9
:10D61000EFA7181624F4C886D986EA86FB86DF9120
:10D62000CF91FF90EF90DF90CF9008952F923F928F
:10D630004F925F926F927F928F929F92AF92BF9222
:10D64000CF92DF92EF92FF920F931F93CF93DF93CE
:10D65000CDB7DEB7A2970FB6F894DEBF0FBECDBF31
:10D660001C0189E296E00E94D76A88E493E00F9457
:10D670002A0D409061125090621260906312709077
:10D680006412C0902906D0902A06E0902B06F090F4
:10D690002C06A7019601C301B2010F945BA681116C
:10D6A0003FC020912D0630912E0640912F065091BB
:10D6B00030066091651270916612809167129091A8
:10D6C00068120F945BA681112BC020E030E040E788
:10D6D00052E460917A0270917B0280917C02909179
:10D6E0007D020F9465A60F9475490E947355A2960A
:10D6F0000FB6F894DEBF0FBECDBFDF91CF911F9163
:10D700000F91FF90EF90DF90CF90BF90AF909F90E0
:10D710008F907F906F905F904F903F902F900895E3
:10D7200060918E0270918F02072E000C880B990B6E
:10D730000F94CC9E20917A0230917B0240917C0222
:10D7400050917D020F940B9F2EE333EC4EE259E390
:10D750000F940B9F6F83788789879A87809109132D
:10D76000882309F40FC1A3019201C701B6010F94E8
:10D7700065A52B013C012091651230916612409104
:10D7800067125091681260912D0670912E0680915B
:10D790002F06909130060F9465A56B877C878D8747
:10D7A0009E87C301B2019F772B853C854D855E85A1
:10D7B0005F770F9466A56B017C0120E030E0A90142
:10D7C0000F94EFA718160CF0DDC020E030E040EF1A
:10D7D00051E4C701B6010F9465A60F9444A60F94B7
:10D7E000DEA67E836D836230710508F4CBC0211400
:10D7F000310409F4C7C02091691230916A12409136
:10D800006B1250916C1260913106709132068091CA
:10D810003306909134060F9465A56F87788B898BBA
:10D820009A8B20916D1230916E1240916F1250912F
:10D83000701260913506709136068091370690918E
:10D8400038060F9465A56B8B7C8B8D8B9E8BAD8181
:10D85000BE81CD01B0E0A0E08F8F98A3A9A3BAA3A9
:10D860002D813E812216330608F08CC0B10190E074
:10D8700080E00F94CA9E6B017C016F8D78A189A115
:10D880009AA10F94CA9E9B01AC01C701B6010F94E7
:10D8900065A66B017C01AC019B016B897C898D893C
:10D8A0009E890F940B9F9B01AC0160916D1270914A
:10D8B0006E1280916F12909170120F9466A5698319
:10D8C0007A838B839C83A70196016F8578898989E8
:10D8D0009A890F940B9F2091691230916A1240919E
:10D8E0006B1250916C120F9466A56F8B788F898F95
:10D8F0009A8FA70196016B857C858D859E850F94F7
:10D900000B9F2091651230916612409167125091E1
:10D9100068120F9466A56B8F7C8F8D8F9E8FA701E9
:10D920009601C301B2010F940B9F209161123091B7
:10D93000621240916312509164120F9466A53F9257
:10D940002F92A1E6B2E1BF93AF938F809884A98410
:10D95000BA84DE0111966D01EF88F88C098D1A8D5D
:10D960002B8D3C8D4D8D5E8D0F945A3A0F900F90FC
:10D970000F900F908091420D8111B7CEBFEF2B1AFF
:10D980003B0A6ECFE0903106F090320600913306EC
:10D990001091340620912D0630912E0640912F06CD
:10D9A000509130066091290670912A0680912B06CD
:10D9B00090912C061F921F92E1E6F2E1FF93EF9304
:10D9C0008F809884A984BA84E5E3CE2EE6E0DE2E2B
:10D9D0000F945A3A0F900F900F900F9086CECF92DF
:10D9E000DF92EF92FF92CF93C0906912D0906A12AB
:10D9F000E0906B12F0906C12A70196010F9466A54F
:10DA00006093691270936A1280936B1290936C12F8
:10DA100083B190913B06911102C084FF26C081E63C
:10DA200092E10E94D76A6091830D7091840D80917C
:10DA3000850D9091860D0F94A8490F945B18A7014E
:10DA400096016091691270916A1280916B129091A7
:10DA50006C120F9465A56B017C01C701B601CF91D3
:10DA6000FF90EF90DF90CF90089515980F945B187A
:10DA700081E00F94E122C82F65E575E585E591E425
:10DA80000F94A8490F945B1882E00F944718A701E0
:10DA900096010F9465A56B017C018C2F0F94E122F8
:10DAA000DCCF8F929F92AF92BF92CF92DF92EF9294
:10DAB000FF924B015C01C0906912D0906A12E09015
:10DAC0006B12F0906C12AC019B01C701B6010F9470
:10DAD000EFA787FF11C0A5019401C701B6010F94FC
:10DAE00065A59F77FF90EF90DF90CF90BF90AF90AC
:10DAF0009F908F900C94EF6CFF90EF90DF90CF9001
:10DB0000BF90AF909F908F9008952F923F924F9229
:10DB10005F926F927F928F929F92AF92BF92CF92BD
:10DB2000DF92EF92FF920F931F93CF93DF9300D07A
:10DB30001F921F92CDB7DEB7D82E2A013B01322E9D
:10DB4000E982FA820B831C830F945B1881E0809337
:10DB50007112FC2CE32CD31010C0ED2CDC100DC086
:10DB600060E070E080EA90E40E94516DFF24F3943D
:10DB7000EE24E3942224239401C02D2C0E94886279
:10DB8000809109138D831092091382E00F94471836
:10DB90006093691270936A1280936B1290936C1267
:10DBA000F1100F94485281E00E94C1658C010E94DF
:10DBB000096710927A0210927B0210927C021092F6
:10DBC0007D02222019F080E00F940C7AEE2019F0EB
:10DBD00081E00F940C7ADD20E9F0411451046104D6
:10DBE0007104C1F0C301B2010F94CC9E9B01AC0142
:10DBF0006091BF0D7091C00D8091C10D9091C20DCB
:10DC00000F9466A560936112709362128093631201
:10DC100090936412332001F189819A81AB81BC8198
:10DC20000097A105B105C1F0BC01CD010F94CC9EB8
:10DC30009B01AC016091C30D7091C40D8091C50D25
:10DC40009091C60D0F9466A560936512709366124D
:10DC50008093671290936812FF2009F499C060E0E6
:10DC600070E080EA90E40E94516D80913906811144
:10DC700002C00F940C7A80913A06811103C081E0B2
:10DC80000F940C7A0E942161E5E0FDE98591959160
:10DC9000A591B491E1E0FDE94591559165917491AB
:10DCA0004093290650932A0660932B0670932C0606
:10DCB00080932D0690932E06A0932F06B0933006E6
:10DCC0006DE276E089E296E00E94D1680E944F62A0
:10DCD00020E030E040E850EC60912D0670912E0677
:10DCE00080912F06909130060F945BA687FF0CC0A1
:10DCF00080E090E0A0E8B0EC80932D0690932E0693
:10DD0000A0932F06B093300680E090E0A6E1B3E444
:10DD100080937A0290937B02A0937C02B0937D0261
:10DD2000109277020F94684860917A0270917B029A
:10DD300080917C0290917D020F9475490F945B183D
:10DD40008091290690912A06A0912B06B0912C066D
:10DD50008093611290936212A0936312B093641245
:10DD600080912D0690912E06A0912F06B09130063D
:10DD70008093651290936612A0936712B093681215
:10DD800081E0809377020F94FD2282E00F940C7A59
:10DD9000CC20E9F081149104A104B104C1F0C501C3
:10DDA000B4010F94CC9E9B01AC016091C70D7091A2
:10DDB000C80D8091C90D9091CA0D0F9466A560930E
:10DDC000691270936A1280936B1290936C120F9485
:10DDD0006848C8010E94A7650F94FD220E94216136
:10DDE0000E945D5FD11007C0311005C08B8D81117D
:10DDF00002C0CC2039F1F11025C09D81992311F189
:10DE000081E0809309130F9447186B017C0180E037
:10DE10000F944718A70196010F94D6919B01AC016E
:10DE20006091691270916A1280916B1290916C12DC
:10DE30000F9465A56093691270936A1280936B12B8
:10DE400090936C1284E10F94A02F0F945B181092A2
:10DE500071120F900F900F900F900F90DF91CF9154
:10DE60001F910F91FF90EF90DF90CF90BF90AF90F8
:10DE70009F908F907F906F905F904F903F902F90EA
:10DE80000895E1E3F3E09FE781918F3731F0DF01FF
:10DE9000119787FF07C08F778C9383E0E933F807EA
:10DEA00099F708959C93F9CF90915902981710F41F
:10DEB0008093590280915A02882339F0E09104043A
:10DEC000F0910504309709F019940895CF93DF93EA
:10DED000CDB7DEB7AE014A5F5F4FFA016191719134
:10DEE000AF0182EF93E00F9485A3DF91CF91089566
:10DEF00062EF73E00D94D6A262EF73E0082E000C7F
:10DF0000990B0D94A6A2CF93C82FC15020F080E2A8
:10DF10000E947C6FFACFCF9108950F931F93CF93F8
:10DF2000DF93EB01142F052F0E947C6FCE010E941E
:10DF3000786F8AE30E947C6FCE010F94FCA19EE073
:10DF4000981B892F0E94836F0F931F9384E092E8A0
:10DF50009F938F930E94666F0F900F900F900F907A
:10DF6000DF91CF911F910F910895CF93C82F862FE6
:10DF7000643008F083E0809330030E947D558C0F5D
:10DF800080932F0344E650E060E08068CF910C94CA
:10DF90000F5E7F928F929F92AF92BF92CF92DF924D
:10DFA000EF92FF920F931F93CF93DF93E09163045F
:10DFB00050916204E51373C0FB01483009F06CC056
:10DFC000C081D0E04901742E6B015C01809159023F
:10DFD000882359F06091600480E00E94B56F0E9430
:10DFE000C162AE01B5010E948D6F809161048823EA
:10DFF00009F455C09091630420911E0630911F06CC
:10E000009217130609F04BC08091DF038730D8F4D4
:10E01000282F30E0F901EE0FFF1FE20FF31FE95A3E
:10E02000FC4F2091020430910304318320838F5FE1
:10E030008093DF03928320E040E070E060E08DEDAC
:10E0400093E70E941263B0929703A0929603D09236
:10E050009A03C092990370929803D0939C03C09343
:10E060009B0390929E0380929D031093A0030093C4
:10E070009F03F092A203E092A103DF91CF911F9141
:10E080000F91FF90EF90DF90CF90BF90AF909F9057
:10E090008F907F900C94CE62C081D18193CF80917C
:10E0A00063048F5F80936304DF91CF911F910F9181
:10E0B000FF90EF90DF90CF90BF90AF909F908F90A8
:10E0C0007F900895CF93DF93EA010E94B56F62EFCE
:10E0D00073E0CE01DF91CF910D94D6A2CF93C42FE0
:10E0E0000E94B56F62EF73E08C2FCC0F990BCF912C
:10E0F0000D94A6A260E080E00E94B56F10922F03FD
:10E10000089540E456E060E081E00E940F5E1092C6
:10E11000300310922F0348E050E06FE770E081E396
:10E1200093E00D9470AA90915A02981709F1809388
:10E130005A028823E9F010921F0610921E061092D0
:10E14000A40583EE93E00F942A0D0F94010B615008
:10E150007109810991096093C5037093C603809387
:10E16000C7039093C8030E94817082E00C94546F9F
:10E170000895CF93C82F1092300310922F0348E0D8
:10E1800050E06FE770E081E393E00F9470AA44E9F8
:10E1900051E162E080E30E940F5E46E950E062E0F8
:10E1A00080E30E940F5E46E950E062E080E30E9457
:10E1B0000F5E46E950E062E080E20E940F5E8091CF
:10E1C000000444E650E060E080620E940F5E84E05C
:10E1D00080932E0344E650E060E08CE00E940F5EE6
:10E1E000C1110E94817044E650E060E086E0CF916A
:10E1F0000C940F5E81E00C94B970CF92DF92FF9285
:10E200000F931F93CF93DF9300D000D01F921F92E4
:10E21000CDB7DEB78A30D9F480913003843018F05E
:10E220008FEF80933003609130036F5F80E00E9436
:10E23000B56F28960FB6F894DEBF0FBECDBFDF9145
:10E24000CF911F910F91FF90DF90CF90089590E8AC
:10E25000980F44E650E061E09A3408F5482F4058A2
:10E26000550B9A0196E0929FA001939F500D1124A7
:10E27000FA01EA5BFA48F490E1E3F3E030E020E0F1
:10E280009FEF6191782F76277F7789F4F901EF5C12
:10E29000FC4F8083F22E44E650E061E08F2D0E9417
:10E2A0000F5E80912F038F5F80932F03C2CF6F3754
:10E2B00009F03CC0F901EF5CFC4F8083922FF92EEE
:10E2C000FA01EF5BFA488E010F5F1F4FD80195915D
:10E2D00088E0182E10FE05900294802D9795881FD7
:10E2E0008D931A94B9F7BF2DE8E0BE02C001112446
:10E2F00044E650E060E080640E940F5E6E01F9E049
:10E30000CF0ED11C44E650E061E0D8018D918D0123
:10E310000E940F5EC016D106A9F780912F0344E634
:10E3200050E060E080680E940F5EB5CF67FF922FDB
:10E330002F5F3F4F2830310509F0A3CF9F3F09F0F1
:10E34000BECFA9CFCF9324E1AC01249FC001259F6C
:10E35000900D112460916D0370916E030F9407A5C9
:10E36000C62F653108F0C4E180916C038C1748F426
:10E370008FEF0E94FD7080916C038F5F80936C0320
:10E38000F3CFCF91089581E090E090936E03809356
:10E390006D030E94A2716CE271E080E090E00D9448
:10E3A000CE0A8F929F92AF92BF92EF92FF920F93FD
:10E3B0001F93CF93DF93CDB7DEB7A0970FB6F89436
:10E3C000DEBF0FBECDBF611571058105910599F4C2
:10E3D00080E3A0960FB6F894DEBF0FBECDBFDF91ED
:10E3E000CF911F910F91FF90EF90BF90AF909F90B2
:10E3F0008F900C94FD7000E0842E912CB12CA12CF8
:10E400009E012F5F3F4F7901A50194010F94B1A4A4
:10E41000F701E00FF11D6083B901CA010F5F6115BB
:10E4200071058105910581F70E0D1F2D111DE01657
:10E43000F10659F0F80182918F018A3020F4805D55
:10E440000E94FD70F4CF895CFBCFA0960FB6F894C4
:10E45000DEBF0FBECDBFDF91CF911F910F91FF9017
:10E46000EF90BF90AF909F908F900895CF92DF92E2
:10E47000EF92FF926B017C01F7FE0BC08DE20E94D0
:10E48000FD70F094E094D094C094C11CD11CE11CA8
:10E49000F11C4AE0C701B601FF90EF90DF90CF90EA
:10E4A0000C94D1710F931F93CF938C01C62FCC2363
:10E4B00059F0F8012491222339F00F5F1F4F849106
:10E4C0000E94FD70C150F3CF8C2F0E94836F8C2F60
:10E4D000CF911F910F9108950F931F93CF93DF93C7
:10E4E0008C01EB010E94817010926C0310936E03FB
:10E4F00000936D0361E080E00E94B56F64E1CE019E
:10E500000E94527262E080E0DF91CF911F910F91E3
:10E510000C94B56FEF92FF920F931F93CF93DF93FD
:10E52000709163043091620473133FC0122FEA01AB
:10E53000062F7C01809159028823D1F00E94C1628C
:10E54000482F6091600480E00E946E7061E1C70115
:10E550000E945272402F6091600493E1981B892FB2
:10E560000E946E7040E26091600483E10E946E70D0
:10E57000809161048823C9F02091630480911E0674
:10E5800090911F062817190681F410925A02812FC4
:10E59000FE01199581E080935A02DF91CF911F917E
:10E5A0000F91FF90EF900C94CE62809163048F5F87
:10E5B00080936304DF91CF911F910F91FF90EF90B3
:10E5C00008950F931F93CF93C82F8B010E94C162B0
:10E5D000482F6091600480E00E946E7062E1C80183
:10E5E0000E9452728C2FCF911F910F910C947C6FCF
:10E5F000CF93DF933091630420916204321321C0E2
:10E60000EB01BC0180915902882319F080E20E943D
:10E61000E172809161048823A1F0209163048091CC
:10E620001E0690911F062817190659F410925A02D7
:10E63000FE01199581E080935A02DF91CF910C94ED
:10E64000CE62809163048F5F80936304DF91CF91EA
:10E6500008953091630420916204321319C0BC0103
:10E6600080915902882319F083E80E94E172809119
:10E670006104882369F02091630480911E069091C3
:10E680001F062817190621F40E9476630C94CE62A7
:10E69000809163048F5F809363040895CF93DF9329
:10E6A000309163042091620432131EC0EB01BC015F
:10E6B00080915902882319F08EE70E94E1728091BF
:10E6C0006104882389F02091630480911E06909153
:10E6D0001F062817190641F460E0CE010E94386336
:10E6E000DF91CF910C94CE62809163048F5F809311
:10E6F0006304DF91CF910895309163042091620407
:10E70000321319C0BC0180915902882319F080E2AC
:10E710000E94E17280916104882369F02091630472
:10E7200080911E0690911F062817190621F40E9459
:10E73000CE6281E00895809163048F5F80936304CB
:10E7400080E008950F931F93CF938C01C62FCC23A5
:10E7500049F0F80181918F01882321F00E94FD701A
:10E76000C150F5CF8C2F0E94836F8C2FCF911F91BA
:10E770000F910895CF93DF93EC018991882319F0CD
:10E780000E94FD70FACFDF91CF9108950E94FD7035
:10E7900090E080E00895109295031092A7050895E7
:10E7A000CF9380919503C1E0811104C0C0E08C2F0C
:10E7B000CF9108950E94CB73FACF8091590288239C
:10E7C00009F452C02091A1033091A20380919D03CE
:10E7D00090919E0321153105D9F040911E0650916C
:10E7E0001F0641155105A1F07CF040919B0350910B
:10E7F0009C034817590741F430939C0320939B03D3
:10E8000010921F0610921E061092A2031092A103EE
:10E8100020919B0330919C0340911E0650911F064E
:10E82000240F351F10921F0610921E062817390755
:10E8300044F080919F039091A003281739070CF4AE
:10E84000C90190939C0380939B0361E080E00E9448
:10E85000B56F40919B0350919C036091960370911A
:10E86000970380E20E948D6F0E94D073882341F14C
:10E87000E0919903F0919A0380919B0390919C03FE
:10E880002091980380832830C9F48091DF03882386
:10E89000B9F081508093DF0390E0FC01EE0FFF1F81
:10E8A000E80FF91FE95AFC4F6281062E000C770B26
:10E8B00020E040E0808191810C9412639183E5CF48
:10E8C00008950E94D07381110C947663089580910D
:10E8D0001E0690911F0697FF07C010921F06109208
:10E8E0001E0687E00F94062380911E0690911F0656
:10E8F000209192032817190619F014F080939203BF
:10E9000080919203809362040E94D073809361048B
:10E9100008958EEF9FE00F943EA48E3F39F091E072
:10E9200020912D03281390E0892F089580E0089509
:10E9300010922D036EEF8EEF9FE00D9462A4853749
:10E9400028E6920709F459C0F8F48E3625E69207B6
:10E9500009F459C050F4833723E69207B1F18536A4
:10E960009446B1F184E694E60895823726E692074C
:10E9700091F1823728E6920709F442C08337954621
:10E9800089F78BEB94E608958C3620E7920731F1F6
:10E9900070F48C362EE6920721F18F362EE6920720
:10E9A00031F184379946F1F689EA94E608958B3679
:10E9B00023E79207F9F0863723E79207A9F08F360D
:10E9C000924781F687E694E608958BEC94E60895E5
:10E9D00083EC94E6089582EB94E6089582EA94E647
:10E9E000089587E994E608958FE894E6089589E804
:10E9F00094E608958EE794E6089587E794E60895EF
:10EA00008EE694E6089583ED94E60895EDE3F5E748
:10EA100085919591A591B4918F3F9F4FAF4FBF4F77
:10EA2000B1F020E031E081E0F90145915591659127
:10EA30007491453A5A45644B7B4409F00895F901B5
:10EA4000349645915491240F351F8F5FEDCF81E0AF
:10EA500008950F931F93811113C010922C031092ED
:10EA60002B0310922D0390912D0398135CC0682FF7
:10EA70008EEF9FE00F9462A481E01F910F910895A3
:10EA8000813089F7E0E0F1E045915591659174910D
:10EA9000453A5A45644B7B4431F7E4E0F1E0A591F7
:10EAA000B491E8E0F1E06591749150E040E030E02D
:10EAB00020E0A417B50729F5261B370B322723279B
:10EAC00032276217730709F0CECFECE0F1E0059131
:10EAD000159125913491EDE3F5E7459155916591B7
:10EAE0007491041715072607370709F0BCCF20E0FB
:10EAF00031E030932C0320932B0391E090932D036E
:10EB0000B2CFFA01E050FF4FE491F0E098E040FD11
:10EB100090E002C0EE0FFF1F9A95E2F72E0F3F1F05
:10EB20004F5F5F4FC6CF80E0A8CF20912D0321110A
:10EB300004C0FC013296CF01089540912B035091FF
:10EB40002C0341155105A9F3FC01259134912F3F68
:10EB5000320779F3F9013896EE0FFF1FE40FF51F26
:10EB600025913491FA01E20FF31F2491222309F336
:10EB7000E2CF8F929F92AF92BF92CF92DF92EF92AD
:10EB8000FF920F931F93CF93DF93E0916304309133
:10EB90006204E31373C0C22F6A017B015C018091A0
:10EBA00059028823A1F10E94C16201E08E3309F06D
:10EBB00000E00C2B802F8270882EE114F10409F400
:10EBC0006FC0E70190E2992E882009F441C0CE0180
:10EBD0000F94FCA114E0180F4EE300FF40E2609197
:10EBE000600480E00E946E7064E1611BC5010E94B8
:10EBF00052728BE50E947C6FCE01882089F10E94C1
:10EC0000786F8DE50E947C6F892D0E947C6F8091CA
:10EC10006104882399F12091630480911E069091EC
:10EC20001F062817190651F5EF28E9F460E0C60120
:10EC30000E943863DF91CF911F910F91FF90EF9069
:10EC4000DF90CF90BF90AF909F908F900C94CE624A
:10EC5000FE0101900020E9F7EC1B13E01E0FBCCF72
:10EC60000E94BA73CECF10925A02C114D10411F08F
:10EC7000F601199581E080935A02DCCF80916304FC
:10EC80008F5F80936304DF91CF911F910F91FF906D
:10EC9000EF90DF90CF90BF90AF909F908F900895AE
:10ECA0008CE798E40E949575EC018EE7982E8CCF46
:10ECB0000F931F93CF93DF938C01EB0187EE9EE4BC
:10ECC0000E9495759F938F938DEF91E89F938F93FB
:10ECD000DF93CF930F9455A3C80FD11D47E050E0A9
:10ECE000B801CE010F942EA41F820F900F900F90A9
:10ECF0000F900F900F90DF91CF911F910F9108957A
:10ED00000F931F93CF93DF93CDB7DEB763970FB603
:10ED1000F894DEBF0FBECDBF309163042091620432
:10ED2000321338C08B01209159022223A9F0BE0171
:10ED30006F5F7F4F0E9458760E94C162482F60919A
:10ED4000600480E00E946E7062E1CE0101960E9434
:10ED5000A2738EE70E947C6F809161048823D1F0BA
:10ED60002091630480911E0690911F0628171906B2
:10ED700089F460E0C8010E9438630E94CE62639605
:10ED80000FB6F894DEBF0FBECDBFDF91CF911F91BC
:10ED90000F910895809163048F5F80936304EFCF98
:10EDA000CF93DF93EC0120E030E04CE852E4609137
:10EDB0006D1270916E1280916F12909170120F947B
:10EDC00066A560936D1270936E1280936F1290938C
:10EDD000701260E070E080EA91E40F94A8490E940C
:10EDE00048640E9481708FEA92E60E949575AC019A
:10EDF00060E080E00E9462708881882339F061E0E1
:10EE000080E00E94B56FCE010E94BA7386EB99E351
:10EE10000E949575AC0162E080E00E94627083E41C
:10EE20009BE20F94E908DF91CF910D945B180F944A
:10EE30001D658F3F11F180E00E9493700E948170E8
:10EE40008BE69AE50E949575AC0161E080E00E9436
:10EE5000627080E20E94FD700F941D65682F70E063
:10EE60006F5F7F4F072E000C880B990B0E94367244
:10EE70000F94CF9D81E00C94937008951F920F9290
:10EE80000FB60F9211240BB60F922F938F939F936F
:10EE9000EF93FF93E0912603E830E8F4F0E0882751
:10EEA000EB5AF8488F4F0D944EA55D7777778277B0
:10EEB0009077A677AF77D277E47780912806811193
:10EEC0000AC08091EE05880F80932503882319F0EE
:10EED00081E080932603FF91EF919F918F912F9175
:10EEE0000F900BBE0F900FBE0F901F901895809142
:10EEF00024038F5F8093240390912503981758F380
:10EF000082E0E7CF83E0809326038FE080932303A2
:10EF10008FEF86BD81E085BD84B58F7E84BDDBCF5C
:10EF2000809123038295807F819588BD8091230302
:10EF3000882321F0815080932303CDCF84E08093F8
:10EF400026038FEF88BD8EEF86BDC5CF85E0809309
:10EF500026038FEF88BD86BD82E085BDBCCF2FEF35
:10EF600028BD809128068111B6CF809124038F5F40
:10EF70008093240390912503891708F4ACCF8091E6
:10EF8000EE0590E08F3791050CF0A5CF86E08093D9
:10EF900026038FE08093230326BD81E085BD84B5E1
:10EFA0008061BCCF809123038295807F819588BD4D
:10EFB000809123038111BECF87E08093260380E8F0
:10EFC00086BD8FEF88BD87CF1092260380E886BD6F
:10EFD0008FEF88BDC1CFCF93C82F682F87E69FE002
:10EFE0000F9462A4CC2319F0CF910D94246D10924C
:10EFF000F1161092FD16CF9108951092B6030F945A
:10F00000010B60930717709308178093091790936B
:10F010000A1708958093220380FD1CC010923E03BE
:10F0200020913E038FEF820F8E3FE8F08091A00089
:10F03000877F8093A0001092AD001092AC009FB724
:10F04000222361F0F8948091020180628093020192
:10F050009FBF08958FEF80933E03E2CFF894809195
:10F0600002018F7DF3CFEFB7F8948091A000886004
:10F070008093A00030E0809172004FEF50E081FF5C
:10F0800004C04091A8005091A900249FC001259F71
:10F09000900D349F900D11246FEF70E00F9407A531
:10F0A0007093AD006093AC00EFBF08951F93CF93B2
:10F0B000DF93D0912203D1FD1DC01091CC03C1E09C
:10F0C00020E030E048E452E460915A0D70915B0D0D
:10F0D00080915C0D90915D0D0F94EFA718160CF0C8
:10F0E000C0E0DE7FCD2B81E0111101C080E0C82B94
:10F0F000C093220380912203DF91CF911F910C9442
:10F100000A78EF92FF920F931F93CF93DF93EC0156
:10F110008B017A010E94655681110BC0A801BE01C6
:10F12000C701DF91CF911F910F91FF90EF900D9448
:10F1300052A4DF91CF911F910F91FF90EF9008950E
:10F140000F931F93CF93DF938C01D62FC72F0F946C
:10F150004CA48F3F980739F46D2F7C2FC8010F9472
:10F160009CA48D2F9C2FDF91CF911F910F9108951B
:10F170000F931F93CF938C01C62F0F943EA48F3F04
:10F1800029F46C2FC8010F9486A48C2FCF911F9166
:10F190000F910895CF93DF93EC010F944CA4BC0121
:10F1A0006F5F7F4FCE01DF91CF910D949CA4CF93E1
:10F1B000DF93EC010F943EA461E0680FCE01DF9174
:10F1C000CF910D9486A42BE0829FC0011124805B17
:10F1D000924F0F944CA421E0019609F420E0822F75
:10F1E0000895CF93DF93C82FD8E0CF5FC8300CF0DD
:10F1F000C0E08C2F0E94E378811103C0D150A9F7A1
:10F20000CFEF8C2FDF91CF91089581EA9DE00F948D
:10F210003EA40E94F17887FD05C0682F81EA9DE039
:10F220000D9462A408950F931F93CF93C82F8B0161
:10F2300060EF74E7823070F069EE74E7843050F06C
:10F2400061EE74E7843031F069ED74E7853011F0D8
:10F2500062ED74E7C8010F94F5A18CEF8C0F82303A
:10F2600028F0C170CF5CF801C6831782CF911F913F
:10F270000F91089561E080EC9FE00F9462A460E03C
:10F280008FEB9FE00F9462A460E08EEB9FE00F9401
:10F2900062A460E08DEB9FE00F9462A460E08CEBD1
:10F2A0009FE00D9462A4CF93C82F82958F700E9427
:10F2B000D35D8C2F8F70CF910C94D35D40913C1215
:10F2C00050913D1290E080E041155105B1F120913F
:10F2D00038123091391290E080E0F901E55BFF4E81
:10F2E000A081A23021F461817281860F971F415065
:10F2F000510919F1F901E25BFF4EA1919F012B54D5
:10F300003041A111FACFF901E55BFF4E2D3EA1E09E
:10F310003A0730F4A191A111E0CF2F5F3F4FF6CF14
:10F320002D3EE1E03E07C9F6EBE4F0E19F012B54EE
:10F330003041A191AA23D1F3D0CF089580913C12FE
:10F3400090913D12181619060CF043C00197909346
:10F350003D1280933C12892BA1F48091471090912B
:10F360004810892B21F410924A1010924910809174
:10F37000491090914A10909339128093381281E08D
:10F38000089580913812909139120396FC01E55B43
:10F39000FF4E208101962111F9CFFC01E55BFF4E64
:10F3A0008D3E21E0920740F441919C012F5F3F4F39
:10F3B0004111E1CFC901F4CFEBE4F0E18D3E21E052
:10F3C0009207C9F6CF018B54904121912223D1F3AA
:10F3D000D2CF80E00895FC0120E03EE2DB014D91B8
:10F3E000BD01403249F0283011F430833196DB0101
:10F3F00011974C91408331962F5F2B3079F7108213
:10F40000089540E050E0BA010D94322AFC012381B6
:10F4100021110D94102C089590911C06911107C094
:10F420009091C00095FFFCCF8093C6000895913065
:10F4300031F49091C80095FFFCCF8093CE000895E1
:10F440008F929F92AF92BF92EF92FF920F931F9372
:10F45000CF93DF93CDB7DEB7A0970FB6F894DEBF9A
:10F460000FBECDBF611571058105910599F480E34B
:10F47000A0960FB6F894DEBF0FBECDBFDF91CF913F
:10F480001F910F91FF90EF90BF90AF909F908F9042
:10F490000C940C7A00E0842E912CB12CA12C9E01AE
:10F4A0002F5F3F4F7901A50194010F94B1A4F7019B
:10F4B000E00FF11D6083B901CA010F5F611571058D
:10F4C0008105910581F70E0D1F2D111DE016F10626
:10F4D00059F0F80182918F018A3020F4805D0E94FA
:10F4E0000C7AF4CF895CFBCFA0960FB6F894DEBF00
:10F4F0000FBECDBFDF91CF911F910F91FF90EF9085
:10F50000BF90AF909F908F900895CF92DF92EF922F
:10F51000FF926B017C01F7FE0BC08DE20E940C7A1A
:10F52000F094E094D094C094C11CD11CE11CF11C57
:10F530004AE0C701B601FF90EF90DF90CF900C94A6
:10F54000207A8F929F92AF92BF92CF92DF92EF92EA
:10F55000FF92CF936B017C01B42E20E030E0A90133
:10F560000F945BA687FF07C08DE20E940C7AF7FA22
:10F57000F094F7F8F094C0E060E070E080E09FE382
:10F58000CB1541F020E030E040E251E40F9465A655
:10F59000CF5FF6CF9B01AC01C701B6010F9466A502
:10F5A0006B017C010F94DEA64B015C014AE00E94D6
:10F5B000207ACC2391F1C501B4010F94CA9E9B011E
:10F5C000AC01C701B6010F9465A56B017C018EE209
:10F5D0000E940C7AC15008F120E030E040E251E492
:10F5E000C701B6010F940B9F4B015C010F94D7A686
:10F5F0006B01770FEE08FF08C701B6010E94857AFC
:10F60000C701B6010F94CC9E9B01AC01C501B401AA
:10F610000F9465A56B017C01DDCFCF91FF90EF903A
:10F62000DF90CF90BF90AF909F908F9008958AE029
:10F630000C940C7A0E940C7A90E080E00895CF93AD
:10F64000DF93EC01FE018491882321F00E940C7A63
:10F650002196F8CFDF91CF910895CF92DF92EF926C
:10F66000FF92C0905A0DD0905B0DE0905C0DF09031
:10F670005D0D83E499E70E941F7B42E0C701B6015C
:10F680000E94A17A8BE399E70E941F7B6091BC03E3
:10F690007091BD038091BE039091BF0341E00E9431
:10F6A000A17AFF90EF90DF90CF900C94177B4F9250
:10F6B0005F926F927F928F929F92AF92BF92CF9202
:10F6C000DF92EF92FF920F931F93CF93DF93CC249F
:10F6D000CA94DC2C76010EEA1FE093E2892E912C6D
:10F6E000A12CB12C412C512C3201D0E0C0E08FEF85
:10F6F000C81609F45DC0C8010F944CA4EC01BC010C
:10F70000990F880B990B0F94CC9E2091730D30911B
:10F71000740D4091750D5091760D0F9465A62B01D7
:10F720003C01C701B6010E94857A87E998E70E94EB
:10F730001F7BC501B4010E94857A87E998E70E9482
:10F740001F7BBE010D2E000C880B990B0E94857A41
:10F7500087E998E70E941F7B20E030E04AE754E405
:10F76000C301B2010F940B9F0F94186585E0880EBA
:10F77000911CA11CB11C0E5F1F4F8FEFC81AD80A35
:10F78000E80AF80A0A3B8FE0180709F0B0CFDF91CA
:10F79000CF911F910F91FF90EF90DF90CF90BF908E
:10F7A000AF909F908F907F906F905F904F90089553
:10F7B0008CE798E40E941F7BB8CF882371F18BE817
:10F7C00098E70E941F7B6091901270E090E080E0CB
:10F7D0000E94857A809190128430D8F01092901215
:10F7E00086E898E70E941F7B8091901290E00F942A
:10F7F00035658091901220915B1230915C123093AC
:10F800005E1220935D120E9496FB0E9448640D9444
:10F810005B188F5F80939012E3CF84E19DE30E9499
:10F82000957570E060E00E94B3CFE5CFCF93DF9392
:10F8300083E898E70E941F7BC1E6D2E16881798165
:10F840008A819B8142E00E94A17A8FE798E70E941B
:10F850001F7B6C817D818E819F8142E00E94A17A15
:10F860008BE798E70E941F7B688579858A859B8551
:10F8700042E00E94A17A87E798E70E941F7B6C858F
:10F880007D858E859F8542E00E94A17A8BED94E66E
:10F890000E941F7B80E00F9439180F94CC9EC7E61E
:10F8A000DDE02C813D814E815F810F9465A642E0B1
:10F8B0000E94A17A83E798E70E941F7B81E00F9462
:10F8C00039180F94CC9E288539854A855B850F941D
:10F8D00065A642E00E94A17A8FE698E70E941F7B0E
:10F8E00082E00F9439180F94CC9E2C853D854E856F
:10F8F0005F850F9465A642E00E94A17A8BE698E7A7
:10F900000E941F7B83E00F9439180F94CC9E2889A6
:10F9100039894A895B890F9465A6DF91CF910D944F
:10F9200018658AE797E70E941F7B60915A0D7091D6
:10F930005B0D80915C0D90915D0D41E00E94A17A7C
:10F9400087E797E70E941F7B60915D1270915E12BE
:10F95000072E000C880B990B0F94CC9E41E00E945F
:10F96000A17A83E797E70E941F7B6091BC037091A7
:10F97000BD038091BE039091BF0341E00E94A17A34
:10F9800080E797E70E941F7B6091591270915A128D
:10F99000072E000C880B990B0F94CC9E41E00E941F
:10F9A000A17A8BE697E70E941F7B60915A0D7091B8
:10F9B0005B0D80915C0D90915D0D41E00E94A17AFC
:10F9C00088E697E70E941F7B60915D1270915E123E
:10F9D000072E000C880B990B0F94CC9E41E00E94DF
:10F9E000A17A84E697E70E941F7B6091F50570E09D
:10F9F00090E080E00E94857A8FE597E70E941F7B68
:10FA00006091EE0570E090E080E00E94857A8BE5E1
:10FA100097E70E941F7B6091850370918603809118
:10FA200087039091880341E00E94A17A0C94177B90
:10FA30000E941F7B0C94177B8F929F92AF92BF9274
:10FA4000CF92DF92EF92FF920F94010B6B017C013A
:10FA500020913202222309F1409178024130E9F0ED
:10FA60008091140290911502A0911602B091170294
:10FA700046015701881A990AAA0ABB0A30E0A8EE83
:10FA8000B3E00F94DEA486169706A806B9066CF0BC
:10FA9000443031F19CF44230D4F4C0921402D0923C
:10FAA0001502E0921602F0921702FF90EF90DF909D
:10FAB000CF90BF90AF909F908F900895453069F799
:10FAC00084EE92EA0E941F7B86E499E706C084EEEA
:10FAD00092EA0E941F7B83E799E70E94187DDDCFA1
:10FAE00084EE92EA0E941F7B8DE599E7F6CFCF93D3
:10FAF00081EA9DE00F943EA4CBE08C9FC0011124CD
:10FB0000805B924F0F944CA48156904F803A9F4057
:10FB1000C8F082E199E70E94187D81EA9DE00F9488
:10FB20003EA48C9FC001112470E060E0805B924F86
:10FB30000F949CA485ED98E70E9458E881E0CF914E
:10FB40000C949370CF9108952F923F924F925F92B1
:10FB50006F927F928F929F92AF92BF92CF92DF92DD
:10FB6000EF92FF920F931F93CF93DF93CDB7DEB742
:10FB7000A4970FB6F894DEBF0FBECDBF0F945B18ED
:10FB80008091420D811117C081E0809372128091A3
:10FB90003906882349F080913A06882329F020917C
:10FBA0003B062F83211120C081E08093531281E70F
:10FBB00099E60F94E766A4960FB6F894DEBF0FBEE1
:10FBC000CDBFDF91CF911F910F91FF90EF90DF900C
:10FBD000CF90BF90AF909F908F907F906F905F90ED
:10FBE0004F903F902F9008958BEA9DE00F943EA494
:10FBF000182F8EE40E948056082F0E9495568E83FF
:10FC0000002329F0873009F4C9C0833029F013306C
:10FC100009F0C3C063E06E8380E090E0A0E8BFE33A
:10FC20008A839B83AC83BD838AEA9DE00F943EA4C4
:10FC3000888F83E40E948056182F0E9495561123C6
:10FC400029F0882319F08B3008F4888F88E50E940A
:10FC50008056882309F4ABC00E94105B20E030E09E
:10FC600048E052E40F9465A520E030E048EB51E411
:10FC70000F9465A56A877B878C879D8789E50E949D
:10FC80008056882309F49CC00E94105B20E030E07D
:10FC900048E052E40F9465A520E030E040EA50E4EB
:10FCA0000F9465A56C8B7D8B8E8B9F8B87E50E9457
:10FCB0008056882309F489C00E94105B2A853B8501
:10FCC0004C855D850F9466A520E030E048E852E45D
:10FCD0000F9466A5698F7A8F8B8F9C8F88E40E9422
:10FCE0008056882309F47AC00E94105B2C893D89D4
:10FCF0004E895F890F9466A520E030E048E852E421
:10FD00000F9466A56D8F7E8F8F8F98A30F94417C83
:10FD100080912C0290912D02A0912E02B0912F0281
:10FD200080930A1390930B13A0930C13B0930D13AD
:10FD30000F94485205EC1FE0C8010F944CA40196A3
:10FD400009F051C00E5F1F4F053D8FE01807A1F766
:10FD5000212CA9E0B3E1BAA3A9A3B987A887512CA4
:10FD6000412C312C042D842D63E00F94EDA4988B4D
:10FD70006884798410E0F889F11137C0812F63E03D
:10FD80000F94EDA4911131C021103FC17E817330D9
:10FD900009F470C08F818E8737C01E836AE979E9C4
:10FDA00089E19FE36A837B838C839D833DCF80E0E1
:10FDB00090E0A0E8BFEF8A879B87AC87BD875ECFC6
:10FDC00060E070E080E89FEF6DCF80E090E0A0E819
:10FDD000BFE7898F9A8FAB8FBC8F80CF60E070E0D8
:10FDE00080E89FE78FCF2F80B4CF60E070E080EC99
:10FDF0009FE7D30111966D937D938D939C931497F8
:10FE0000BE81B330C1F11E86812F0E943B5F4B0142
:10FE10005C01802F0E943B5F6B017C01A501940176
:10FE20006A857B858C859D850F94EFA718160CF449
:10FE30001CC1298D3A8D4B8D5C8DC501B4010F9489
:10FE4000EFA718160CF411C1A70196016C897D89E2
:10FE50008E899F890F94EFA718160CF406C12D8D7B
:10FE60003E8D4F8D58A1C701B6010F94EFA718160C
:10FE70000CF4FBC033941F5F24E0620E711C17303A
:10FE800009F079CF6FEF461A560A888599854C9606
:10FE90009987888797E04916510409F063CF0F943A
:10FEA0001B93A0915D06AF83B091DE03B88781E01C
:10FEB00080935D068AE0830D8093DE0381E00E94DB
:10FEC000546F80E090E0A0EAB0E4809369129093D0
:10FED0006A12A0936B12B0936C1265E575E585E527
:10FEE00091E40F94A84980E00E94C1659CA38BA374
:10FEF000312C832D67E00F94EDA4F82E092F682F85
:10FF000070E07F876E8780FF03C076E0791B072F44
:10FF1000802F63E00F94EDA4911105C08F2D0F94F5
:10FF2000EDA411E0911110E0802F0E943B5F688BDF
:10FF3000798B8A8B9B8B8F2D0E943B5F4B015C01E1
:10FF40008E81833009F099C01111C8C027E0AE85B9
:10FF5000BF852A9FF0012B9FF00D1124E00FF11DAA
:10FF6000EE0FFF1FEE0FFF1FE75FFC4E60E070E03B
:10FF700080EC9FE761837283838394833394E1E30E
:10FF80003E12B7CF80E090E0A0EAB0E4809369121F
:10FF900090936A12A0936B12B0936C1265E575E5AD
:10FFA00085E591E40F94A8490F945B18B1E33B16E3
:10FFB00009F43CC280913D0391E0980F90933D037A
:10FFC000882309F4D3C160E080E00E94E4DC84E38C
:10FFD00096E30E9495750E9458E880E00E94B6E77B
:10FFE00081E0809378028AE89CE60E947FDC2F8182
:10FFF00020935D0668856093DE0382E00E94546F63
:020000021000EC
:100000000F945B1810927212D6CD011103C0112308
:1000100009F4BCCE812F63E00F94F9A4840D952DD3
:10002000911D880F991F8D53904F0F944CA4BC01C4
:10003000990F880B990B0F94CC9E2AE037ED43E281
:100040005CE30F940B9F9B01AC0160910A137091CC
:100050000B1380910C1390910D130F9466A5F3016F
:10006000618372838383948391CEFE85FF2309F499
:1000700002CF222009F4FECEFECE288939894A8992
:100080005B896A857B858C859D850F94EFA7181603
:1000900004F1288939894A895B89698D7A8D8B8D2C
:1000A0009C8D0F945BA687FD14C0A50194016C89FB
:1000B0007D898E899F890F94EFA7181654F0A501AA
:1000C00094016D8D7E8D8F8D98A10F945BA687FF17
:1000D00005C0112309F452CF211050CF10E0A7E042
:1000E0008E859F85A89FF001A99FF00D1124E00F38
:1000F000F11FEE0FFF1FEE0FFF1FE75FFC4E418069
:10010000528063807480C12CD12CE0EAEE2EE0E4B2
:10011000FE2E222051F023E333E343EB5EE3C301E1
:10012000B2010F9466A56B017C01A7019601609155
:10013000691270916A1280916B1290916C120F94F7
:100140005BA687FF10C0C0926912D0926A12E0923B
:100150006B12F0926C1265E575E585E591E40F94FC
:10016000A8490F945B18688979898A899B8960936B
:100170006112709362128093631290936412809262
:10018000651290926612A0926712B092681265E6AC
:1001900072E181E692E10E94796960E070E086E1B7
:1001A00093E40F94A8490F945B188091420D882323
:1001B00039F07F8170935D0688858093DE03FBCCE8
:1001C000812C912C70E2A72E71ECB72E222051F0D9
:1001D0002A813B814C815D81C301B2010F9465A5E9
:1001E0004B015C01488DC501B4010F944B7C81111A
:1001F0000BC082E696E50E9495759F938F930F94AE
:1002000000A30F900F90BECE2091691230916A1218
:1002100040916B1250916C12C701B6010F9465A505
:1002200020E030E0A9010F945BA687FF36C060E0B4
:1002300070E080EA90E46093691270936A12809390
:100240006B1290936C1265E575E585E591E40F946A
:10025000A8490F945B18488DC501B4010F944B7CDD
:10026000882339F22091691230916A1240916B1201
:1002700050916C1260E070E080EA90E40F9465A504
:100280002DEC3CEC4CEC5DE30F945BA687FF05C0C6
:1002900087EE97E70F9427A375CEC0906912D09090
:1002A0006A12E0906B12F0906C122220A1F0A7016C
:1002B0009601C301B2010F9465A59B01AC015F7764
:1002C0006A817B818C819D810F945BA687FF03C02F
:1002D0008EEA97E7DFCF8FEA9FE00F943EA4882352
:1002E00009F440C086EA9FE00F943EA48823D1F130
:1002F00060918503709186038091870390918803B4
:100300000E9411572091730D3091740D4091750D1D
:100310005091760D0F9465A69B01AC01E7E0AE8588
:10032000BF85EA9FC001EB9F900D1124080F191F94
:10033000000F111F000F111F075F1C4EC701B601F0
:100340000F9465A5D80111966D937D938D939C9321
:1003500014978091DE0381508093DE0381E00E9438
:10036000546F0CCE20E030E0A901D8CF85E00F9487
:100370000623C12CD12C90EAE92E90E4F92E80E0DE
:1003800096E30E9495750E9494DE90E080E00E94C2
:10039000ADDD81E00E9470F980E00F94E122182F1A
:1003A00060E070E080E89FEB0E94EF6C81E00F94CA
:1003B000E122C0926912D0926A12E0926B12F0921E
:1003C0006C1265E575E585E591E40F94A8490F94F5
:1003D0005B18812F0F94E12282E00F94471820E0F0
:1003E00030E040EA50E40F94EFA7181644F2EF8192
:1003F000E0935D06F885F093DE0381E00E94937040
:10040000DD24D394DF92812C912C5401CC24C3940D
:10041000E12CF12C870121E040E050E0BA0181E0BD
:100420000E94856DD09253120F90C5CB10923D0360
:100430008BA19CA10E94A765109227061092260608
:1004400080E10E9446D5882391F00E94777D81EA61
:100450009DE00F943EA42BE0829FC0011124805B9D
:10046000924F0F944CA49093270680932606609198
:10047000260670912706072E000C880B990B0F9407
:10048000CC9E90582091730D3091740D4091750D54
:100490005091760D0F9465A60F940E5280EC9FE05C
:1004A0000F943EA491E0813009F090E099834FEBE6
:1004B0005FE06CE4CE0101960E94AF56F82E4EEB41
:1004C0005FE062E5CE0101960E94AF56082F4DEB2A
:1004D0005FE066E4CE0101960E94AF56182F4CEB08
:1004E0005FE062E4CE0101960E94AF56212F110F0A
:1004F000330B082E000C990B5C01A21AB30A8F2D46
:10050000FF0C990B280F391F46E0429F6001439F63
:10051000D00C1124F12CE12C002E000C110B081B27
:10052000190BB701665F7C4E3B01460177E07A8389
:10053000D3012D903D904D905D903D01FD0134978C
:10054000FB87EA87B401092C000C880B990B0F94E8
:10055000CC9E2FE333EC4EE259E30F940B9FA201A4
:1005600091010F9466A5AA85BB856D937D938D93AC
:100570009C931397BA81B150BA83800E911EB1112A
:10058000D7CFCA0CDB1CECE1EE0EF11CF4ECEF163D
:10059000F10439F60F941B938DE40E948056882352
:1005A00009F484C00E9495562E81273009F094C02A
:1005B000882309F491C0BB24B394AA24AA94AB0C59
:1005C00009A11AA1612C8EEF882E8B0C6A2D862D25
:1005D0000F94D95199249394960C81116EC06B2D70
:1005E000862D0F94D951C12CD12C7601712C8823E2
:1005F00081F020E030E0A901D8015D966D917D91F8
:100600008D919C9190970F9466A56B017C01772446
:100610007394682D862D0F94D951882369F0F801C1
:100620007B972081318142815381C701B6010F94AC
:1006300066A56B017C0173946A2D892D0F94D951A5
:10064000882361F0F8012581368147815085C701F3
:10065000B6010F9466A56B017C0173946A2D8FEF30
:10066000860D0F94D951882331F1F80133972081F9
:10067000318142815381C701B6010F9466A56B0198
:100680007C017394672D70E090E080E00F94CC9E25
:100690009B01AC01C701B6010F9465A6D801119664
:1006A0006D937D938D939C93149707C08CEA9DE086
:1006B0000F943EA479CF7110E5CF692C0C5F1F4FCA
:1006C000B7E09B1283CFB394E9A1FAA17C96FAA379
:1006D000E9A3F8E0BF1271CF81E0809309138FE4A2
:1006E0000E948056811103C00E94986A79CC0E94B2
:1006F00095568111F9CF0E949C6572CCEC01F8945B
:100700000F94E80D179A10923906169A10923A062D
:10071000149A87EC92EA0E941F7B86EB98E70E946E
:10072000187D209779F0CE010E94187DBE0185E9E1
:100730009CE00F949CA462E484E99CE00F9486A45E
:100740000E947A66CEEAD8E7F1CF88E493E00F946E
:100750002A0D80913C1290913D12892B79F0E09105
:100760003812F0913912E55BFF4E8081813011F033
:10077000863021F480E99AE60C94187D08958091E2
:100780003C1290913D12892B29F00E94A5830E9472
:100790009E79F5CF109239121092381210924A10A9
:1007A0001092491081E0809353120895EF92FF92C6
:1007B0000F931F93CF93DF9380910913882389F1BF
:1007C00080E498E70E94187D8AE298E70E94187DED
:1007D00089E198E70E94187DC7E0DCE1C15058F13B
:1007E000CD9F7001112401E010E086E198E70E949E
:1007F0001F7BF801EE0FFF1FEE0FFF1FEE0DFF1D19
:10080000EA5FFC4E608171818281938145E00E94A4
:10081000A17A0F5F1F4F0830110539F70E94177B2F
:10082000DDCF8DE498E7DF91CF911F910F91FF907D
:10083000EF900C94187DDF91CF911F910F91FF9055
:10084000EF900895CF92DF92EF92FF926B017C01BF
:10085000C0922703D0922803E0922903F0922A0342
:10086000809143038230B1F420E030E040E950E46D
:10087000C7010F945BA687FF14C08091970D9091DC
:10088000980DA091990DB0919A0D803D9740A105CA
:10089000B10520F5C701B601FF90EF90DF90CF9032
:1008A00008952AE939E949E95EE3C701B6010F94E1
:1008B0005BA687FF0AC020E030E048E351E4C701AF
:1008C000B6010F940B9F6B017C0184E295E70E94B7
:1008D0001F7BC701B6010F941865DCCF2AE939E9FF
:1008E00049E95EE3C701B6010F945BA687FDE3CF3C
:1008F00020E030E040E85EE3C701B6010F940B9FB3
:1009000020E030E048E550E40F9466A5DCCFCF92BC
:10091000DF92EF92FF92CF93909143039817B9F132
:10092000C82FC0902703D0902803E0902903F090AF
:100930002A0320E030E0A901C701B6010F945BA6AD
:10094000882341F0C092BB0DD092BC0DE092BD0D4A
:10095000F092BE0D87E095E70E941F7BC13011F138
:10096000E0F0C23011F1C09343036091BB0D709170
:10097000BC0D8091BD0D9091BE0D0E9422846093AC
:10098000BB0D7093BC0D8093BD0D9093BE0DCF91A8
:10099000FF90EF90DF90CF9008958FEF94E70E9443
:1009A000187DE1CF8BEF94E7FACF87EF94E7F7CF8D
:1009B0000F945B18179AE9E3F6E01082169A1182F9
:1009C000149A80E00E9487848FEF9FEF90937302C8
:1009D000809372022FEF20936F0290933E028093D8
:1009E0003D0220933F029093710280937002909396
:1009F0003C0280933B020895182FF894CDB7DEB7E0
:100A000000D0CF90DF90EF9088E199E20FB6F89494
:100A1000A895809360000FBE909360009FB7F894F4
:100A2000E2E0F1E08081886080839FBF0F94E80D51
:100A300086EB94E70E94187D8EEA94E70E941F7B64
:100A4000612F70E090E080E04AE00E94207A8AEA1C
:100A500094E70E941F7B8E2DB60190E040E10E943A
:100A6000207A86EA94E70E941F7BBE0190E080E036
:100A700040E10E94207A0E94177B40E060E072E231
:100A800090E080E00F942D7880E99AE60E94187D2E
:100A90000E947A66C82F729A682F83E09DE00F94B7
:100AA00062A480910F06882319F08C2F0E94FC8489
:100AB0000E947A661F920F920FB60F92112483E064
:100AC0000E944A851F920F920FB60F92112482E066
:100AD0000E944A8541ED50E065ED73E787E69DE0B1
:100AE0000F94D8A10F94CD390F941F140E94A564C0
:100AF00084EE92EA0E941F7B83EB93E70C94187DAF
:100B000044E050E064E170E087E69DE00F942EA49D
:100B100043E050E065ED73E787E69DE00F941DA28A
:100B2000892B09F05DC0E9E9F4E74591559165919C
:100B3000749188ED90E00E942F5EEDE9F4E7459115
:100B40005591659174918CED90E00E942F5EE1EAE1
:100B5000F4E7649180EE90E00E94B878E2EAF4E76E
:100B60006591749181EE90E00E94A078E4EAF4E748
:100B70006591749183EE90E00E94A078E5E9F4E736
:100B8000459155916591749184ED90E00E942F5E9E
:100B900041E754E760E170E080EB90E00E948178EB
:100BA00041E854E760E170E080EC90E00E948178D9
:100BB00041ED50E064E170E087E69DE00F942EA4E3
:100BC0000E94A5640F94CD390F941F1484EE92EA0D
:100BD0000E941F7B89E993E70E94187D81E00895B8
:100BE0000E946A8564E070E084E190E00E946556AE
:100BF00091E08927089565ED73E787E69DE00F94FE
:100C0000F5A141ED50E064E170E087E69DE00F94CE
:100C100052A484EE92EA0E941F7B89E893E70C9429
:100C2000187DCF93DF93EC018991882319F00E94FE
:100C30000C7AFACFDF91CF9108950E9411860C941F
:100C4000177B2F923F924F925F926F927F928F927B
:100C50009F92AF92BF92CF92DF92EF92FF920F934B
:100C60001F93CF93DF93CDB7DEB7A0970FB6F8945D
:100C7000DEBF0FBECDBF8FE590E00E94EF55882309
:100C800009F4A1C00E9487558F37910561F48091C6
:100C900044059091450590934305809342058AE76A
:100CA00093E70E94187D6E014FE1C40ED11C992478
:100CB00093940E948755181619060CF078C08091FD
:100CC0007312882329F00E949066882309F46FC06C
:100CD0008091930381116BC02091440530914505AB
:100CE00080914205909143058217930711F3F90112
:100CF000EE53FB4F80812F5F3F4F2F773327309389
:100D00004505209344058F3F09F079C08091190370
:100D1000882309F471C090921803109219031F8E52
:100D200018A280901C03882021F280911A038F8FD3
:100D3000F1E0F81518F480911B0388A310921C03AE
:100D40001601822D8C19881508F0B3CFF10111918D
:100D50001F018FE193E00F945F0B17FDF2CF80919D
:100D60004710909148101A3009F44BC11D3009F416
:100D700048C18F3591050CF049C11B3311F4909295
:100D80001E0320911E032111DCCF9C012F5F3F4FDA
:100D900030934810209347102091491030914A1009
:100DA000255B3F4E820F931FFC011383CACF8091B6
:100DB000471090914810181619060CF451C28091F2
:100DC000D713811167C2A0960FB6F894DEBF0FBE8D
:100DD000CDBFDF91CF911F910F91FF90EF90DF90EA
:100DE000CF90BF90AF909F908F907F906F905F90CB
:100DF0004F903F902F9008959092190390CF90912B
:100E00001803992309F458C0893FE9F170F5863F2A
:100E100009F44AC0873F09F443C085E493E70E9480
:100E20001F7B80E493E70E941F7B109117038CE3E4
:100E300093E710FD02C087E393E70E941F7B012F19
:100E4000027082E393E711FD02C08DE293E70E94F6
:100E50001F7B8CE293E70E94187D002349F185E413
:100E600080930B02109218035ACF8A3F41F08B3FB8
:100E7000A1F680911703816080931703CECF8091F4
:100E800017038E7FF9CF10921C0310921803109253
:100E90001703109216031092190310921503BDCF79
:100EA000809117038260E8CF809117038D7FE4CF94
:100EB00090E290930B02D6CF9091190330911703D3
:100EC000992331F1E0911C0330FF49C020911503B3
:100ED000222309F440C091E09E0F90931C03AE2F93
:100EE000B0E0A65EBC4FFFEFFC9340911603442395
:100EF00051F0EE5FE0931C03E92FF0E0E65EFC4F5B
:100F00004083109216032150209315031092190369
:100F1000E0911C0330FF6CC090911503992349F1B7
:100F200021E02E0F20931C03AE2FB0E0A65EBC4F35
:100F30008C9380911603882351F0EE5FE0931C039D
:100F4000E22FF0E0E65EFC4F808310921603915092
:100F500090931503E4CE42E040931503D7CF91E080
:100F60009E0F90931C03F0E0E65EFC4F9FEF908392
:100F7000CDCFA82FAF7030E021E0AF3029F0B0E046
:100F8000A050BE4F3C9120E0482F407F403F59F495
:100F9000226020FF13C09092150321FF0CC0E2E0F5
:100FA000E0931503BCCE82958F70A82FB0E0A050BF
:100FB000BE4F9C91EECF90931603B1CE81E08E0F81
:100FC00080931C03AE2FB0E0A65EBC4F3C933A303A
:100FD00009F4A5CE21FF03C090921503A0CEEE5FC9
:100FE000E0931C03E82FF0E0E65EFC4F908397CE81
:100FF00091E09E0F90931C03F0E0E65EFC4F80832F
:101000008ECE009719F410921E03DDCE0091491088
:1010100010914A10025B1F4E800F911FFC0110823D
:101020001A83098380911E038111FDC0F80180811C
:101030008E3409F084C04AE050E0BE016F5F7F4FFC
:10104000C80101960F94C99F2B013C01E980FA80E9
:10105000F7018081803231F4FFEFEF1AFF0AFA8244
:10106000E982F4CF80913E1290913F12A0914012FC
:10107000B09141120196A11DB11D84159505A605DB
:10108000B70549F044E050E065E773E7C7010F9406
:101090001DA2892BA1F46AE270E0C7010F9495AA02
:1010A0009093BC048093BB04009709F441C0F801FD
:1010B000F12C8E179F07F1F02191F226FACF87ECE1
:1010C00092EA0E941F7B82EF93E60E941F7B609151
:1010D0003E1270913F1280914012909141120E94F5
:1010E000857A0E94177B0E94375610924810109202
:1010F000471069CE0E94A256F816190639F087ECFF
:1011000092EA0E941F7B83ED93E6DFCFE091BB0460
:10111000F091BC041082E980FA8060E773E7C701B0
:101120000F94ECA1892B39F589E396E60E947E8322
:1011300087EC92EA0E941F7B89EA93E6C6CF8981F9
:101140009A81FC012081203221F401969A838983BF
:10115000F6CF6AE270E00F9495AA892B39F087ECFC
:1011600092EA0E941F7B8FE793E6AFCF44244A9414
:10117000542C3201D0CF44E050E06BE673E7C70156
:101180000F941DA25C01F7018081873481F4809166
:10119000610D853061F082E492E10F945F0BF6E01F
:1011A000F093610D60E085EA9FE00F9462A4AB28A4
:1011B00021F080913B12811198CF26E077FC21E04D
:1011C0008091491090914A10FC01E55BFF4E20830D
:1011D00049815A81F801DA0140175107A1F50190C0
:1011E0000020E9F79F01201B310B0396280F391FC0
:1011F0002D3EF1E03F0779F130934A1020934910DA
:1012000080913C1290913D12019690933D128093F3
:101210003C1277FC08C040923E1250923F126092FE
:1012200040127092411210924810109247100E9482
:101230008755892B09F4C7CD8FE590E00E94EF55C3
:1012400081117FCDC0CD6D9161939D01241B350B24
:101250006111F9CFCACF10924A1010924910D0CF25
:101260008091600D60E273E0811102C060ED77E073
:101270008FE193E00F94300B882309F4A0CD1092F6
:101280001E03109248101092471080E693E70E94C8
:10129000187D99CD80916A16882309F494CD8091A8
:1012A000471090914810892B09F08DCD80913C1208
:1012B00090913D12892B11F410921D0312E001E070
:1012C0004091EB165091EC166091ED167091EE1670
:1012D0008091E4169091E516A091E616B091E7167C
:1012E000481759076A077B0708F0C1C080911D03A2
:1012F0008111BDC00F945E6C40916F1650917016B5
:1013000060917116709172164093EB165093EC1623
:101310006093ED167093EE162091471030914810AF
:101320008A3061F08D3051F0833209F487C02F3557
:10133000310524F48F3F980709F087C02115310546
:1013400009F441CD80916A16811103C040E050E05C
:10135000BA018091491290914A12481B590BA091F1
:101360004910B0914A10FD01E55BFF4E10834183A7
:1013700052831396255B3F4EF901EA0FFB1F108243
:10138000A55BBF4EFD0101900020E9F73197EA1BF4
:10139000FB0BF89480913C1290913D120196909332
:1013A0003D1280933C12EC5F8091491090914A105D
:1013B000E80FF92FF11DF0934A10E0934910809146
:1013C0006A16882309F43DC08091EB169091EC16C3
:1013D000A091ED16B091EE168093491290934A12A7
:1013E000A0934B12B0934C12ED3EF14021F41092B9
:1013F0004A1010924910789410921E0310924810CF
:10140000109247104091EB165091EC166091ED163A
:101410007091EE168091E4169091E516A091E61673
:10142000B091E716481759076A077B0700F58FE563
:1014300090E00E94EF55811143CFC5CC00931D036E
:101440007DCF80E090E0DC01C7CFA9014F5F5F4F07
:1014500050934810409347104091491050914A10C2
:10146000455B5F4E240F351FF901838329CF4091DF
:10147000EB165091EC166091ED167091EE1680917E
:10148000E4169091E516A091E616B091E71648177C
:1014900059076A077B0708F496CC0E945E79892B6E
:1014A00009F091CC0F946F658CE693E60E94187D4D
:1014B0000F94CD146B017C010E940B658CE3882E88
:1014C000912CA12CB12CC701B601A50194010F9458
:1014D000B1A4CA01B901A50194010F94B1A47F93ED
:1014E0006F93C701B60120E13EE040E050E00F9469
:1014F000B1A43F932F938CE493E79F938F938E0136
:101500000F5F1F4F1F930F930F9455A384EE92EA22
:101510000E941F7BC8010E941D86C8010E94D3DC67
:101520000F948672109256020FB6F894DEBF0FBE6B
:10153000CDBF8091D813882359F00F94A167809173
:10154000600D882309F43FCC86E00F94A02F3BCC9C
:1015500081E00F94C5728091D8138111EECFEFCF47
:101560000F931F93CF93DF93C82F8091F116813093
:1015700009F449C0823009F45FC00E94EC66811111
:10158000FFC080915D1290915E12009739F4209116
:10159000591230915A12232B09F4F2C040913302B0
:1015A0005091340260913502709136024115510517
:1015B0006105710509F4E4C0892B31F48091591259
:1015C00090915A12892B29F08091AD05882309F456
:1015D0003FC18091600D882321F040EE52E369E223
:1015E00070E08DEA95E00F946B0B882309F4CAC074
:1015F0000F94E80D80E696E30E9495750E9458E8E6
:101600000F941805BFC00F94E56D882309F4B5CF7A
:1016100081E09091FE16911101C080E08093F41654
:101620008091380E9091390E909301178093001796
:1016300082E08093F116A1CF0F94E56D1092F5161C
:101640008091F116823009F098CF8091F6168111C1
:1016500040C0D091FE1681E0D11101C080E0909190
:10166000F416891709F489CF8093F41686EF96E172
:101670000F945F0BDD23B1F18091F216882311F1F5
:101680008091940381111EC0809101138130D1F0AB
:1016900080913E0D90913F0D891B8F7099F40E94AF
:1016A0009B6681110FC080915E0D843059F08FE5EB
:1016B0009FE00F943EA4811105C061E08EE098E3A5
:1016C0000E94386381E08093F51681E0809359028F
:1016D00054CF64E670E086EF96E10F94300B8111F1
:1016E000B8CF4BCF8091F316882379F38091940380
:1016F0008111EBCF80913E0D90913F0D891B8F7032
:1017000021F40E949B66882301F38091731281115A
:10171000DCCF809101138130C1F280915E0D843065
:10172000A1F28FE59FE00F943EA48111CECF8AE312
:1017300095E69F938F9380E295E69F938F930F9406
:1017400000A31092F3161092F21660E070E0CB0145
:101750000F947C6560E070E0CB010E94136785E622
:101760009FE00E94D77881E09FE00E94CA7882E0E3
:101770009DE60F94E7660F900F900F900F90A5CF06
:101780001092AD0580913C1290913D12039714F494
:101790000E94218690913E0D80913F0D981781F017
:1017A0008091610D863061F468E873E182E492E132
:1017B0000F94300B882321F082E492E10F945F0BA9
:1017C0004091440350914503609146037091470353
:1017D000411551056105710509F03FC0409137027F
:1017E000509138026091390270913A0241155105C9
:1017F00061057105A9F088E493E00F946B0B8823D1
:1018000079F090913E0D80913F0D981309C0C11160
:1018100007C0179A10923906169A10923A06149A2F
:10182000C091551290913F0D80913E0D981701F196
:1018300080913F0D9EE6899FF0011124EC55F94FF0
:10184000C08190913E0D981799F08F5F8F70F9CFFE
:101850008DEA95E00F942A0D95CF88E493E00F94DC
:101860006B0B882309F4BACF8AE998E70E947E833C
:10187000CC2309F4BEC080913F0390914003A09116
:101880004103B0914203892B8A2B8B2B81F40F9457
:10189000010B605E7C4F8F4F9F4F60933F037093AF
:1018A00040038093410390934203CFEF0FC00F9406
:1018B000010B00913F0310914003209141033091AF
:1018C0004203601771078207930778F38091B6038C
:1018D000882309F497C0C093650280915F04811149
:1018E00007C081E080935F040F94969710925F0485
:1018F0008091A6058823C9F11092A6054FB7F894E8
:101900008091A405282F082E000C330B37FF03C04D
:10191000319521953109243031050CF476C0982F8A
:1019200087FF02C093E0980F9595959520911E062C
:1019300030911F06290F311D97FD3A9530931F06F0
:1019400020931E06837887FF03C081508C6F8F5FC2
:101950008093A4054FBF86E00F940623809159021F
:10196000811103C081E0809359028091A7058823EB
:1019700061F00E94CB73E0910604F0910704309768
:1019800021F080915A02811119952091CF1330E0F6
:10199000A8EEB3E00F94DEA4AB01BC0180ED93E1AF
:1019A0000F946B0B882399F08091CE1380FD0E94D9
:1019B000917C8091CE1382FD0E94167C8091CE1383
:1019C00081FD0E94706580ED93E10F942A0D809156
:1019D000600D811102C00E941C7D40E355E760E06C
:1019E00070E08CE893E0DF91CF911F910F910D94FF
:1019F0006B0B10923F031092400310924103109220
:101A0000420364CFC0931D0668CF1092A4054FBF58
:101A100080E0A2CFCF93DF93EC010F94433781E0B6
:101A20000E94B08A80E00E94546F209799F0C233E0
:101A3000D10540F062E370E080E090E00F94CE0AC0
:101A4000E297EBCFBE0190E080E00F94CE0AD0E0A9
:101A5000C0E0E3CFDF91CF910895CF93DF93C82FFC
:101A6000DFEF0F94433781E00E94B08A8091FF122C
:101A70008F3FD9F480919412843021F48091971291
:101A80008111EFCF8091D2129091D312019749F733
:101A90008091F9129091FA128932904811F360E026
:101AA00089E290E80F94F274DCCFD093FF12853076
:101AB00039F4CF3FF9F261E08C2F0F942A9ED1CFF9
:101AC0008430C1F6DF91CF910895FF920F931F9359
:101AD000CF93DF93EC01F62E662309F44BC00F94ED
:101AE000FCA18C01C8010E94EF55882309F453C062
:101AF0008091491090914A10FC01E55BFF4E23E074
:101B00002083825B9F4EBE01FF20E9F10F94F5A177
:101B100084EE92EA0E941F7B81E693E60E941F7B7F
:101B20008091491090914A10825B9F4E0E941186CD
:101B30008AE293E70E94187D8091491090914A10A3
:101B40000496080F191F0D3E81E01807F9F0109355
:101B50004A100093491080913C1290913D120196D9
:101B600090933D1280933C12DF91CF911F910F9182
:101B7000FF900895FC0101900020E9F731978F0153
:101B8000081B190BAFCF0F94A9AAC2CF10924A100D
:101B900010924910E0CF87EC92EA0E941F7B81E609
:101BA00093E60E941F7BCE01FF2059F00E941F7B0D
:101BB00085E992EADF91CF911F910F91FF900C94EC
:101BC000187D0E941186F4CFCF93DF933091630488
:101BD00020916204321320C0EB01BC0180915902B4
:101BE000882319F080E20E94E172809161048823C9
:101BF00099F02091630480911E0690911F0628178A
:101C0000190651F4209721F061E0CE010E94658D04
:101C1000DF91CF910C94CE62809163048F5F8093AB
:101C20006304DF91CF9108950F931F93CF93DF93B8
:101C3000D62F8C01C0E0F8018591949161E00E945B
:101C4000658DCF5F0E5F1F4FDC13F5CFDF91CF9116
:101C50001F910F910895CF93DF93CDB7DEB76E97A5
:101C60000FB6F894DEBF0FBECDBF9E012C5D3F4F77
:101C7000F901419151919F016EE170E0CE01019611
:101C80000F9494A360E0CE0101960E94658D6E963C
:101C90000FB6F894DEBF0FBECDBFDF91CF91089590
:101CA0002F923F924F925F926F927F928F929F926C
:101CB000AF92BF92CF92DF92EF92FF920F931F935A
:101CC000CF93DF93CDB7DEB7C356D1090FB6F894E3
:101CD000DEBF0FBECDBF82E0809378020091381244
:101CE00010913912025B1F4E45E050E067EF71E83A
:101CF000C8010F941DA2892B09F09BC18091600D32
:101D0000882309F44DC084EF9EE70F948939882316
:101D100079F08091BD041F928F9384EC95E69F9398
:101D20008F930F9400A30F900F900F900F9008C007
:101D300080EF9EE70F948939882341F010920804C0
:101D400081E0809378020E94A5833AC28DEE9EE7DF
:101D50000F948939882321F18091BB049091BC04B0
:101D600061E003960F944E710F945E6C8C0180912C
:101D70006F1690917016A0917116B09172168093A3
:101D8000EB169093EC16A093ED16B093EE16802F01
:101D90000E940C7A0A30110539F70F946F65D0CF85
:101DA0008DEE91E80F9489398111CACF89EE91E8BF
:101DB0000F948939882321F14091B9035091BA03D6
:101DC0002CE3249FC001259F900D11249F938F9396
:101DD0004091B7035091B803249FC001259F900DF7
:101DE00011249F938F9382EE97E69F938F930F9486
:101DF00000A30F900F900F900F900F900F90A0CF17
:101E000084EE91E80F948939882311F18CE89FE0E2
:101E10000F943EA4811110C061E087E09DE60E940E
:101E2000658D60E085EA9FE00F9462A460E08FE733
:101E30009CE00F9462A484CF813009F081CF0F948D
:101E4000851682E492E10F945F0B0F940D0B78CF0F
:101E50008DED91E80F948939882321F080E00F946B
:101E6000A1956ECF87ED91E80F94893981110E9479
:101E70007A6684ED91E80F9489398823A9F044E1CA
:101E800050E065E17DE0CE0101960F942EA48C898F
:101E9000882329F089EC91E80F9427A351CFCE0134
:101EA00001960F94CDAA4CCF85EC91E80F94893917
:101EB000882329F089EB91E80E94187D41CF85EBBA
:101EC00091E80F948939882319F086E991E8F4CFD5
:101ED00081E991E80F948939882319F00E94987458
:101EE0002FCF8EE891E80F948939882379F081EA21
:101EF0009DE00F943EA42BE0829FC001112470E06E
:101F000060E0805B924F0F9480A41ACF8BE891E839
:101F10000F948939882351F00E94817040E070E06D
:101F200060E084E690E00F94F324D8CF87E891E84E
:101F30000F9489398823E1F086E50E948056882332
:101F400009F4FECE0E94A25611E0892B09F410E09C
:101F50000F945B188091091390E01817190609F483
:101F6000EFCE1093091389E692E10F94333AE8CE4D
:101F700080E891E80F948939882309F4E1CE84E45C
:101F80000E9480568823A1F00E94105B20E030E080
:101F90004AE754E40F940B9F20E030E040E05FE319
:101FA0000F9466A50F94DEA6CB010E94E2E8C8CE8E
:101FB0008CE791E80F948939882349F18091600D6D
:101FC000882329F18091BB049091BC0402969093E0
:101FD000BC048093BB040E94105B6B017C016FEF1B
:101FE00087EA9DE00F9462A420E030E04AE754E4E1
:101FF000C701B6010F940B9F20E030E040E05FE3A3
:102000000F9466A50F94DEA685EA9DE07CCF85EA55
:102010009DE00F944CA4BC0190E080E00F94CA9E18
:1020200020E030E04AE754E40F9465A60F94186569
:1020300087CED8018C91873411F00C94449B109377
:10204000BC040093BB040E94A25690935603809355
:1020500055038B34910509F445C60CF04BC184300F
:10206000910509F4AAC50CF0C5C097FDCFC0029731
:102070000CF0A2C10E943C558C010E94375C60911B
:102080001706709118068091190690911A060F9400
:10209000CA9E6B017C0140906D1250906E12609050
:1020A0006F12709070128090350690903606A09056
:1020B0003706B0903806A5019401C301B2010F9410
:1020C00065A520E030E048EC52E40F940B9F9B01A3
:1020D000AC01C701B6010F94EFA71816D4F4A30101
:1020E0009201C501B4010F9465A520E030E048ECF1
:1020F00052E40F940B9FA70196010F9466A50F94CD
:10210000DEA66093170670931806809319069093C5
:102110001A068091E90D882309F446C188E50E94DA
:102120008056811141C189E50E94805681113CC1D0
:102130008AE50E948056811137C185E40E9480564D
:10214000882309F431C120916D1230916E124091B3
:102150006F12509170126091350670913606809121
:102160003706909138060F9465A56B017C012DEC24
:102170003CEC4CEC5DEB0F945BA687FF07C18091B4
:102180001B0681110C94F9B90F945B1880913506E8
:1021900090913606A0913706B091380680936D1263
:1021A00090936E12A0936F12B09370128DE692E12D
:1021B0000F94003A90911B0681E089270F948A9032
:1021C000CD59DF4F0FB6F894DEBF0FBECDBFDF9104
:1021D000CF911F910F91FF90EF90DF90CF90BF9024
:1021E000AF909F908F907F906F905F904F903F90B7
:1021F0002F9008958531910509F4D9C0FCF48A30F7
